:020000040800F2
:10000000000001108D31040895440308499D000843
:100010009132040891320408913204080000000073
:10002000000000000000000000000000D54A0308A6
:10003000D34A030800000000D14A030851B1000868
:100040009132040891320408913204089132040874
:1000500091320408913204085990010885910108F1
:10006000499101080D910108D1900108F922040875
:10007000E9220408D9220408C9220408B922040884
:10008000A522040891220408913204089132040840
:1000900091320408913204089132040895900108C5
:1000A00081A70008F1A700089132040801A8000800
:1000B000E1A70008D1A70008C1A7000891320408F1
:1000C00091320408913204089132040891320408F4
:1000D000913204081DB30008913204087DB2000873
:1000E0001D900108913204089154030871A700087B
:1000F00091A7000891320408A1A700087D220408F6
:100100009132040891320408B1A700089132040822
:1001100091320408913204088D0C0208710C020817
:100120006922040855220408412204082D220408EB
:10013000192204089132040891320408913204080B
:10014000913204089132040891320408974403085C
:1001500005220408F1210408DD210408DDB10008AE
:100160009132040891320408913204089132040853
:100170009132040891320408913204089132040843
:080180009132040891320408D9
:08018800242D04000100000019
:1001900016000800FC2D0020142E00200000000096
:1001A000400600081D000100D82F0020603000200C
:1001B000000000004806000827000400F82F002077
:1001C00064300020000000004A0600080A020A000D
:1001D000E8300020F8300020000000004E06000843
:1001E0002C00100064330020543300200000000075
:1001F0008D0D02082B00240098330020743300205A
:10020000000000005D0D020829005000803200202F
:10021000BC330020000000000000000009020100C3
:1002200072360020A03600200000000058060008AA
:100230000102050020360020A43600200000000046
:10024000A52E0208000205000C340020AC36002068
:10025000000000000000000003123300933A002069
:10026000603A0020000000005C06000825005A00EB
:10027000AC390020063A0020000000000000000019
:10028000F6110C00A0390020943900200000000075
:100290009006000815007000B438002024390020B2
:1002A00000000000000000002A006000F437002079
:1002B0005438002000000000E95503081400020033
:1002C00040400020B8400020000000009C060008CC
:1002D0001E0004005C410020CC440020000000000F
:1002E0009E06000822000C00FC430020D0440020A1
:1002F00000000000A20600081B00F4006C4500206E
:100300003C54002000000000299802080E02020060
:100310003A4700203055002000000000AE060008DB
:100320002F001100EE530020345500200000000083
:10033000B00600080510060014540020485500209F
:1003400000000000C2060008F5216C00E044002017
:10035000505500200000000081B002080C0024006D
:100360004657002050580020000000006501030897
:100370000E20EA003A5600207458002000000000C9
:1003800055560308130004009857002060590020B8
:1003900000000000C80600080201030025560020E6
:1003A00064590020000000008D01030806001600BB
:1003B0005C640020AC670020000000007556030854
:1003C000FB01010098630020C467002000000000CA
:1003D00085960008FC01090064620020C8670020BF
:1003E00000000000519600080A1012005C5A00201C
:1003F000D467002000000000CC0600083400100084
:1004000088590020E867002000000000115603080A
:1004100012200C0078590020F8670020000000002E
:10042000DE0600080101040048680020C8760020AC
:10043000000000000000000008020900887600208B
:10044000CC7600200000000017820108FF010100A7
:10045000B0760020D876002000000000EA060008F0
:1004600002000C0094760020DC76002000000000E2
:1004700000000000F70106007C760020E8760020EE
:1004800000000000EC06000803010A0024770020A9
:100490003077002000000000F20600081F000E0068
:1004A00090780020647A002000000000FC0600081C
:1004B0000502010078780020747A00200000000016
:1004C0000A0700081A000800A0890020B889002047
:1004D000000000000C070008030001003884002021
:1004E000C0890020000000000000000018102C004F
:1004F00018910020789100200000000049100208A7
:100500000D00340044910020A49100200000000060
:1005100095C1030802020300DC890020D891002065
:1005200000000000000000000C020100CC89002047
:10053000DC910020000000001407000826000E00D7
:1005400018980020089800200000000079B00308E7
:100550000B201000E49500202898002000000000E7
:100560001607000810000300BC9D0020C89D002055
:10057000000000002607000828001000AC9D0020A5
:10058000CC9D002000000000795F020823001000CD
:100590009C9D0020DC9D002000000000458E03088B
:1005A00019000500949D0020EC9D00200000000033
:1005B0002A070008F8110100909D0020F49D0020FA
:1005C0000000000030070008000104008C9D00209E
:1005D000F89D0020000000003207000801200800FC
:1005E000849E0020B09E0020000000003607000816
:1005F00004008000BCBC0020D4C500200000000026
:1006000000000000F9010400FC9E002054C60020F8
:100610000000000009820108FD012400D89E00208E
:1006200058C6002000000000E1970008FE01090004
:10063000E8C700203CC80020000000008D9600089C
:10064000C409000019012828000020030000000050
:100650004A01B400D601000028000000000000009C
:10066000000000000000000000000000000000008A
:10067000000000000000000000000000000000007A
:100680000000000000000000000000000000010069
:100690000000000000000000000000000300000057
:1006A0000100C800141E010064002C012800000095
:1006B000000000000000000000000000000000003A
:1006C00000002000020100000800040000300100CA
:1006D000005A0000000090012C01C80064000000D6
:1006E00000010005465246340000000024010000CD
:1006F0000000040101006C16000000000000000072
:100700000000010000000005000000007E05EA0571
:10071000B405320001002B21231E640002000000FA
:1007200001000A0129000001050000002801000065
:0E073000040090010000E8036400040A0001C8
:10073E000100000001010000747A040838AB0408BF
:10074E000000000000000000847A04088C7A04087F
:10075E000000000001200000907A0408987A040836
:10076E0000000000014000009C7A0408189504085F
:10077E000000000001200000A87A0408B47A0408E2
:10078E000000000004000000B87A040890AD0408D0
:10079E000000000004000000C47A0408A0A90408A8
:1007AE00000000000100000002010000685E0C0065
:1007BE00FF0000000000803F0000803F00000000AE
:1007CE0000000000000000000000803FE001010872
:1007DE0001010000FFFFFFFF000101010100000009
:1007EE0009024300020100C03209040000010202A6
:1007FE000100052400100105240100010424020259
:10080E000524060001070582030800FF0904010004
:10081E00020A0000000705010240000007058102E0
:10082E0040000000FF000000000001FFFF0000007C
:10083E0001010000FFFFFFFFE9CA020800000000EF
:10084E007C020020B8B60408000000000000000082
:10085E00000000000000000038AB0408000000009B
:10086E0000000000040300200400000064B6040829
:10087E000D00000071D20208B41A00200000000022
:10088E0098B004080D00000099D20208A81A0020A2
:10089E000000000098B104080800000000000000ED
:1008AE009C1A00200400000004B104080D00000092
:1008BE0091CB0208901A002000000000A8B1040895
:1008CE0003000000B9D60208841A002000000000C0
:1008DE00C8B6040803000000B9D60208781A002032
:1008EE000000000004AE040801000000000000003B
:1008FE000000000000000000000000000E000000DC
:10090E00000000000000000000000000B8B604085F
:10091E0000000000000000000000000000000000C9
:10092E0038AB0408000000000000000004030020A3
:10093E000400000010B604080300000085D0020871
:10094E006C1A00200800000004B104080D0000001D
:10095E0091CB0208901A002000000000A8B10408F4
:10096E0003000000B9D60208841A0020000000001F
:10097E00C8B6040803000000B9D60208781A002091
:10098E000000000004AE040801000000000000009A
:10099E000000000000000000000000000E0000003B
:1009AE00000000000000000000000000D0B60408A7
:1009BE000000000000000000000000000000000029
:1009CE0038AB040800000000000000000403002003
:1009DE000400000018B6040803000000B9D602088F
:1009EE00C01A00200000000004AE04080100000040
:1009FE0000000000000000000000000000000000E9
:100A0E000E000000000000000000000000000000CA
:100A1E0020700020702D7200000000000000000009
:100A2E0028160020FFFFFFFFFA0000000100000063
:100A3E00010000002D202D2D202D2D2D2D202D2DB2
:100A4E002D0000000000000000000000000000006B
:100A5E0000000000ECAD0408F4AD0408FCAD040881
:100A6E000000000000000000000000000000000078
:100A7E00D9AD040804000000193702080000000078
:100A8E000000000004AE0408010000000000000099
:100A9E000000000000000000000000000E0000003A
:100AAE0000000000000000000000000016470020BB
:100ABE000100C40900000000144700200100C40911
:100ACE0000000000124700200100C40900000000D1
:100ADE00104700200100C409000000000C47002050
:100AEE000100C409000000000E4700200100C409E7
:100AFE00000000000A4700200100C40900000000A9
:100B0E00084700200100C40900000000D055002055
:100B1E000100C80001000000CE55002032003075E3
:100B2E0032000000CD550020055A0500C8550020A2
:100B3E0000FF0100CC55002001000000240300201E
:100B4E00CA550020020000005C660408C75500204C
:100B5E0000FF0100CB5500200100000024030020FF
:100B6E00C9550020020000005C6604080000000069
:100B7E00000000002C030020347800209CFF2C0184
:100B8E00000000009E0000200A00000068660408B5
:100B9E0040580020E0150C1700000000A1000020B6
:100BAE0008000000286A0408A000002005000000CC
:100BBE005C6704086E3600200200000080660408A0
:100BCE007E5700200100FF7F010000007D570020AE
:100BDE00020000008C6604082E5600200300000060
:100BEE009C6604082D560020030000009C66040835
:100BFE002C5700200000F401010000002A570020AD
:100C0E000000F40101000000285700200000F4014C
:100C1E0001000000265700200000F4010100000032
:100C2E002457002000FF010044570020E803D0079E
:100C3E000A00000042570020006401000A00000074
:100C4E003E570020006401003D5700200064010063
:100C5E0043570020006401000A0000003C570020AA
:100C6E00006401000A0000004157002000640100EA
:100C7E000A00000040570020006401000A00000036
:100C8E003F570020006401000A0000003B5700207F
:100C9E0000FF01000A0000003A57002000FF01008B
:100CAE000A000000365600200000F401010000008A
:100CBE00345600200000F4010100000032560020DE
:100CCE000000F40101000000305600200000F40185
:100CDE0001000000365700201400E8030100000058
:100CEE0034570020E8033075010000003357002010
:100CFE0000C801003257002000C801003157002003
:100D0E0000C8010030570020006401000A000000F6
:100D1E002F57002000FF01000A000000735700202B
:100D2E0000C801007257002000C801007157002052
:100D3E0000C801007057002000C801006F57002046
:100D4E0000C801006E57002000C801006D5700203A
:100D5E0000C801006C57002000C801006B5700202E
:100D6E0000C8010038AE04080000000000000000BA
:100D7E00000000000000000048AE0408090000005A
:100D8E0000000000D00300200400000050AE040854
:100D9E000900000000000000C40300200400000051
:100DAE00DCB304080900000000000000B8030020B6
:100DBE0004000000A47B04080900000000000000ED
:100DCE00AC0300200400000058AE04080900000027
:100DDE0000000000A00300200400000060AE040824
:100DEE000900000000000000940300200400000031
:100DFE0068AE04080900000000000000880300200F
:100E0E000400000070AE040809000000000000009D
:100E1E007C0300200400000004AE04080100000062
:100E2E0000000000000000000000000000000000B4
:100E3E000E00000000000000000000000000000096
:100E4E0084AF040800000000000000000000000055
:100E5E000000000038A00408070000000000000099
:100E6E00F40300200000000094AF04080800000006
:100E7E0000000000E803002000000000A0AF0408FE
:100E8E000800000000000000DC030020000000004D
:100E9E0004AE040801000000000000000000000085
:100EAE0000000000000000000E0000000000000026
:100EBE000000000000000000A8AF040800000000C1
:100ECE00000000000000000000000000B8AF0408A1
:100EDE000D000000000000003004002000000000A3
:100EEE00C0AF04080D000000000000002404002024
:100EFE0000000000C8AF040807000000000000005A
:100F0E001C04002000000000D0AF04080D000000FB
:100F1E00000000001004002000000000D8AF0408FC
:100F2E000D0000000000000004040020000000007E
:100F3E00E0AF04080700000000000000FC030020E2
:100F4E000000000004AE04080100000000000000D4
:100F5E000000000000000000000000000E00000075
:100F6E00000000000000000000000000E8AF0408D0
:100F7E000000000000000000000000000000000063
:100F8E0038A004080C00000000000000D25500201C
:100F9E0000000000FCAF04080C0000000000000080
:100FAE00D4550020000000000CB004080C00000016
:100FBE00000000000A560020000000001CB00408CB
:100FCE000C00000000000000FE5500200000000094
:100FDE0030B004080C00000000000000D6550020C0
:100FEE00000000003CB004080C00000000000000EF
:100FFE00D85500200000000044B004080C0000008A
:10100E0000000000DA5500200000000058B004086F
:10101E000C00000000000000DC5500200000000065
:10102E0060B004080C00000000000000DE55002037
:10103E000000000068B004080C0000000000000072
:10104E001C5600200000000080B004080C000000B8
:10105E0000000000E0550020000000008CB00408E5
:10106E000C00000000000000E2550020000000000F
:10107E0034AD04080C00000000000000E455002010
:10108E000000000094B004080C00000000000000F6
:10109E00E655002000000000A0B004080C0000007F
:1010AE0000000000E855002000000000ACB004086D
:1010BE000C00000000000000EA55002000000000B7
:1010CE00B8B004080C00000000000000EC55002031
:1010DE0000000000C4B004080C0000000000000076
:1010EE00EE55002000000000D0B004080C000000F7
:1010FE00000000000256002000000000D8B00408D6
:10110E000C0000000000000000560020000000004F
:10111E00E0B004080C000000000000000E56002095
:10112E0000000000ECB004080C00000000000000FD
:10113E001056002000000000F8B004080C0000005B
:10114E000000000016560020000000001CAF04082E
:10115E000C00000000000000F05500200000000010
:10116E0004B104080C00000000000000F855002037
:10117E00000000000CB104080C000000000000008C
:10118E00F25500200000000018B104080C00000009
:10119E0000000000F45500200000000024B10408F7
:1011AE000C00000000000000F655002000000000BA
:1011BE002CB104080C00000000000000FA550020BD
:1011CE000000000058A004080C0000000000000001
:1011DE00045600200000000038B104080C00000086
:1011EE0000000000FC5500200000000044B104087F
:1011FE000C000000000000000C5600200000000053
:10120E0050B104080C00000000000000065600203B
:10121E000000000058B104080C000000000000009F
:10122E00085600200000000060B104080C00000009
:10123E0000000000125600200000000068B10408F3
:10124E000C000000000000001456002000000000FA
:10125E0004AE0408010000000000000000000000C1
:10126E0000000000000000000E0000000000000062
:10127E00000000000000000070B104080000000033
:10128E0000000000000000000000000080B1040813
:10129E0005000000000000002C5600200000000099
:1012AE0004AE040801000000000000000000000071
:1012BE0000000000000000000E0000000000000012
:1012CE00000000000000000088B1040800000000CB
:1012DE0000000000000000000000000038AB040811
:1012EE000000000000000000E71C002004000000C9
:1012FE0094B104080D0000007D370208840400201C
:10130E000000000064B604080D000000FD3602085F
:10131E00780400200000000098B004080D000000C2
:10132E00E13602086C0400200000000098B10408A9
:10133E00080000000000000060040020040000000F
:10134E0004B104080D000000792F02085404002097
:10135E0000000000A0B10408090000000000000019
:10136E004804002004000000A8B104080300000097
:10137E00B9D602083C0400200000000004AE0408A8
:10138E00010000000000000000000000000000004E
:10139E00000000000E000000000000000000000031
:1013AE0000000000ACB104080000000000000000C6
:1013BE000000000000000000BCB104080D00000099
:1013CE00000000009C04002000000000C4B10408CE
:1013DE000A000000000000009C57002000000000E2
:1013EE00D0B104080A00000000000000A45700203D
:1013FE0000000000D8B104080A0000000000000040
:10140E00AC57002000000000E0B104080800000006
:10141E0000000000900400200000000004AE04084C
:10142E0001000000000000000000000000000000AD
:10143E00000000000E000000000000000000000090
:10144E0000000000E8B104080000000000000000E9
:10145E000000000000000000FCB104080D000000B8
:10146E0000000000B4040020000000000CB20408CC
:10147E000400000015D30208000000000000000068
:10148E0014B204080D00000000000000A8040020A3
:10149E000000000028B2040804000000F1D2020887
:1014AE00000000000000000004AE0408010000006F
:1014BE00000000000000000000000000000000001E
:1014CE000E00000000000000000000000000000000
:1014DE0030B2040800000000000000000000000010
:1014EE000000000044B204080700000000000000E5
:1014FE00F00400200000000050B2040808000000B4
:10150E0000000000E4040020000000005CB20408AB
:10151E000800000000000000D804002000000000B9
:10152E0068B204080800000000000000CC0400208F
:10153E000000000074B20408080000000000000063
:10154E00C00400200000000004AE040801000000EA
:10155E00000000000000000000000000000000007D
:10156E000E0000000000000000000000000000005F
:10157E0080B204080000000000000000E30200201A
:10158E0000000000D07A04080B00000000000000EC
:10159E0068050020000000008CB204080B0000005B
:1015AE00000000005C0500200000000098B2040856
:1015BE000B0000000000000050050020000000009D
:1015CE00A4B204080B000000000000004405002037
:1015DE0000000000B0B204080B0000000000000084
:1015EE003805002000000000D87A04080B00000027
:1015FE00000000002C05002000000000BCB2040812
:10160E000B0000000000000020050020000000007C
:10161E00C8B20408070000000000000018050020F2
:10162E0000000000D0B20408070000000000000017
:10163E001005002000000000DCB204080B000000C2
:10164E00000000000405002000000000E8B20408BD
:10165E000800000000000000F80400200000000058
:10166E0004AE0408010000000000000000000000AD
:10167E0000000000000000000E000000000000004E
:10168E000000000000000000F4B20408000000009A
:10169E0000000000000000000000000008B3040875
:1016AE000800000000000000980500200000000067
:1016BE0014B3040808000000000000008C05002090
:1016CE000000000020B30408080000000000000025
:1016DE0080050020000000002CB304080800000064
:1016EE0000000000740500200000000004AE040895
:1016FE0001000000000000000000000000000000DB
:10170E00000000000E0000000000000000000000BD
:10171E000000000034B304080000000000000000C8
:10172E00E00200200000000044B304080B0000009B
:10173E0000000000E00500200000000050B3040887
:10174E000B00000000000000D40500200000000087
:10175E005CB304080700000000000000CC05002068
:10176E000000000068B3040807000000000000003D
:10177E00C40500200000000074B304080700000038
:10178E0000000000BC0500200000000080B304082B
:10179E000800000000000000B0050020000000005E
:1017AE0088B304080800000000000000A405002013
:1017BE000000000004AE040801000000000000005C
:1017CE000000000000000000000000000E000000FD
:1017DE0000000000000000000000000090B30408AC
:1017EE000000000000000000E002002000000000E9
:1017FE009CB3040807000000000000002C06002027
:10180E0000000000A4B30408070000000000000060
:10181E002406002000000000ACB3040807000000FE
:10182E00000000001C060020000000006C7B040875
:10183E000700000000000000140600200000000059
:10184E00747B040807000000000000000C06002056
:10185E00000000007C7B0408070000000000000070
:10186E000406002000000000B4B3040807000000C6
:10187E0000000000FC05002000000000BCB30408BE
:10188E000700000000000000F4050020000000002A
:10189E00C4B304080700000000000000EC0500209F
:1018AE000000000004AE040801000000000000006B
:1018BE000000000000000000000000000E0000000C
:1018CE00000000000000000000000000000000000A
:1018DE0065CD0208340600202A5600201B000000A9
:1018EE00AC660408295600200A3201002856002052
:1018FE0001FA01002456002000C8010022560020E3
:10190E00E803D007010000004652534B59463400FD
:10191E00C655002000030100C5550020000301003C
:10192E0089CC020865CC0208100700202DCC0208D5
:10193E00EDCB020888070020C5CC0208ADCC02080A
:10194E003C0800207BCD0208C1D20208480B0020C3
:10195E006936020800000000980B002019D4020816
:10196E00E9CF0208740C0020A1CD0208000000008F
:10197E00140D002045CE020815CE0208A00D002041
:10198E00D1CE020819CF0208400E00203857002091
:10199E0001030100E1CD0208B5CD0208580F002069
:1019AE0075CE020839D30208E40F002045CF020895
:1019BE0095D30208AC1000202E5700200103010021
:1019CE00CCB304080000000000000000000000007E
:1019DE0000000000D8B3040808000000000000005A
:1019EE00CC11002000000000E0B304080700000046
:1019FE0000000000C411002000000000F0B3040835
:101A0E000700000000000000BC11002000000000D4
:101A1E00FCB304080700000000000000B411002011
:101A2E000000000008B404080D00000000000000D3
:101A3E00A81100200000000014B4040803000000E8
:101A4E00B9D602089C1100200000000004AE040864
:101A5E000100000000000000000000000000000077
:101A6E00000000000E00000000000000000000005A
:101A7E00000000001CB4040800000000000000007C
:101A8E0000000000000000002CB404080A00000052
:101A9E0000000000E07B04080000000034B40408DD
:101AAE000A00000000000000547A04080000000044
:101ABE003CB404080A000000000000007457002027
:101ACE000000000044B404080A00000000000000FA
:101ADE00D81100200000000004AE04080100000030
:101AEE0000000000000000000000000000000000E8
:101AFE000E000000000000000000000000000000CA
:101B0E004CB40408000000000000000000000000BB
:101B1E000000000058B4040803000000B9D6020803
:101B2E00081200200000000064B404080300000046
:101B3E00B9D60208FC110020000000006CB40408A5
:101B4E0003000000B9D60208F011002000000000CA
:101B5E0074B404080500000000000000C455002005
:101B6E00000000007CB40408070000000000000024
:101B7E00E81100200000000088B4040807000000EF
:101B8E0000000000E01100200000000004AE040878
:101B9E000100000000000000000000000000000036
:101BAE00000000000E000000000000000000000019
:101BBE000000000094B404080000000000000000C3
:101BCE000000000000000000A8B40408030000009C
:101BDE00B9D602082C12002000000000B4B404088C
:101BEE0003000000B9D60208080100200000000022
:101BFE00BCB4040803000000B9D60208201200206D
:101C0E0000000000C4B4040803000000B9D60208A6
:101C1E00141200200000000004AE040801000000B1
:101C2E0000000000000000000000000000000000A6
:101C3E000E00000000000000000000000000000088
:101C4E00D0B40408000000000000000000000000F6
:101C5E0000000000DCB4040807000000E1D3020815
:101C6E00881200200000000028B1040803000000C4
:101C7E00B9D602087C12002000000000E8B4040867
:101C8E0003000000B9D60208701200200000000008
:101C9E00F0B4040803000000B9D602086412002054
:101CAE0000000000F8B4040807000000C5D30208C5
:101CBE005C12002000000000007B040803000000FE
:101CCE00B9D60208501200200000000004B5040826
:101CDE0003000000B9D602084412002000000000E4
:101CEE0010B5040803000000B9D60208381200200F
:101CFE000000000004AE0408010000000000000017
:101D0E000000000000000000000000000E000000B7
:101D1E0000000000000000000000000021CD0208BD
:101D2E00DDCC020890120020B5CF020800000000A2
:101D3E0044130020D1CB0208B5CB0208D0130020EB
:101D4E000000000000000000841400208DCF020867
:101D5E00FDD30208101500201CB504080000000079
:101D6E0000000000000000000000000028B504087C
:101D7E0003000000B9D602081C1600200000000067
:101D8E0030B5040803000000B9D602081016002072
:101D9E000000000050A1040803000000B9D602089C
:101DAE0004160020000000003CB5040803000000EB
:101DBE00B9D60208F81500200000000048B5040846
:101DCE0003000000B9D60208EC1500200000000048
:101DDE0050B504080200000069D50208000000009A
:101DEE000000000058B504080200000069D5020882
:101DFE00010000000000000064B5040802000000AD
:101E0E0069D502080200000000000000000000007A
:101E1E000E000000000000000000000000000000A6
:101E2E00C055002088136F1701000000C255002016
:101E3E0088136F170000000070B504080000000042
:101E4E0000000000000000000000000080B5040843
:101E5E000800000000000000FC1600200400000036
:101E6E008CB504080800000000000000F0160020E9
:101E7E0000000000A8B1040804000000C5D002084C
:101E8E00000000000000000004AE04080100000085
:101E9E000000000000000000000000000000000034
:101EAE000E00000000000000000000000000000016
:101EBE00BE55002088136F170100000070780020B7
:101ECE0088136F170000000049CB020800000000C5
:101EDE000817002094570020010000001C6704081A
:101EEE00727800200100000028670408687800203E
:101EFE00020000003067040892BD002000000000C0
:101F0E000000000090BD0020000000000000000056
:101F1E008EBD002000000000000000008CBD0020DF
:101F2E0000000000000000008ABD0020000000003C
:101F3E000000000088BD002000000000000000002E
:101F4E00201D00200000000000000000BC550020F5
:101F5E00020000003C670408C8B504080000000039
:101F6E0000000000000000000000000080B5040822
:101F7E0008000000000000008C1700200400000084
:101F8E008CB5040808000000000000008017002037
:101F9E0000000000A8B10408040000001DCB0208D8
:101FAE00000000000000000004AE04080100000064
:101FBE000000000000000000000000000000000013
:101FCE000E000000000000000000000000000000F5
:101FDE00D8B504080000000000000000000000005A
:101FEE0000000000E8B504080D0000001DD1020835
:101FFE00BC17002004000000F4B504080D0000001A
:10200E006DCB0208B01700200400000000B60408D3
:10201E000D000000E1D00208A4170020000000000F
:10202E000CB6040803000000A5D002089817002083
:10203E000800000018B6040803000000B9D6020814
:10204E00C01A00200000000004AE040801000000C9
:10205E000000000000000000000000000000000072
:10206E000E00000000000000000000000000000054
:10207E00FCAD04080000000000000000000000009D
:10208E0000000000D9AD04080400000079D1020858
:10209E00000000000000000004AE04080100000073
:1020AE000000000000000000000000000000000022
:1020BE000E00000000000000000000000000000004
:1020CE006CB60408000000000000000000000000D4
:1020DE000000000014A304080D0000000000000022
:1020EE001C180020040000007CB604080800000044
:1020FE0000000000101800200400000088B604083C
:10210E000800000000000000041800200400000079
:10211E0090B604080800000000000000F817002028
:10212E000400000098B6040808000000000000003B
:10213E00EC17002004000000A0B604080800000000
:10214E0000000000E017002004000000A8B60408FC
:10215E000800000000000000D4170020040000005A
:10216E00B0B604080800000000000000C8170020E8
:10217E000400000004AE040801000000000000008E
:10218E000000000000000000000000000E00000033
:10219E0000000000000000000000000035CB020827
:1021AE0000000000281800200000000000000000C1
:1021BE00A0180020000000000000000040190020C0
:1021CE006E78002004000000486704086C78002038
:1021DE00E0150C17000000006B78002008000000CE
:1021EE00286A04086A780020050000005C6704086D
:1021FE000000000000000000901900200100000007
:10220E00006002401060024000000000000B000061
:10221E0000002000000000000000000000600240EE
:10222E002860024000000000060C000000002000A4
:10223E00000000000000000000600240406002400C
:10224E0000000000100D0000000020000000000043
:10225E0000000000006002405860024000000000D4
:10226E00160E00000000200000000000000000001C
:10227E00006002407060024000000000200F00006D
:10228E00000020000000000000000000006002407E
:10229E0088600240000000002610000000002000B0
:1022AE00000000000000000000600240A06002403C
:1022BE0000000000301100000000200000000000AF
:1022CE000000000000600240B86002400000000004
:1022DE00362F00000000200000000000000000006B
:1022EE00006402401064024000000000003800004C
:1022FE0000004000000000000000000000640240EA
:10230E002864024000000000063900000000400072
:10231E000000000000000000006402404064024023
:10232E0000000000103A0000000040000000000015
:10233E0000000000006402405864024000000000EB
:10234E00163B0000000040000000000000000000EE
:10235E00006402407064024000000000203C000057
:10236E000000400000000000000000000064024079
:10237E008864024000000000264400000000400077
:10238E00000000000000000000640240A064024053
:10239E00000000003045000000004000000000007A
:1023AE000000000000640240B8640240000000001B
:1023BE003646000000004000000000000000000053
:1023CE004C69040805080400000000005C6704085E
:1023DE00286A0408486704080000000078690408A9
:1023EE0005080A00000000005C670408286A04085B
:1023FE0068660408000000000000000001020304EB
:10240E00010203040607080900FFFF000000000098
:10241E00AA5505010000012D202D2D202D2D2D2D2D
:10242E00202D2D2D2D0000000000000000000000CA
:10243E00000000000000AA550B010000AA5507017C
:10244E000000AA5509020000000000000100000073
:10245E00C012AA5503009F000403090412010002D2
:10246E0002020040830440570002010203010000F3
:10247E00D9230308C5240308951E030821780208F2
:10248E00452603089D1A0308B91A03081178020895
:10249E0001780208000000000000000008000000A3
:1024AE00017C0208B97B02083D8F02080000000083
:1024BE00DD7702080D7B02088D7B0208757A020813
:1024CE000000000000000000D17702080942030856
:1024DE000742030805420308FF410308FD410308B4
:1024EE000342030801420308194203080B42030882
:1024FE00294303083D43030815430308014303081A
:10250E00ED4203080101D601BD930308000000004F
:10251E000000000084A0040800000000000000007D
:10252E00A1010308A08601000400000000000000C5
:10253E00000000000000000000000000000000008D
:10254E00000000000000000028B10408D89F040815
:10255E0000000000FD2C01087D00000006000000B8
:10256E00000000000000000000000000000000005D
:10257E0000000000000000000000000064B7040826
:10258E000000000000000000690D0108E8030000D3
:10259E00030000000000000000000000000000002A
:1025AE00000000000000000000000000000000001D
:1025BE006CB70408000000000000000049E30308A7
:1025CE0010270000030000000000000000000000C3
:1025DE0000000000000000000000000000000000ED
:1025EE000000000078B70408000000006D98030892
:1025FE00D1EB0008204E0000050000000000000096
:10260E0000000000000000000000000000000000BC
:10261E00000000000000000014A2040800000000EA
:10262E0000000000A5B40008102700000100000003
:10263E00000000000000000000000000000000008C
:10264E000000000000000000000000007CB704083D
:10265E0000000000000000001D960008E8030000C6
:10266E000500000000000000000000000000000057
:10267E00000000000000000000000000000000004C
:10268E0088B704080000000000000000D10603080F
:10269E00204E0000030000000000000000000000BB
:1026AE00000000000000000000000000000000001C
:1026BE000000000098B704080000000000000000B1
:1026CE00D9040308204E00000300000000000000A3
:1026DE0000000000000000000000000000000000EC
:1026EE000000000000000000A8B704080000000071
:1026FE000000000051980008400D03000300000088
:10270E0000000000000000000000000000000000BB
:10271E0000000000000000000000000048A10408B6
:10272E000000000000000000F9CB03081027000095
:10273E00010000000000000000000000000000008A
:10274E00000000000000000000000000000000007B
:10275E00F49F0408000000000000000045AA0208D3
:10276E001027000003000000000000000000000021
:10277E00000000000000000000000000000000004B
:10278E0000000000E49F04080000000000000000AC
:10279E00F1EA000850C30000010000000000000034
:1027AE00000000000000000000000000000000001B
:1027BE0000000000000000001CAF04080000000034
:1027CE000000000059E60008A861000001000000AA
:1027DE0000000000000000000000000000000000EB
:1027EE000000000000000000000000001CA2040811
:1027FE000000000000000000F5B90008A00F000066
:10280E0001000000000000000000000000000000B9
:10281E0000000000000000000000000000000000AA
:10282E00B8B704080000000000000000D5B202088E
:10283E001027000001000000000000000000000052
:10284E00000000000000000000000000000000007A
:10285E000000000050A1040800000000000000006D
:10286E0045C302081A4100000100000000000000EC
:10287E00000000000000000000000000000000004A
:10288E00000000000000000080A20408000000000C
:10289E0000000000FD2D03081027000001000000BD
:1028AE00000000000000000000000000000000001A
:1028BE0000000000000000000000000074AD0408DD
:1028CE00000000000000000049D802081A41000074
:1028DE0001000000000000000000000000000000E9
:1028EE0000000000000000000000000000000000DA
:1028FE00C4B70408000000000000000095A70108FE
:10290E00400D030000000000000000000000000069
:10291E0000000000000000000000000000000000A9
:10292E0000000000CCB7040800000000000000000A
:10293E0031A70108400D0300000000000000000058
:10294E000000000000000000000000000000000079
:10295E000000000000000000D4B7040800000000D2
:10296E0000000000D1370208A0860100030000001D
:10297E000000000000000000000000000000000049
:10298E000000000000000000000000000000803F7A
:10299E000000000000000000000000000000803F6A
:1029AE000000000000000000000000000000000019
:1029BE000000000000000000000000000000000009
:1029CE00000000000000803F00000000000000003A
:1029DE0000000000010000000000803F50010000D8
:1029EE000700000002000000BC22002000000000D2
:1029FE0000000000000000000000000000000000C9
:102A0E0000000000000000000000000000000000B8
:102A1E0000000000000000000000000000000000A8
:102A2E000000000000000000000000000000000098
:102A3E000000000000000000000000000000000088
:102A4E000000000000000000000000004300000035
:102A5E000000000000000000000000000000000068
:102A6E000000000000000000000000004300000015
:102A7E000000000000000000000000000000000048
:102A8E0000000000000000000000000043000000F5
:102A9E000000000000000000000000000000000028
:102AAE0000000000000000000000000043000000D5
:102ABE000000000000000000000000000000000008
:102ACE0000000000000000000000000043000000B5
:102ADE0000000000000000000000000000000000E8
:102AEE000000000000000000000000004300000095
:102AFE0000000000000000000000000000000000C8
:102B0E000000000000000000000000004300000074
:102B1E0000000000000000000000000000000000A7
:102B2E000000000000000000000000002F35040827
:102B3E000B3504080000000045BD0408D5AD04089F
:102B4E00DB840408DB840408DB840408DB840408CB
:102B5E00DB840408DB840408DB840408DB840408BB
:102B6E00DB840408FFFFFFFFFFFFFFFFFFFFFFFFF8
:102B7E00FFFF0000010041534349490000000000DF
:102B8E000000000000000000000000000000000037
:102B9E0000000000000041534349490000000000BE
:102BAE000000000000000000000000000000000017
:0C2BBE000000000000000000010000000A
:108000002DE9F74F6A4CDFF8ACE123880091DEF8E8
:108010000010B4F90480C3EB21125B00C3EBE10351
:10802000B4F9021052435943131308FB03F84FEA03
:10803000A83808EBE12101EB8102B1F5FA3802F131
:1080400080024FEAE1794FEA222349F1FF39B4F97E
:1080500008200193A8FB08AB08FB09F30BEB430BCB
:10806000A161D31702FB09F108FB0311A2FB08234E
:108070000B441F03160347EA1257B4F90A2002FB08
:108080000BF1D3170AFB03130546A2FB0A0119449F
:10809000020A42EA016292194FEA2123E6887B41F3
:1080A000003243F50043A2FB060106FB03114A1010
:1080B000CB1752EA03016FD0B4F91060B4F90E0087
:1080C000F71706FB0BF10AFB0711A6FB0AAB8B4463
:1080D00000FB09F6C11708FB0161A0FB0889894470
:1080E000DEF804104FEA4846C1F5801E4FEA4947C2
:1080F00047EAD8371AEB060AB4F90C8076464BEB00
:10810000070BF71700264FEACE70F90716EB0A06A1
:108110004FEAC80741EA5E0147EB0B0740F6354ED0
:10812000861B61EB0707A6FB0E010EFB07113AF059
:1081300059FEB4F916204E13470B47EAC14702FB1C
:1081400006FED31707FB03EEA2FB07237344564337
:1081500007FB0366A2FB07233344560E46EAC31609
:108160003218B4F914604FEA636747EB01037143B7
:10817000F71700FB0717A6FB00013944C60C46EAB7
:10818000413692194FEAE147B4F912607B41100A77
:1081900040EA0360320112180DB1120A2A60009BF6
:1081A00013B11A46019B136003B0BDE8F08F00BF06
:1081B0007840002090240020704770474FF480538F
:1081C0008382704707B506236A46F72111F0C4F889
:1081D0009DF801309DF800100B4A1B0143EA013362
:1081E0009DF8021043EA111353609DF804309DF886
:1081F00003101B0143EA01339DF8051043EA1113F4
:10820000136003B05DF804FB902400200378022B78
:1082100003D13122742111F059B87047A849A948F7
:10822000A94A2DE9F84F012303700B88128823F027
:1082300040031B041B0C0B800B8823F038031B042A
:1082400052084FEA13430BD042F48072002A92FA8C
:10825000A2F1B1FA81F208BF4FF0FF32013AD20029
:108260001343974A9BB2138013889BB243F0400399
:108270001380964B1B6813B11A689B8853839049EF
:1082800040F2E93302E0002B00F09E810A89013BB5
:1082900012F0020F9BB2F6D005238B8140F2E93336
:1082A000874902E0002B00F08F810A89013B12F020
:1082B000010F9BB2F6D08B89814940F2E93302E08D
:1082C000002B00F0A5810A89013B12F0020F9BB23E
:1082D000F6D000238B8140F2E933794902E0002B8C
:1082E00000F096810A89013B12F0010F9BB2F6D093
:1082F0008B89734940F2E93302E0002B00F084815E
:108300000A89013B12F0020F9BB2F6D006238B8143
:1083100040F2E9336A4902E0002B00F075810A89D6
:10832000013B12F0010F9BB2F6D08B89644940F2F9
:10833000E93302E0002B00F063810A89013B12F06F
:10834000020F9BB2F6D000238B8140F2E9335C49E7
:1083500002E0002B00F054810A89013B12F0010F6A
:108360009BB2F6D08B89DFF86CA155499AF808408A
:1083700040F2E93344F0010402E0002B00F03C81BC
:108380000A89013B12F0020F9BB2F6D004238B81C5
:1083900040F2E9334A4902E0002B00F02D810A89BE
:1083A000013B12F0010F9BB2F6D08B89444940F299
:1083B000E93302E0002B00F01B810A89013B12F037
:1083C000020F9BB2F6D0A4B28C8140F2E9333C4953
:1083D00002E0002B00F00C810A89013B12F0010F32
:1083E0009BB2F6D08B893A4F3B88002B47D0DFF801
:1083F000E890DFF8E880324C4FF0000B072699F840
:10840000015040F2E93302E0002B00F0D5802089D2
:10841000013B10F0020F9BB2F6D0A68140F2E93387
:1084200002E0002B00F0C8802089013B10F0010F12
:108430009BB2F6D0A38940F2E93302E0002B00F0B2
:10844000BF802089013B10F0020F9BB2F6D0ADB285
:10845000A58140F2E93302E0002B00F0B1802089D1
:10846000013B10F0010F9BB2F6D0A3893B8819F8AD
:10847000010F08F8010F0BF1010B9B45BFDB104802
:1084800040F2E93302E0002B00F0AE800289013BAC
:1084900012F0020F9BB2F6D007238381084940F205
:1084A000E93302E0002B00F09F800A89013B12F0C3
:1084B000010F9BB2F6D08B89014840F2E93311E0FD
:1084C000003C00401D3600206C1D0020C4890020A7
:1084D0009C00002090240020133400209B240020C6
:1084E000002B7DD00289013B12F0020F9BB2F7D026
:1084F000FF238381484940F2E93301E0002B6FD02C
:108500000A89013B12F0010F9BB2F7D08B899AF8D0
:108510000840414840F2E93301E0002B5CD0028979
:10852000013B12F0020F9BB2F7D0042383813A493A
:1085300040F2E93301E0002B4ED00A89013B12F0F2
:10854000010F9BB2F7D08B89334840F2E93301E049
:10855000002B3DD00289013B12F0020F9BB2F7D0F5
:10856000A4B22D49848140F2E93301E0002B2FD0E1
:108570000A89013B12F0010F9BB2F7D08B89274B80
:108580001B6813B11A689B881383234A138823F04E
:1085900040031B041B0C1380138823F038031B04B7
:1085A0001B0C138013889BB243F0400313801C4BB9
:1085B00000211970BDE8F88F204610F065FE3AE7FB
:1085C000204610F061FE51E7134810F05DFE73E69F
:1085D000114810F059FED2E70F4810F055FEB3E7EE
:1085E0000D4810F051FE92E70B4810F04DFE63E786
:1085F000094810F049FEF6E6074810F045FED5E6BA
:10860000054810F041FEAEE6034810F03DFE8DE651
:10861000014810F039FE6CE6003C0040C48900209F
:108620001D360020AA490A8822F040022DE9F047B1
:108630001204A84F120C3B880A800A8822F03802E4
:1086400012045B084FEA124200F00D8243F480707E
:1086500090FAA0F10028B1FA81F108BF4FF0FF3184
:108660000139C9000A439A499B4D92B20A800A888F
:1086700092B242F040020A80296811B10A688888E3
:108680005083964A1278012A00F05482C0F00D827D
:10869000022A40F0D481924E082232704FF4C37205
:1086A000DFF844828A48A8F80020028822F04002BD
:1086B0001204120C0280028822F038021204120CFA
:1086C0005BB143F4807090FAA0F30028B3FA83F30F
:1086D00008BF4FF0FF33013BDB0013437C4A9BB2E2
:1086E000138013889BB243F04003138011B10B68D1
:1086F0008A885A83764C4FF010094FF0010A40F2F5
:10870000E93302E0002B00F0A4812289013B12F042
:10871000020F9BB2F6D01FFA89F3A38140F2E9332E
:1087200002E0002B00F095812289013B12F0010F3D
:108730009BB2F6D0A38940F2E93302E0002B00F0AF
:108740008C812289013B12F0020F9BB2F6D0A4F873
:108750000CA040F2E93302E0002B00F07E81228978
:10876000013B12F0010F9BB2F6D0A38909F1010978
:10877000B9F1200FC3D1296811B10B688A881A8317
:10878000534B1A8822F040021204120C1A801A88E5
:1087900022F038021204120C1A801A8892B242F0A7
:1087A00040021A8018883A8820F040000004000C2B
:1087B00018801B8823F038031B0452084FEA134328
:1087C0000BD042F48072002A92FAA2F0B0FA80F242
:1087D00008BF4FF0FF32013AD20013433C4A9BB22C
:1087E000138013889BB243F04003138011B10B68D0
:1087F0008A885A833478364940F2E93302E0002B04
:1088000000F04B810A89013B12F0020F9BB2F6D0B7
:1088100000238B8140F2E9332D4902E0002B00F068
:108820003C810A89013B12F0010F9BB2F6D08B8983
:10883000274940F2E93302E0002B00F032810A8937
:10884000013B12F0020F9BB2F6D0A4B28C8140F231
:10885000E9331F4902E0002B00F023810A89013B24
:1088600012F0010F9BB2F6D08B891E4B18491C7871
:1088700040F2E93302E0002B00F0F7800A89013B67
:1088800012F0020F9BB2F6D002238B8140F2E93343
:108890000F4902E0002B00F0E8800A89013B12F04A
:1088A000010F9BB2F6D08B89094940F2E93302E00F
:1088B000002B00F0DE800A89013B12F0020F9BB210
:1088C000F6D0A4B28C8140F2E933014911E000BF37
:1088D000003C00406C1D0020C4890020D889002085
:1088E0009F000020DF8900209C000020002B00F06A
:1088F000C0800A89013B12F0010F9BB2F6D08B8930
:108900009A4B9B481C7840F2E93302E0002B00F0C0
:10891000B4800289013B12F0020F9BB2F6D0032310
:108920008381934940F2E93302E0002B00F0A580F7
:108930000A89013B12F0010F9BB2F6D08B898C485B
:1089400040F2E93302E0002B00F09B800289013BFA
:1089500012F0020F9BB2F6D0A4B28549848140F296
:10896000E93302E0002B00F08C800A89013B12F011
:10897000010F9BB2F6D08B897E4B7D481C7A40F26A
:10898000E93344F0040401E0002B7ED00289013B6E
:1089900012F0020F9BB2F7D004238381744940F296
:1089A000E93301E0002B70D00A89013B12F0010F7E
:1089B0009BB2F7D08B896E4840F2E93301E0002B7F
:1089C00067D00289013B12F0020F9BB2F7D0A4B22C
:1089D0006749848140F2E93301E0002B59D00A89CC
:1089E000013B12F0010F9BB2F7D08B892B6813B1BA
:1089F0001A689B8813835E4A5F4C13885F4823F094
:108A000040031B041B0C1380138823F038031B0442
:108A10001B0C138013889BB243F040031380B8F8FB
:108A2000002000213BF031FE2378D3B1544B1B785A
:108A3000002B00F0858000232370BDE8F087514EA5
:108A4000327812F0400F0CBF4FF4C3724FF4F07243
:108A500026E6204610F018FC6DE6204610F014FCC7
:108A600084E6BDE8F0871946FCE5414810F00CFCAF
:108A70001AE73F4810F008FC42E73D4810F004FCBC
:108A80005DE73B4810F000FC76E7394810F0FCFB4E
:108A900091E7374810F0F8FBA8E7354810F0F4FBF1
:108AA000C6E6334810F0F0FBDFE6314940F2E93327
:108AB00001E0002B55D00A89013B12F0020F9BB256
:108AC000F7D0A0238B8140F2E933294901E0002B44
:108AD00047D00A89013B12F0010F9BB2F7D08B8976
:108AE000234940F2E93301E0002B35D00A89013BEC
:108AF00012F0020F9BB2F7D000238B8140F2E933D2
:108B00001B4900E043B30A89013B12F0010F9BB2FD
:108B1000F8D08B89D8B200F00603022B194E03D08F
:108B200000F00503012B11D03B8829680822327020
:108B30005B08B3E5134E482232704FF4F072AFE594
:108B4000FFF76CFB00232370BDE8F0873B882968A2
:108B5000482232705B08F0E7054810F095FBC0B280
:108B6000D9E7034810F090FBBAE700BFE089002086
:108B7000003C004090240020000000209C240020A5
:108B80001D3600209F0000209F49A04A2DE9F84F84
:108B9000012313700B889E4A23F040031B041B0C17
:108BA00012880B800B8823F038031B0452084FEA0D
:108BB00013430BD042F48072002A92FAA2F1B1FA68
:108BC00081F208BF4FF0FF32013AD20013438E4AC0
:108BD0009BB2138013889BB243F0400313808D4BEC
:108BE0001B6813B11A689B885383874940F2E933A5
:108BF00002E0002B00F090810A89013B12F0020F85
:108C00009BB2F6D080238B8140F2E9337E4902E0AB
:108C1000002B00F081810A89013B12F0010F9BB209
:108C2000F6D08B89784940F2E93302E0002B00F05E
:108C300077810A89013B12F0020F9BB2F6D0002324
:108C40008B8140F2E933704902E0002B00F068812B
:108C50000A89013B12F0010F9BB2F6D08889C0B29D
:108C60006C4B196811B10B688A881A83664A6A4C82
:108C700013886A4D23F040031B041B0C13801388D8
:108C800023F038031B041B0C138013889BB243F0A2
:108C90004003138023782F68834240D0FFF7C2FC43
:108CA0005F4E604AB6F84E34B2F80080DFF87CC1FF
:108CB000002210464FF0050B4FF0060A4FF007094F
:108CC000F5181CF80340297BA14203F1010700F1CC
:108CD000050112D006EB010E31182C731D0A81F824
:108CE000ECB181F8EEA181F8EF3181F8F09181F8D3
:108CF000ED51013206308EF8EC41BBB2434502F132
:108D0000010280F09780632ADADDA6F84E3400284D
:108D100040F096803D4A00231370BDE8F88F424B27
:108D20003F4E1B78002BBCD1D6F84434FB1AB3F568
:108D30007A7FB6D91388364823F040031B041B0CF6
:108D400000881380138823F038031B0442084FEA7D
:108D500013430BD042F48072002A92FAA2F0B0FAC8
:108D600080F208BF4FF0FF32013AD2001343264A87
:108D70009BB2138013889BB243F04003138011B160
:108D80000B688A885A83A0211F4839F095F8002182
:108D90001D4839F091F81F4B1B6813B11A689B8866
:108DA0001383194ADFF88880138823F040031B04DB
:108DB0001B0C1380138823F038031B041B0C138037
:108DC00013889BB243F04003138098F80030182BAF
:108DD00000F0B780430700F1B08000F005000128E3
:108DE00000F0C08060B92378580609D5D6F8482429
:108DF0002B68002A00F0BB809B1A642B00F2BA801B
:108E0000C6F844744DE700BF003C00401D3600200A
:108E10006C1D0020C48900209F00002034C8002061
:108E2000902400209C000020D889002014340020C9
:108E3000CD8900200023A6F84E3400283FF46AAF05
:108E40005449554B1A880B8823F040031B041B0C14
:108E50000B800B8823F038031B0452084FEA13439E
:108E60000BD042F48072002A92FAA2F1B1FA81F298
:108E700008BF4FF0FF32013AD2001343454A9BB27C
:108E8000138013889BB243F040031380434B1E684A
:108E900016B13368B2885A833E4A414F93890138EC
:108EA0004FF47A734FF6FF74002F44D03D780137AA
:108EB00001E0A34239D01189013B89079BB2F8D563
:108EC000ABB293814FF47A7302E0ABB2A3422CD0E1
:108ED0001189C90703F1FF35F7D501389189411C84
:108EE000E2D116B13368B2881A832A4A138823F074
:108EF00040031B041B0C1380138823F038031B044E
:108F00001B0C138013889BB243F040031380254A47
:108F100000231370BDE8F88F1E4810F0B5F981E604
:108F20001C4810F0B1F9C0B29AE61A4810F0ACF93A
:108F30001A4B1E68D5E7FF25BDE70023C6F8483465
:108F40005EE72378184A03F04003002B00F0070186
:108F50000CBF4FF00D0E4FF0100E13805180A2F891
:108F600006E037E723785C067FF540AF48E7C6F8B0
:108F7000483445E7FFF756FB98F80030182B7FF48C
:108F80003FAFB6F84C34084A01339BB2A6F84C34D4
:108F9000938035E7003C00406C1D0020C489002010
:108FA0007C2600201D360020D08900202DE9F84FB6
:108FB000A94F3B7803B1FEE7A84CA94A01233B70B7
:108FC0002388128823F040031B041B0C2380238872
:108FD00023F038031B0452084FEA13430BD042F42A
:108FE0008072002A92FAA2F4B4FA84F208BF4FF019
:108FF000FF32013AD2001343984ADFF870829BB2E5
:10900000138013889BB243F040031380D8F80030DC
:1090100013B11A689B885383924B01220D461A7034
:1090200004468E4940F2E93302E0002B00F0A381B0
:109030000A89013B12F0020F9BB2F6D000238B810C
:1090400040F2E933854902E0002B00F094810A895F
:10905000013B12F0010F9BB2F6D08B897F4940F2A1
:10906000E93302E0002B00F09A810A89013B12F0FB
:10907000020F9BB2F6D000238B8140F2E93377498F
:1090800002E0002B00F08B810A89013B12F0010FF6
:109090009BB2F6D08B89714940F2E93302E0002B94
:1090A00000F079810A89013B12F0020F9BB2F6D0E1
:1090B00009238B8140F2E933684902E0002B00F07C
:1090C0006A810A89013B12F0010F9BB2F6D08B89AD
:1090D000624940F2E93302E0002B00F058810A892E
:1090E000013B12F0020F9BB2F6D0A4B28C8140F289
:1090F000E9335A4902E0002B00F049810A89013B1B
:1091000012F0010F9BB2F6D08B89574E534C013DA4
:109110004FF0000A4FF00A0B40F2E93302E0002B57
:1091200000F010812289013B12F0020F9BB2F6D0B1
:10913000A4F80CB040F2E93302E0002B00F0028109
:109140002289013B12F0010F9BB2F6D0A38940F2B5
:10915000E93302E0002B00F0F9802289013B12F094
:10916000020F9BB2F6D01FFA8AF3A38140F2E933D3
:1091700002E0002B00F0EA802289013B12F0010F8F
:109180009BB2F6D0A38915F8019F40F2E93302E0C3
:10919000002B00F0DF802289013B12F0020F9BB20E
:1091A000F6D00B23A38140F2E93302E0002B00F05C
:1091B000D1802289013B12F0010F9BB2F6D0A38926
:1091C00040F2E93302E0002B00F0C8802289013B25
:1091D00012F0020F9BB2F6D01FFA89F9A4F80C9096
:1091E00040F2E93302E0002B00F0B8802289013B15
:1091F00012F0010F9BB2F6D0A389336833B11A681D
:109200009B8851690B4214BF538313830AF1010AEF
:10921000BAF1360F80D140F2E933104802E0002B5A
:1092200000F0B1800289013B12F0020F9BB2F6D030
:1092300008238381094940F2E93302E0002B00F062
:10924000A2800A89013B12F0010F9BB2F6D08B89F4
:10925000024840F2E9330EE01D360020003C004099
:109260006C1D00202536002000C80020C489002085
:10927000002B00F084800289013B12F0020F9BB2A8
:10928000F6D0A0238381484940F2E93301E0002B66
:1092900075D00A89013B12F0010F9BB2F7D08B8980
:1092A000414CA02540F2E93301E0002B5AD022893D
:1092B000013B12F0020F9BB2F7D0A58140F2E933D7
:1092C00001E0002B4ED02289013B12F0010F9BB22E
:1092D000F7D0A38940F2E93301E0002B46D0228980
:1092E000013B12F0020F9BB2F7D00023A38140F2A2
:1092F000E93301E0002B39D02289013B12F0010F44
:109300009BB2F7D0A089C0B28306CBD4D8F8003086
:1093100013B11A689B881383234A138823F04003F0
:109320001B041B0C1380138823F038031B041B0C35
:10933000138013889BB243F04003002113803970DF
:10934000BDE8F88F20460FF09FFF00E720460FF0A2
:109350009BFF18E720460FF097FF31E720460FF0FC
:1093600093FF4AE720460FF08FFFB3E720460FF048
:109370008BFFC0B2C8E70C480FF086FF6EE60A48C4
:109380000FF082FF8CE708480FF07EFF60E7064889
:109390000FF07AFFB9E604480FF076FF98E602482E
:1093A0000FF072FF77E600BF003C004030B4147845
:1093B00074B11E23074D13FB01012944801A831841
:1093C0001D2BD8BF0C7012F8014F0131002CF6D1C3
:1093D00030BC704714340020F8B5434C434A23880E
:1093E000128823F040031B041B0C23802388C1F147
:1093F000030123F0380341EA80071B045208FFB23F
:109400004FEA13430BD042F48072002A92FAA2F181
:10941000B1FA81F208BF4FF0FF32013AD200134394
:10942000314A334D9BB2138013889BB243F0400303
:1094300013802B6813B11A689B8853832A4CBFB2E0
:10944000102640F2E93301E0002B45D02289013B90
:1094500012F0020F9BB2F7D0B3B2A38140F2E9330E
:1094600001E0002B38D02289013B12F0010F9BB2A2
:10947000F7D0A38940F2E93301E0002B30D02289F4
:10948000013B12F0020F9BB2F7D0A78140F2E93303
:1094900000E02BB32289013B12F0010F9BB2F8D000
:1094A000A3890136202ECCD12B6813B11A689B8872
:1094B00013830D4A138823F040031B041B0C1380F5
:1094C000138823F038031B041B0C138013889BB2F2
:1094D00043F040031380F8BD20460FF0D5FEC9E7E6
:1094E00020460FF0D1FEDCE7003C00406C1D002060
:1094F000C489002038B5454B1D7A00287BD105F082
:10950000F70543491D720B88424A23F040031B04B0
:109510001B0C12880B800B8823F038031B045208A5
:109520004FEA13430BD042F48072002A92FAA2F160
:10953000B1FA81F208BF4FF0FF32013AD200134373
:10954000334A354C9BB2138013889BB243F04003DF
:109550001380236813B11A689B88538340F2E93360
:109560002B4901E0002B49D00A89013B12F0020F80
:109570009BB2F7D004238B8140F2E933244901E008
:10958000002B3BD00A89013B12F0010F9BB2F7D0B0
:109590008B891F4940F2E93301E0002B32D00A8960
:1095A000013B12F0020F9BB2F7D0ADB28D8140F2B9
:1095B000E933174900E02BB30A89013B12F0010F90
:1095C0009BB2F8D08B89236813B11A689B881383E8
:1095D0000F4A138823F040031B041B0C13801388CD
:1095E00023F038031B041B0C138013889BB243F039
:1095F0004003138038BD45F0080582E704480FF0AA
:1096000043FEC6E702480FF03FFEDCE7902400204F
:10961000003C00406C1D0020C489002038B50B4C74
:1096200023688BB15A68821A002A054604DA0CE0D6
:109630005A68AA1A002A07DB9A68226018461A6834
:1096400090472368002BF3D138BD38BD209500200A
:109650000B4B002210B4027203F59074032102E058
:10966000072A09DC9979890702D5197981540132D1
:109670009C4203F11803F3D15DF8044B704700BF1F
:109680005078040828230370704700BF012332215B
:10969000312241704271037203700371704700BF41
:1096A000436A8269D154436A0169826B01338B42F8
:1096B00028BF00234362002A2FD0EFF311825023EA
:1096C00083F31288836B1968C9072CD470B45E6861
:1096D0006EB9456A816A8D4217D084690C44DC609A
:1096E0000ED9691A59608562002180F85C101968EA
:1096F00041F00101D2B2196082F3118870BC704749
:109700000469611A59608662EEE7012380F85C30D3
:10971000D2B282F3118870BC7047826DD36843F077
:109720008003D3607047D2B282F31188704700BFC4
:10973000426B10B462B1C36CC2684469D11A013B78
:10974000615C5DF8044B08BF1346C364C8B2704740
:10975000016A4369C4685B5C0131A14228BF1146BC
:1097600001625DF8044BD8B2704700BF836B13B140
:1097700090F85C007047836A406A181AB0FA80F06B
:1097800040097047416A836A99420AD3CB1A816BB8
:10979000026961B14968501E0B4483420AD2C01A63
:1097A000704702691144CB1A816B0029F2D1501E17
:1097B000C01A704700207047436B43B1C26C5B68AE
:1097C00093422FBF981AC0689B1AC0187047C2698D
:1097D000036A9A422FBFD01AC0688018C01A704717
:1097E0000A4B30B503F1140493F900205D78072A81
:1097F000C8BF143A811804330D7313F8025C855402
:1098000013F8012C0A76A342EED130BD6847040854
:1098100003682DE9F041DF691FB13B46BDE8F04127
:109820001847002A164611DD04460D460E4400E096
:1098300023689B68204698470028F9D0236815F8CC
:10984000011B1B6820469847AE42F1D1BDE8F0816C
:109850002DE9F0478C4B1B78DB07074644D58B4B33
:109860008B4D1C788B4E012C59D01CD3022C07D168
:1098700089498A4A09881288914201D901241C70B9
:10988000EB7AE3B12B89D3B1854B1B78BBB127F0C1
:1098900031F8002800F09B802B7B83422CBF0121F4
:1098A000002131700CE07C497E4A098810886A7B6F
:1098B000801A8842E2DAEB7A0024002BE2D1317878
:1098C0002A79632A06D8022C774E00F0BA803378C2
:1098D000002B5DD1754AAB7A8C4238BF0C461470B0
:1098E000002B4CD1BDE8F0876B4B694D19885B8824
:1098F000E878CB1A83EAE3728142A2EBE3721DD3CC
:109900002B788B421AD3614B1C78E01E012861D959
:109910006749097802294FD0012C5E4EA5D15F4AD4
:109920005D491288687B0988121A914239DD5D4AC7
:1099300012888A42A4D200241C70A1E7B1EB400F28
:10994000E1DC524B1C78E11E012940F29480022A8E
:10995000DEDC57494F4E0878DFF84481DFF844C118
:10996000DFF838E100210324022834701C7088F8E5
:109970000010ACF80010AEF8001081D11FE0012CEF
:1099800071D0022C0BD10720BDE8F04733F0EEB8C0
:109990007068381A474B984258DD72709AE7BDE8F4
:1099A000F08702241C706BE7022AD2DD4049097857
:1099B00002294FF0040464D13949364E09783E48F3
:1099C000022ACCBF00220122C28081804BE7022103
:1099D000317075E7022A9BDC95F800C091FBFCFC16
:1099E0000CF1010CBCF1080FDFF8B4A0304EA878E0
:1099F00095F801E096F800802A4CDFF8A090254EFB
:109A0000A8BF4FF0080C8AF800C01FFA8CFA10FBB0
:109A10000AF01EFB0AFE80B2DFF88CA02080A9F8B5
:109A200000E000244FF0640EB8F1020F34701C7097
:109A3000CAF804408AF801E07FF439AF0FFA8CF1DC
:109A4000BDE73078A0B9012377603370C2F16402BA
:109A50001A4B00FB02F083FB0023C017A0EBA350BE
:109A60006430707036E70820BDE8F04733F07EB808
:109A70007368F81A8EE7032C96D10D4909780229EC
:109A80009AD0044EFCE600BF1C770020B06800208E
:109A9000E4950020B668002088780020B468002093
:109AA0009E780020B2680020C42F00204C45002082
:109AB000CD8900207F969800D08900206BCA5F6B0B
:109AC000038A2DE9F0478589ADB21D4029D00F46A4
:109AD00006464FF000484FF00009B5FA85F328FA22
:109AE00003F2D24391B21B3B15403182042B16D8AE
:109AF000DFE803F03129211903007B6A002B32D003
:109B000003F1FF3A1FFA8AFAC7F824903C6A34B18D
:109B100023682046514698476468002CF8D1002DF0
:109B2000DBD1BDE8F0873868716B036889B298476C
:109B3000002DD2D1F5E77868B16B036889B29847F8
:109B4000002DCAD1EDE7B868F16B036889B2984778
:109B5000002DC2D1E5E7F868316C036889B29847F7
:109B6000002DBAD1DDE7F36A1FFA83FACEE700BF12
:109B700030B50446806D61718389A26823F4005377
:109B80001B041B0C838185B0A379009213F004029F
:109B900030D04FF4805213F00203ADF8042056D1B8
:109BA000ADF806304FF480630022ADF8083011F0B4
:109BB0000103ADF80C2028D1ADF80A3008238D0739
:109BC000694648BFADF80A3028F0F6FDA279A36DCA
:109BD000D10724D412F0080F9A8A1BD122F0080270
:109BE0001204120C9A829A8992B242F400529A811B
:109BF00005B030BD13F00203ADF8042024D04FF4BB
:109C000000551346ADF80650CEE70423ADF80A30F0
:109C10000C23D4E792B242F008029A82E3E70D499E
:109C20008B420FD0A1F548418B4209D00A498B42A3
:109C3000D0D10520012138F0A1FAA279A36DC9E79E
:109C40000220F7E70020F5E7ADF80630ACE74FF467
:109C50000053A5E7001001400014014010B5044670
:109C6000806DA160838923F400531B041B0C838146
:109C7000A37984B013F00402009135D04FF48052E0
:109C800013F00203ADF8042056D1ADF806304FF4BE
:109C900080636279ADF80830D1074FF00003ADF86A
:109CA0000A30ADF80C3045BF0423ADF80A30082364
:109CB0000C236946920748BFADF80A3028F07CFDB6
:109CC000A279A36DD1071FD412F0080F9A8A16D17A
:109CD00022F008021204120C9A829A8992B242F47B
:109CE00000529A8104B010BD13F00203ADF80420B5
:109CF0001FD04FF400511346ADF80610C9E792B2D9
:109D000042F008029A82E8E70D498B420FD0A1F594
:109D100048418B4209D00B498B42D5D10520012106
:109D200038F02CFAA279A36DCEE70220F7E70020E5
:109D3000F5E7ADF80630ACE74FF40053A5E700BFF8
:109D4000001001400014014008B5012102200FF06D
:109D500041F9094B1B7803F00503052B08D00021BE
:109D600001200FF037F9002108460FF033F9FEE724
:109D70002CF0A4FFF3E700BF60760020022828BF84
:109D8000022010B4084C094B207000EB8002C0EB9D
:109D9000C20207495DF8044B013003EB4203C0B235
:109DA0000B6033F009B800BF785900203A56002004
:109DB0005496002008B530F0C5FD0FF047FCBDE813
:109DC000084030F0A7BD00BF38B5484B5A89998983
:109DD000914224BF00225A81198ADA89914224BF14
:109DE0000022DA81DA78CAB1072A41496AD091F8AB
:109DF0005300404D012400210A282C709C70D97119
:109E00005DD00C2807D0002A6CD0DFED3B7A072A02
:109E10000ED00A2862D0DFED397A09E0344A92F890
:109E200053000A2856D00C285BD1D979DFED347A5B
:109E3000344C9FED350AA278002918BFF0EE407A25
:109E4000062A04D8314901EB820191ED050A2179F6
:109E500079B1013A032A0BD8F7EE007A87EE800A2F
:109E600039F056FC2388984228BF1846208038BD18
:109E700038BD9B781F4A07EE103A1178B8EEC77AC2
:109E800067EE277A07EE101AB8EEC77A27EE277A20
:109E9000B4EEC70AF1EE10FAEADD80EE277AFDEEA5
:109EA000C77A17EE903A102BA8BF1023012BB8BF2A
:109EB0000123DBB28B4238BF0B46137038BDDFED98
:109EC000147AA4E791F853000A2803D00C28ACD0E8
:109ED000D9799AE7D979DFED0E7AA9E7DFED0D7A26
:109EE000A6E7D979DFED047AA2E700BF5C5A00202B
:109EF000705A0020909D00206F1203396F12833A30
:109F00000AD7A3395C6400206F120338684704083D
:109F10005304E9380F506E3A2DE9F047AC4FAD4E7F
:109F200030F010FDBE421ED2DFF82C83DFF82C93F8
:109F30004446258862197DB14A450DD2052D0BD9BD
:109F400033886188C3F30B03994200F0E480144620
:109F500025886219002DEFD17168304614360FF054
:109F600001FBBE42E4D39C4A1378A3F117010229F6
:109F70000FD99A4911F83300002840F0FB80D8002F
:109F80000144497829B1964911F833300BB91823A7
:109F90001370944B5A78022A00F2DD80924993485C
:109FA00002EB420201EB82011A780160022A00F200
:109FB000DB8002EB82018E4BC2EBC10203EB42035A
:109FC000998C5A8C8B4C9142236001D300225A8485
:109FD000894B9A78042A00F0EE8032B91A88B2F5DB
:109FE000F07F84BF4FF4F0721A80844DFFF7ECFECF
:109FF0002B68834A1A40002A00F0E680D80700F157
:10A00000D580590400F1CD801A0700F1BC809B0473
:10A0100000F1C0802EF064FC10B97A4832F0BAF832
:10A020004FF400700FF0D4FA4FF400300FF0D0FA74
:10A030004FF400100FF0CCFA4FF000700FF0C8FA98
:10A040004FF080600FF0C4FA35F07EF80021302226
:10A050006D483AF01AFB20682CF066FA6B4B2568C5
:10A0600003F1500103E00433994200F081801A7833
:10A07000002AF8D19C78D8788442F4D26449654BA0
:10A080000A7028461D6019F04DFD634A6349107936
:10A09000634A644B1160C822642111FB0021002235
:10A0A00059609A60DA601A615A619A61DA6183F8DC
:10A0B000202083F8212030F05BFA5B4B9FED5B5A48
:10A0C0001B885B4A9FED5B6A55795B4C5B495C483A
:10A0D000086006EE903AF8EEE66A1388C5EE265A56
:10A0E00007EE103A53881279C4ED005A07EE903A01
:10A0F000B8EEC77A534BF8EEE77A1D725A7227EE24
:10A10000067A67EE867ABDE8F04783ED017AC3ED03
:10A11000007A30F0FFBB63799B077FF418AF71685A
:10A1200094F804A030460FF01DFA3388BAEB133FC1
:10A1300004D01436BE42FFF4FBAE14E77388706897
:10A14000AA1FC3F30B039A4204F10601A8BF1A46E3
:10A1500039F00AF9EDE700225A701A7823482249AB
:10A160000160022A7FF625AF00221A70204B27E7F4
:10A17000012283E7D8000C186468002C7FF400AF3C
:10A1800017241470FCE630480FF022FA2B689B0469
:10A190007FF540AF2D480FF01BFA40200FF018FA62
:10A1A00038E72B480FF014FA2B682DE729480FF0F9
:10A1B0000FFA2B6825E79A8AB2F57A7FBFF415AFBC
:10A1C0004FF47A729A8210E743F008032B6015E788
:10A1D0004006000890010008404000202872040852
:10A1E000B06A04087859002046570020589600208D
:10A1F0003A560020549600205C64002098570020B6
:10A2000009600002449100208C2D00208032002043
:10A21000A4220020C02D0020849E0020A29D0020AA
:10A22000C82D002030410020F82F0020C0C9FB4875
:10A23000FC2D002017B7D138FC2F0020689E00208D
:10A240003661023D449E0020016000020940000288
:10A250000920000208600002024000080080000897
:10A2600008B530F06FFB0FF0F1F930F053FBFFF75A
:10A2700053FE0120BDE8084032F09EBD38B50D4CBC
:10A280000D4DAC4206D26168204614340FF06AF9D5
:10A29000AC42F8D310F0F8F9084A094B094C1460A5
:10A2A000002209491A705A7008480860BDE8384011
:10A2B0001FF04EBF90010008400600085496002091
:10A2C000785900203A560020589600204657002022
:10A2D00008B5FFF7D3FF30F035FB0FF0B7F9BDE855
:10A2E000084030F017BB00BFF0B50C2934D8DFE8C8
:10A2F00001F0893333335E33333334333333070080
:10A30000048C9689B2F802E01788734D24F48054C7
:10A310002404240C0484038C8488818B23F400534C
:10A3200021F4E6411B0409041B0C46EA0E06090C45
:10A3300043EA063341EA0721A8429BB2A4B289B29C
:10A3400000F09E8005F58065A84200F09980926833
:10A350008480818302640384F0BD048C9589B2F803
:10A3600002C0B2F800E05C4F24F480742404240C92
:10A370000484038C8688818B23F400731B0421F0F2
:10A3800073011B0C45EA0C04090443EA0423090C7D
:10A39000B8429BB2B6B241EA0E015CD04F4CA0422B
:10A3A00059D0926886808183C2630384F0BD048C97
:10A3B0009589B2F802C0B2F800E0474E24F01004CC
:10A3C0002404240C0484038C8788018B23F020034D
:10A3D00021F4E6411B0409041B0C45EA0C04090C9A
:10A3E00043EA041341EA0E21B0429BB2BFB289B2E4
:10A3F0005DD03A4CA0425AD0926887800183826334
:10A400000384F0BD048C9789B2F802E01688324DBF
:10A4100024F001042404240C0484038C8488018B1C
:10A4200023F002031B0421F073011B0C47EA0E0703
:10A4300009043B43090CA8429BB2A4B241EA0601BD
:10A4400025D005F58065A84221D0926884800183DB
:10A4500042630384F0BDD589148A578A23F40063CC
:10A4600043EA05254FF6FF332B40958826F44056E6
:10A470003C4343EA052346EA04169BB2B6B290E792
:10A48000158A24F4804444EA8514A4B25FE7D6898F
:10A49000158A578A23F00803334324F440749688BE
:10A4A0003D4323F004032C433343A4B2CDE7D489C6
:10A4B000158A568A23F0800343EA04134FF6BF74CB
:10A4C0001C40938827F44067354344EA031347EA66
:10A4D00085079BB2BFB28FE7000001400004014036
:10A4E0002DE9F84F4FF4A07200219148914CDFF80C
:10A4F0006892914D914E924FDFF860823AF0C5F824
:10A5000090489149DFF858E2DFF858C20022135909
:10A51000834200F0E980B3F1804F00F0E780AB4266
:10A5200000F0F280B34200F0F180BB4200F0F08016
:10A53000734500F0EF80634500F0EE80434500F086
:10A54000ED80DFF824A2534500F0EA800AF5806A26
:10A55000534500F0E7800AF5806A534500F0E48037
:10A56000AAF5983A534500F0E1800AF5806A534510
:10A5700000F097800AF5806A534508BF0D2300F06C
:10A5800091801832B2F59C7FC1D16A4EDFF8DCA110
:10A5900006F59C774FF003094FF0020803E01836E8
:10A5A000B74200F09F80B379002BF8D033791C09B3
:10A5B000013C032C03F00F03F1D8644A32F8140075
:10A5C00040FA03F2D207EAD5012505FA03F3013B6D
:10A5D000184038F057FC5E4B1B5D18441AEBC00264
:10A5E000DDD05AF830305B4C317A03F13F4000F552
:10A5F0007E00800A205C00F01F044009032805FA51
:10A6000004F57BD0042873D0022804D14E48406C56
:10A6100005434D484564B2F804E0BEFA8EF2C2F13B
:10A620001F0292B2D00803EB800002F00702046A16
:10A6300092000F25954024EA05040462046A01FA99
:10A6400002F22243002502624FF0010C2A4603E089
:10A65000102A05F10205A2D00CFA02F030EA0E0130
:10A6600002F10102F4D11C6809FA05F1C9430C405A
:10A670001C60D3F800B008FA05F444EA0B041C602F
:10A680009C680C409C609C689C605C6824EA0000AC
:10A69000586058685860D8680140D960D968D96056
:10A6A000D6E70C2309EBC3034FF0010A1B7903F033
:10A6B0001F0B5B09032B0AFA0BFA09D0042B0CD0F1
:10A6C000022B7FF45EAF4B6C4AEA03034B6458E7FE
:10A6D0000B6C4AEA03030B6453E70B6B4AEA030370
:10A6E0000B634EE7BDE8F88F0023DBE70123D9E7D2
:10A6F0001548006B0543144805638CE71248006C4D
:10A7000005431148056486E70223CBE70323C9E725
:10A710000423C7E70523C5E70623C3E70723C1E7EB
:10A720000823BFE70923BDE70A23BBE70B23B9E7EB
:10A73000E48900205078040800040040000800402C
:10A74000000C004000000140003802408C790408F1
:10A750008879040818780408D067040800040140C8
:10A760000010004000140040004001407CC6002062
:10A7700001490248FFF7A4B9FC8A002000180040F4
:10A7800001490248FFF79CB9D48A002000400140EB
:10A7900001490248FFF794B9AC8A00200004014047
:10A7A00001490248FFF78CB9AC8A0020000401403F
:10A7B00001490248FFF784B9848A0020000C004058
:10A7C00001490248FFF77CB95C8A0020000800407C
:10A7D00001490248FFF774B9348A002000040040A0
:10A7E00002494FF08040FFF76BB900BF0C8A002090
:10A7F00001490248FFF764B9E489002000000140E4
:10A8000001490248FFF75CB9E489002000000140DB
:10A81000F0B50468A30AA3F58013502B2AD8DFE80B
:10A8200003F02A7A8E9229297E2929292929292982
:10A830002929292929292929292929292929292988
:10A840002929292929292929292929292929292978
:10A850002929292929292929292929292929292968
:10A8600029298286292929292929292929292929A2
:10A8700029298A00F0BD4FF0480E01264779B00023
:10A880004FEA970C00296BD063460227A5899F40A9
:10A8900083190CEB43032F4303F1040C3A4DBFB271
:10A8A00045F8231045F82C20A781EFF311815022A1
:10A8B00082F31288821905EBC2021369002B46D07D
:10A8C00013620433821905EBC202576917B11F6086
:10A8D00053690433821905EBC202976917B11F60EF
:10A8E00093690433821905EBC202D76917B11F605F
:10A8F000D36904330027CAB21F6082F31188304441
:10A9000005EBC000036A2BBBA38923F001031B04E2
:10A910001B0CA381F0BD4FF0700E0226AEE74FF482
:10A920009C7E0726AAE74FF0200E0026A6E74FF0F0
:10A93000E80E0526A2E74FF4887E06269EE74FF034
:10A94000980E03269AE74FF0C00E042696E705EB13
:10A950000E03B7E7A3899BB243F00103A381F0BDC7
:10A960000223BF0803FA07F7A389074D9BB223EA26
:10A97000070387190CEB470CA3810CF1040345F87E
:10A980002C1045F8232090E7E489002010B50368D7
:10A9900082480139834282B089B200F0CA80A0F5B2
:10A9A0008060834200F0C58000F58040834200F063
:10A9B000B78000F58060834200F0B28000F58060CF
:10A9C000834200F0AD80764C188824686408B4FB9C
:10A9D000F2F4013CA4B282B2B3F1804F0AD07148C4
:10A9E000834207D000F58060834203D000F5806089
:10A9F000834202D122F0700292B26B48834200F08F
:10AA0000A18000F58060834200F0A68022F44072AD
:10AA100000F56C4092B283421A80D9621C854FD0F7
:10AA20005E4A93424CD001229A821A8892B242F036
:10AA300001021A80B3F1804F00F09880594A934286
:10AA400000F0968002F58062934200F0938002F558
:10AA50008062934200F0908002F58062934200F0A1
:10AA60008D8002F58062934200F08A8002F5704288
:10AA7000934200F0878002F57052934200F0848088
:10AA800002F58062934200F0818002F58062934279
:10AA90007ED0A2F5983293427CD002F58062934238
:10AAA0007AD002F58062934208BF0D2215D002A829
:10AAB0004FF0012340F8043D27F0EEFD02B010BD39
:10AAC0000122002119869A821A88384892B242F0EF
:10AAD000010283421A80ADD10A46354B03EBC20313
:10AAE00001A85C798DF80440012300228DF805301F
:10AAF0008DF807308DF8062027F0CEFD1B2C08D0EE
:10AB00002E2CDBD12B4B019301A827F0C5FD02B001
:10AB100010BD294B019301A827F0BEFD02B010BD66
:10AB20001F4C18882468B4FBF2F4013CA4B282B232
:10AB300052E71B4C18882468B4FBF2F4013CA4B221
:10AB400082B257E701201A80D9621C8598821A8840
:10AB500092B202431A8071E701201A80D9621C85E3
:10AB600098821A8892B202431A8063E70122B4E7FE
:10AB70000222B2E70322B0E70422AEE70522ACE7E7
:10AB80000622AAE70722A8E70822A6E70922A4E7E7
:10AB90000A22A2E70B22A0E70C229EE70004014054
:10ABA000585A0020000400400010004000000140FE
:10ABB000D06704082C010001190100012B4B9842B9
:10ABC0003CD0B0F1804F3BD0A3F57C43984239D0C4
:10ABD00003F58063984237D003F58063984235D0FF
:10ABE00003F58063984233D003F58063984231D0F7
:10ABF00003F5704398422FD003F5705398422DD03F
:10AC000003F5806398422BD003F58063984229D0E6
:10AC1000A3F59833984227D003F58063984207D074
:10AC200003F58063984208BF0D2202D000207047D0
:10AC30000C220F4B03EBC203187970470022F8E790
:10AC40000122F6E70222F4E70322F2E70422F0E70A
:10AC50000522EEE70622ECE70722EAE70822E8E70A
:10AC60000922E6E70A22E4E70B22E2E700000140BE
:10AC7000D06704082DE9F04F013085B0C3B20393CB
:10AC80000B4602918B4C8C4E002B00F09A803220A8
:10AC90008A4D8B4FDFF82C9236F06AF94FF4FA7A2E
:10ACA0004FF0100C4FF47A70D9F80430C3F3080356
:10ACB000002B40F0DE80EFF31183002B40F0D980B1
:10ACC0002968A26800BF2B689942F9D1D7F800E043
:10ACD00000FB0EF39B1AB3FBFEF300FB01314FF0B8
:10ACE000010E0191D9F80430C3F30803002B40F0A2
:10ACF0008780EFF31183002B40F082802B68A168DE
:10AD000000BF2A689342F9D1D7F800B000FB0BF2DC
:10AD1000521AB2FBFBF200FB0323019A9B1AB3F514
:10AD20007A7FDFD3BAF1010ABED1039B002B40F03A
:10AD3000BD804FF47A7ADFF88C9150464FF0100CBA
:10AD4000D9F80430C3F30803002B75D1EFF3118356
:10AD5000002B71D12968A26800BF2B689942F9D1F4
:10AD6000D7F800E000FB0EF39B1AB3FBFEF300FBE9
:10AD700001314FF0010E0191D9F80430C3F30803FB
:10AD800013BBEFF31183FBB92B68A16800BF2A68DE
:10AD90009342F9D1D7F800B000FB0BF2521AB2FB84
:10ADA000FBF200FB0323019A9B1AB3F57A7FE3D3EE
:10ADB000BAF1010AC4D1029B013B0293002B7FF43C
:10ADC00066AF05B0BDE8F08FEFF311888CF3128801
:10ADD000A1682368DB0344BFC6F800E0A1682B68C4
:10ADE00032685FFA88F888F31188D7F800801A442F
:10ADF00000FB08F35B1AB3FBF8F300FB0233D2E766
:10AE0000EFF311888CF31288A1682368DB0344BF39
:10AE1000C6F800E0A1682B6832685FFA88F888F30A
:10AE20001188D7F800801A4400FB08F35B1AB3FBC3
:10AE3000F8F300FB023370E7EFF311828CF3128812
:10AE4000D4F808E02368D90303D501233360D4F88C
:10AE500008E02B683168D2B282F311883A6819444D
:10AE600000FB02F3A3EB0E03B3FBF2F300FB013193
:10AE70007FE7EFF311828CF31288D4F808E023689F
:10AE8000D90303D501233360D4F808E02B68316877
:10AE9000D2B282F311883A68194400FB02F3A3EBA3
:10AEA0000E03B3FBF2F300FB013118E7184635F04F
:10AEB000C1FE3EE710E000E030C8002034C80020AA
:10AEC00038C8002000ED00E0204B5B68C3F30803A6
:10AED00030B4BBB9EFF31183A3B91D4B1D4C1868F7
:10AEE000A16800BF1A689042F9D11B4B1C684FF44F
:10AEF0007A7202FB04F3591AB1FBF4F130BC02FB85
:10AF000000107047EFF31182102383F31288114968
:10AF10008C680B6813F4803F104B02D0012018603E
:10AF20008C680B49D2B20D68186882F311880A4BFD
:10AF300019684FF47A72284402FB01F31B1B30BCE2
:10AF4000B3FBF1F302FB0030704700BF00ED00E0FF
:10AF500034C8002010E000E038C8002030C80020CD
:10AF60002DE9F84F8046FFF7AFFF254E2549DFF862
:10AF7000A0E0254A254D844610274FF47A7401201D
:10AF8000DEF80430C3F30803D3B9EFF31183BBB980
:10AF90000B68D2F808A000BFD1F800904B45F7D15C
:10AFA000D6F800B004FB0BF9A9EB0A09B9FBFBF9D1
:10AFB00004FB0393A3EB0C034345E1D3BDE8F88FF7
:10AFC000EFF3118A87F31288D2F808B01368DB0315
:10AFD00044BF2860D2F808B00B68D5F800905FFA3B
:10AFE0008AFA8AF31188D6F800A0994404FB0AF380
:10AFF000A3EB0B03B3FBFAF304FB0933DAE700BF5F
:10B0000038C8002034C8002010E000E030C800201C
:10B0100000ED00E02DE9F04FDFF830C1474A484924
:10B02000484E494D8046102718F1FF38C0F0848003
:10B03000DCF80430C3F30803002B5CD1EFF3118379
:10B04000002B58D10B68946800BF08688342F9D17F
:10B05000D6F800904FF47A7000FB09FEAEEB040EB8
:10B06000BEFBF9FE00FB03EEDCF80430C3F308037B
:10B070004FF47A740120FBB9EFF31183E3B90B6845
:10B08000D2F808A000BFD1F800904B45F7D1D6F810
:10B0900000B004FB0BF9A9EB0A09B9FBFBF904FBAF
:10B0A0000393A3EB0E03B3F57A7FBDD2DCF8043033
:10B0B000C3F30803002BDFD0EFF3118A87F3128864
:10B0C000D2F808B01368DB0344BF2860D2F808B098
:10B0D0000B68D5F800905FFA8AFA8AF31188D6F8DF
:10B0E00000A0994404FB0AF3A3EB0B03B3FBFAF3B0
:10B0F00004FB0933D5E7EFF3118487F31288D2F804
:10B1000008901368D80303D501232B60D2F8089068
:10B110000B682868E4B284F31188D6F800A04FF4D5
:10B120007A7400EB030E04FB0AF3A3EB0903B3FBF1
:10B13000FAF304FB0E3E97E7BDE8F08F10E000E065
:10B1400034C8002038C8002030C8002000ED00E0DE
:10B1500030B4EFF31183102282F312880649074CB2
:10B160000A680748013200250A602560DBB20268E0
:10B1700083F3118830BC704734C8002030C80020E9
:10B1800010E000E00F4B1B88014643B90E4B0F4AFD
:10B190001B7810680BB981F001010DF013BF0C4B47
:10B1A0005A691AB118B91A68106058747047094A78
:10B1B00018681188084A92FBF1F201210260597463
:10B1C000704700BF0CC800200EC8002010C8002027
:10B1D00014C800202CC8002020A1070038B5264B39
:10B1E0005C69636B73B1A36DA26BD2B1998A1A8843
:10B1F000C90592B201D5D20700D438BD4FF6F77217
:10B200001A8038BDA36D99891A88890692B2EBD548
:10B210009206E9D5E26AD2B19888216B80B2904754
:10B22000E1E799891A880D0692B2DFD51006DDD5BF
:10B23000A26A616A8A4219D0A1692569885C9880EE
:10B240000132B2FBF5F105FB1122A262CEE79B8829
:10B25000E2696169DBB28B54E269E068A36D013297
:10B26000B2FBF0F100FB1122E261BDE7DA6822F0E7
:10B270008002DA60BAE700BF6476002038B5264B5A
:10B280009C68636B73B1A36DA26BD2B1998A1A8863
:10B29000C90592B201D5D20700D438BD4FF6F77276
:10B2A0001A8038BDA36D99891A88890692B2EBD5A8
:10B2B0009206E9D5E26AD2B19888216B80B29047B4
:10B2C000E1E799891A880D0692B2DFD51006DDD51F
:10B2D000A26A616A8A4219D0A1692569885C98804E
:10B2E0000132B2FBF5F105FB1122A262CEE79B8889
:10B2F000E2696169DBB28B54E269E068A36D0132F7
:10B30000B2FBF0F100FB1122E261BDE7DA6822F046
:10B310008002DA60BAE700BF6476002038B5264BB9
:10B320001C68636B73B1A36DA26BD2B1998A1A8842
:10B33000C90592B201D5D20700D438BD4FF6F772D5
:10B340001A8038BDA36D99891A88890692B2EBD507
:10B350009206E9D5E26AD2B19888216B80B2904713
:10B36000E1E799891A880D0692B2DFD51006DDD57E
:10B37000A26A616A8A4219D0A1692569885C9880AD
:10B380000132B2FBF5F105FB1122A262CEE79B88E8
:10B39000E2696169DBB28B54E269E068A36D013256
:10B3A000B2FBF0F100FB1122E261BDE7DA6822F0A6
:10B3B0008002DA60BAE700BF6476002070B4EFF371
:10B3C0001186502383F31288836B1A68D20720D426
:10B3D0005D686DB9446A826A944217D081691144EC
:10B3E000D9600ED9A21A5A608462002280F85C20CB
:10B3F0001A6842F00102F1B21A6081F3118870BC40
:10B40000704701698A1A5A608562EEE7012380F865
:10B410005C30F3B283F3118870BC704703685B6AD9
:10B4200003B11847704700BF03681B6A03B1184790
:10B43000704700BF03682DE9F041DF691FB13B464B
:10B44000BDE8F0411847002A164611DD04460D46B6
:10B450000E4400E023689B68204698470028F9D0F6
:10B46000236815F8011B1B6820469847AE42F1D1AE
:10B47000BDE8F08103689B69184700BF03685B69FA
:10B48000184700BF03681B69184700BF0368DB68E3
:10B49000184700BF03689B68184700BF03685B68D4
:10B4A000184700BF2DE9F04FBC4B1E788BB0002E23
:10B4B00040F08180BA4BBB4C1D78BB4FDFF80CB31A
:10B4C00005F00105A4F10A0954F80A0CB8B14FF0CF
:10B4D000CC0808FB0698FFF7E1FF80B154F80A0C8E
:10B4E000FFF7D4FF14F8023C024683B924283BD06E
:10B4F00075B354F80A0CFFF7D1FF0028EED10136DE
:10B50000032E04F1CC04DFD10BB0BDE8F08F012B8A
:10B510002ED0022B33D0032B40D0042B00F06981B6
:10B52000052B00F05781062BE3D114F801ECBEF196
:10B53000000F00F0D881BEF1010F00F01B82013630
:10B540000023032E04F8023C04F1CC04BCD1DBE759
:10B55000232A54F80A0C00F08281944B93F832307D
:10B560009342B8D136F01EFE012304F8023CC0E736
:10B570004D2800F06781002304F8023CB9E700235E
:10B580003C2804F8023C00F057813E28B1D101224A
:10B59000032304F8012C04F8023CAAE7C028EAD8E7
:10B5A0000021042304F8050C04F8040C04F8061C1C
:10B5B00004F8023C9DE77E4B18680028A4D00DF0EB
:10B5C00031FFDFF80CA27B4DDFF8F891DAF80000CC
:10B5D000FFF764FF002897D0DAF80000FFF756FF66
:10B5E00009281BD03F2819D02B68002B67D10428CD
:10B5F00000F0BA810C2800F0CA807F28E6D0A0F1C4
:10B600002002D2B25E2AE1D80BB92028DED05A1C23
:10B6100009F803002A6011F0E7FED7E72C68002C38
:10B620005AD1654FA34607F51C78BBF1000F08BF40
:10B63000BB4610374745F8D1BBF1000F00F04E81F3
:10B64000103FDBF800003A68065D135D9E4220441F
:10B6500002EB040140F04081661E4E4422460BB9C5
:10B66000FD2A5CD906F8013F01322A6010F8013F3B
:10B6700011F801EF9E45F2D00AB15F4512D04F4854
:10B680002AF018F85F4508D35BF8100B2AF012F87F
:10B69000092011F0A9FEBB45F6D949482AF00AF85D
:10B6A0002A680024944291D2661E4E4416F8010F77
:10B6B00011F09AFE2B6801349C42F7D386E70C28E0
:10B6C00065D00A2834D00D2832D07F2800F0BE8003
:10B6D000FF2B3FF67BAF92E7374E002706F51C782D
:10B6E000BB4602E0103646450DD02246316848463A
:10B6F0000EF0F8F90028F5D1B346002FF2D1374605
:10B7000010364645F1D13B465F469B46002B98D10B
:10B71000002F3FF45BAF294829F0CCFFB4E7511C60
:10B72000202009F80200296009F801300A46A4E740
:10B7300029F0D0FF2321234838F0BEFF002800F075
:10B740001181A0EB0900286090B1431E19F8031085
:10B75000202940F02C8109EB030243B112F8011DAE
:10B76000202903F1FF304FD10346002BF6D12B6087
:10B770004FF480720021484638F087FF074B1B7852
:10B78000002B3FF4C1AE0E4829F094FF1EE70E488F
:10B7900029F090FF0A4829F08DFF17E71C3600209A
:10B7A0001C77002012BA0020E028002044910020DD
:10B7B000EC360020F0370020704B0408C4790408F0
:10B7C000CC790408F0360020D4790408984704089E
:10B7D000E836002014F8063C14F8051C99426FD88E
:10B7E00014F8043C83427FF4C6AE062304F8023CFE
:10B7F0009BE614F8043C04F8030C5A40052304F8B3
:10B80000042C04F8023C74E62B606A4C002204F518
:10B810001C7809F8032002E0103444454CD021681C
:10B82000484619F0B7FF0028F6D0444544D2E368F3
:10B83000984700232B609BE7032204F8013C04F89F
:10B84000022C56E6022304F8023C52E6013B002299
:10B8500059482B6009F8032029F02CFFB6E6574B16
:10B860005749DB78574ADFF888E11060003318BF8A
:10B8700001230B70544B554ACEF80030544B7A607C
:10B880004FF0400E012187F80CE03860B8607D73FE
:10B890005048197029F046FF4F4829F00BFF4FF42C
:10B8A000006010F0A5F94D4B93F83230232B3FF494
:10B8B00059AE14F8023C36E6494829F0FBFEB8E7D9
:10B8C00014F8041C08EB03005140013304F8041C75
:10B8D00004F8063C82720CE62246CDE64148103F51
:10B8E00029F0E8FED0E69BE80F000DF1280C0DF1E1
:10B8F000080888E80F004CF824ED14F8053C14F80B
:10B9000003AC0694624623444FF0010C414606A85E
:10B91000ADF822E00793ADF820A08DF824C005F023
:10B920001BFC40B1029A304B03924146A4F10A003D
:10B93000029325F0EDF9DDF80480002304F8023CC1
:10B94000B8F1000F3FF4DBAD54F80A0C25F0A0FA73
:10B95000013654F80A0CC047032E04F1CC047FF4DE
:10B96000B3ADD1E52868EFE6204819F029FB0BB00C
:10B97000BDE8F08F14F8053C14F8032C069423441A
:10B9800007936E2A4FF0000308930993ADF8202027
:10B990007FF4D5AD06A80EF027F906A80EF018F929
:10B9A00006A80EF015F906A80EF012F9C7E5034631
:10B9B0002BE700BF704B0408FC790408785900207D
:10B9C00018690020E8360020E428002011980008BB
:10B9D0001C360020007A0408CC7904084491002029
:10B9E000E0790408C47904084CC80020F03600202F
:10B9F000EC3600202DE9F04F2DED028B95B0064678
:10BA000030F01EF99C4B1D7825B115B0BDEC028BB2
:10BA1000BDE8F08F994B1B685A05F6D5DFF8A89260
:10BA2000D9F80020002A00F02381954CD4F8283161
:10BA300003F5F43348339E42C0F01A81914F94F8D5
:10BA40002C313968C4F82861013384F82C318B0714
:10BA500001F1858511F0140F41F0668594F82C31C1
:10BA600013F0070801F0DA85282B874B029301F0C9
:10BA700056875E209047854B1B78002B6BD0804CFF
:10BA8000834AD4F83431F31A934201F20F84DFF879
:10BA90003CA29AF80080B8F1000F33D1DFF8009291
:10BAA000D9F80000FFF7FAFCC0B201280ED902282D
:10BAB000784F42F040803B78002B42F0E681D4F88A
:10BAC0003C31F31AB3F57A6F82F0528272480768FC
:10BAD000002F40D09AF80030BBB9704BD9F8000065
:10BAE0001B689B781E3B012B4FF0020142F2DF8165
:10BAF00004302FF05DFF012200238AF8002084F833
:10BB0000483126E0644807682FB3D4F8443140F642
:10BB1000B732F31A93421ED994F84031002B02F049
:10BB20000080013BDBB284F84031002B01F06E86CF
:10BB300017F8011B94F84821076094F849315848D8
:10BB40000A440133006884F8482184F849310CF034
:10BB500037FEC4F84461534A029B12781B68012ADD
:10BB600003F101030C9301F0CB824F4B1B787BB1A7
:10BB7000DFF85C91D9F8003053B1414C029BD4F806
:10BB80005C21D3F800B0ABEB0202632A01F2E6813C
:10BB9000DFF8408198F800A0BAF1020F01F0128698
:10BBA0003C4F97F87430032B01F0A8843F4B1B786F
:10BBB00073B13F4D2B685BB1314CFFF785F9D4F879
:10BBC0006831039044F61F62C31A934200F22C813D
:10BBD000384B1B78002B7FD1374B1B7843B1284C57
:10BBE000D4F8B83203F50043E8339E4281F0FE8278
:10BBF000324B1B78002B3FF408AF214E304C314DB7
:10BC000006F2C1272068FFF749FC00283FF4FDAE8B
:10BC10002068FFF73BFC2B7880465A1E33B1206822
:10BC20002A70FFF73BFC0028F2D1EEE603223946EA
:10BC3000781E38F010FD96F8C03296F8C12286F8CA
:10BC4000C38283F47F4383F0FF039B1A1FFA88F8B3
:10BC50009BB2B8EB132FD5D196F8C222DBB29A4231
:10BC6000D0D1781E27F0C8FF2B7818442870C9E778
:10BC7000054B0293FFE600BF1C3600205C620020EB
:10BC800030290020F495002034C8002006970020B9
:10BC90003F0D0300040000206C96002068960020F1
:10BCA0006496002007970020149700201C9700201E
:10BCB000209700208C9700209D9700202697002039
:10BCC0002C9700203097002074960020709600205A
:10BCD0005C7A0020FA310020474C2278002A41F09B
:10BCE0000682DFF83C9199F80040002C79D1434D51
:10BCF0002878002842F05480414C424DD4F8B022BC
:10BD00002978414B93FBF1F313449E42FFF464AF57
:10BD100094F8B4323D4AC4F8B062D75CFB0702F134
:10BD2000F981B80702F19281790702F13F823A075F
:10BD30004CD5374BDFF8EC800D930DF15009A3F192
:10BD40003D0249F8202D0021A3F1400203F8401CD8
:10BD500002231121517093704846D8F800100DF05D
:10BD600053FF4846D8F804100DF04EFFB8F80E30D7
:10BD7000284903EBC3039B00053381FB0321DB1739
:10BD8000C3EBA10189B248460DF056FFB8F8103058
:10BD900003EB8303590089B248460DF04DFF1E4B5B
:10BDA0001B789B0743BFB8F8081001F57A7189B278
:10BDB0004FF47A7148460DF03FFF0C9B98F8142021
:10BDC000591C0C9148461A702FF0E0FE94F8B432DA
:10BDD0002978013393FBF1F201FB123384F8B4327A
:10BDE000FAE60E4D2F6E002F41F0D485044B89F8F2
:10BDF0000070C3F8B062EFE6F89600209497002038
:10BE0000302900209C970020A086010098970020F0
:10BE1000B89600206766666652960020A4970020B8
:10BE200095970020409F002094F86E31002B41F040
:10BE30006185DF4B1B6803F00802002A48F60341C6
:10BE40004AF60B404BF60F4249F6074704BF02463D
:10BE50000F4613F0040F4FF0190118BF17469B0649
:10BE600084F86E1103D547F4804747F0200724F08B
:10BE700033FDC7F30909002842F0D881CD4B9B79E7
:10BE8000002B42F02A83984664204FF0FF3A4FF08F
:10BE9000000C0C970D97ADF83CC0CDF842C0CDF822
:10BEA00046C0CDF84AC0CDF83890ADF83E80ADF828
:10BEB00040A08DF84E000CAF0FCFDFF808E384F8F8
:10BEC00005C0AEE80F0097E80F00AEE807002EF8B7
:10BED000023B71464FF0010C1B0CFE271F20C822AD
:10BEE00001F81E39A770A27184F807C0E07094F8B9
:10BEF0007E01207180F0F10383EA0313DAB21309A3
:10BF000083F0E70343EA022383EAC2031BB283EA16
:10BF10000312D2B2C3F3072383EA121343EA0223C4
:10BF200083EAC2031BB283F0C80282EA0212D2B2D1
:10BF3000C3F3072383EA121343EA022383EAC2030B
:10BF40001BB283EA0C0787EA0717FFB2C3F3072285
:10BF500082EA171242EA072200EB0C0382EAC707C3
:10BF60000EEB0C0084F87E31278011F8013B7B40FA
:10BF700083EA0313DBB21A0982EA172242EA032298
:10BF800082EAC3031BB29FB281422780EDD183F0C6
:10BF90007C0383EA0313DBB24FEA131E8EEA172EEB
:10BFA0008EEA032E8EEAC30E0FFA8EFE1FFA8EF96A
:10BFB000DFF814C2A4F800905FFA8EFE4FEA192948
:10BFC00084F8289084F827E00CF5D37804F1220A4D
:10BFD000DCF80000DCF80410DCF80820DCF80C3099
:10BFE00047460FC70CF1100CD445B846F0D1DCF829
:10BFF00000003860704F9CF8043088F8043007F176
:10C00000270884F8CDE184F8CE9117F8011F28683D
:10C010000CF0D6FBB845F8D194F86F21002A41F016
:10C02000FD836649029B08781B680A2184F86F111A
:10C03000002801F09B85DFF894E10128BEF800108C
:10C04000059142F251820228BEF8028002F0C381BB
:10C05000BEF804100491032802F05A820428BEF8A6
:10C0600006A002F050820528BEF8087002F0478250
:10C070000628BEF80AC002F03F820728BEF80C105E
:10C0800001D0BEF80E2094F87EB10C938BF03003F3
:10C0900083EA0313DBB24FEA131E494884F804B065
:10C0A0008EF07A0E4EEA032E00888EEAC303DFF884
:10C0B00020E1C0EB00208EFB009E8644C0171BB21F
:10C0C000C0EB6E200690C3F3072E83EA0310059B96
:10C0D000C0B24FF0000963F30F098EEA1013059305
:10C0E0004FF0000E049B68F31F4967F30F0E4FF0EB
:10C0F0000008002763F30F0861F30F07059BCDF8D5
:10C1000034906CF31F4E62F31F474FF0000C9DF804
:10C110001820CDF83CE06AF31F48CDF8388010971E
:10C120008DF844C08DF8452043EA00230DF1300816
:10C1300083EAC007B8E80F003FB287F0C80989EA70
:10C140000919DFF880E084F805C05FFA89F9C7F3C0
:10C150000727AEE80F0087EA191747EA092398E88E
:10C16000030083EAC9031BB283F023074EF8040BD4
:10C1700087EA0717FFB2C3F3072282EA1712704655
:10C1800042EA072282EAC70720F814190BF1010BD3
:10C190004FF0230CFE211622C82384F87EB127809D
:10C1A00084F807C00EF1020EA170E270A37111E0D5
:10C1B000F4950020E4950020D72A0020A0930020C9
:10C1C0003847002038290020322900200847002065
:10C1D0000308208010F8013B7B4083EA0313DBB2A5
:10C1E0001A0982EA172242EA032282EAC3031BB237
:10C1F0009FB270452780EDD183F0F40383EA0313E7
:10C20000DBB24FEA131E8EEA172E8EEA032E8EEA59
:10C21000C30E0FFA8EFE1FFA8EFCD64FA4F800C094
:10C220004FEA1C295FFA8EFE84F81EE084F81F9006
:10C230007968BA683868FB6807F5D37CACE80F000A
:10C2400038697969BA6904F2C518ACE8070004F2E4
:10C25000A71784F8C59184F8C4E117F8011F28686E
:10C260000CF0AEFAB845F8D194F87231002B41F0D9
:10C270005183C14F3B681922980684F8722140F11E
:10C280000E83BE4BDFF800831B78990741F192863D
:10C2900098F81430042B8CBF4FF003094FF00209BB
:10C2A000FEF712FEB8F81030B8F808200C9003EB37
:10C2B00083035B00ADF84A304FF47A70D8F8003051
:10C2C0008DF84C900E93B8F80E1098F814E0D8F84A
:10C2D00004308DF84DE000FB02F24FF0000A4FF001
:10C2E000FF300DF13009CDF834A010920F93ADF866
:10C2F00048101190CC46BCE80F00DFF890E2AEE8A1
:10C300000F009CE80F00AEE807007246182122F8E3
:10C310001C39E17194F87E1184F805A081F078034E
:10C3200083EA0313D8B2030983F0F60343EA002338
:10C3300083EAC0031BB283EA0310C0B2C3F307232E
:10C3400083EA101343EA002383EAC0031BB283F09D
:10C35000C80080EA001C5FFA8CFCC3F3072080EA67
:10C360001C1040EA0C2080EACC0000B280F01803D8
:10C3700083EA0313DBB2C0F3072080EA131040EA1C
:10C38000032080EAC30301F1010CFE204FF01E0AD6
:10C390004FF0C80BA0700EF1020E217184F87EC11F
:10C3A000238084F803A084F806B0184612F8011B15
:10C3B000414081EA0111C9B20B0983EA102343EA23
:10C3C000012383EAC10109B288B272452080EDD110
:10C3D00081F0180181EA0111C9B20A0982EA102329
:10C3E00083EA012383EAC1031BB29AB26149228026
:10C3F000DBB2120A04910692059384F8272084F890
:10C4000026308E4601F5D37B04F1220ADEF80000C7
:10C41000DEF80410DEF80820DEF80C30DC46ACE86C
:10C420000F000EF1100ED645E346EFD1DEF8000006
:10C43000CCF800009DF81430DFF854A184F8CC311A
:10C440009DF8183084F8CD31D3461BF8011F2868B9
:10C450000CF0B6F94A4B5B45F7D1FEF735FDD8F83D
:10C4600000103B68B8F808200591D8F80410069130
:10C4700013F0140F4FF47A7101FB02F141F01D85A6
:10C480000F4694F87EB10C908BF06A003D4BDFF8BC
:10C4900004E1B3F90420109780EA0010C0B2030948
:10C4A00083F0D50343EA002383EAC0031BB283EA87
:10C4B0000310C0B2C3F3072383EA101343EA002337
:10C4C00083EAC0031BB28EFB020E05980D90D217B3
:10C4D0004FF00008C2EBAE0206980E9083F0C80C35
:10C4E0000F91ADF84A20ADF84480ADF84680ADF824
:10C4F00048808CEA0C1CCE465FFA8CFCC3F30727FD
:10C50000BEE80F0087EA1C1747EA0C2787EACC072A
:10C51000DFF878C084F804B03FB2ACE80F0087F0D1
:10C5200021039EE8070083EA0313DBB2C7F3072762
:10C5300087EA13170BF1010E47EA03278CE807007F
:10C5400087EAC30384F87EE14FF0210B4FF0FE0E23
:10C550001C27C8220CF10C0C84F8058084F807B065
:10C5600084F802E0ACF11C01E7701846A271238048
:10C5700012E000BF32290020F495002052960020DE
:10C58000FD2A002000960020409F0020382900202E
:10C59000D72A00206766666611F8012B424082EABE
:10C5A0000212D2B2130983EA102343EA022383EA78
:10C5B000C20212B290B261452080EDD182F06802D1
:10C5C00082EA0212D2B24FEA121B8BEA102383EAEC
:10C5D000022B8BEAC20B0FFA8BFB1FFA8BF3DB4F9C
:10C5E00023805FFA8BFB1B0A059384F8253084F8BF
:10C5F00024B007F5D37C04F1220838687968BA685A
:10C60000FB68E646AEE80F0010374745F446F4D124
:10C610003B88AEF800309DF81430CD4F84F8CAB195
:10C62000D04684F8CB3118F8011F28680CF0C8F800
:10C630004745F8D194F87EC1C64A84F804C08CF00E
:10C64000EB0383EA0313D9B20B0983F0C50343EA72
:10C65000012383EAC1031BB283EA0310C0B2C3F310
:10C66000072181EA101141EA002181EAC00109B2E3
:10C670000CCA81F0C80787EA0717FFB24FF0000E17
:10C68000C1F307210D93CDF838E081EA17130C921E
:10C6900099E8070043EA072383EAC7030FFA83F800
:10C6A000AD4B84F805E088F0310783E8070087EA9E
:10C6B0000717FFB2C8F3072383EA171343EA0723D8
:10C6C00083EAC703277A607AA27AE17A94F80CE0C9
:10C6D00094F811801BB25F4087EA0717FFB2C3F3DB
:10C6E000072383EA171343EA072383EAC7031BB22E
:10C6F000584080EA0010C0B2C3F3072383EA101346
:10C7000043EA002383EAC0031BB25A4082EA0210C4
:10C71000C0B2C3F3072282EA101242EA002282EA80
:10C72000C00212B2514081EA0111C9B2C2F307231B
:10C7300083EA111343EA012383EAC1031BB28EEAA1
:10C74000030E8EEA0E1E5FFA8EFEC3F3072383EA02
:10C750001E1343EA0E23677BA07BE17B227C83EAE6
:10C76000CE031BB25F4087EA0717FFB2C3F307236C
:10C7700083EA171343EA072383EAC7031BB258402F
:10C7800080EA0010C0B2C3F3072383EA101343EA20
:10C79000002383EAC0031BB2594081EA0111C9B2E8
:10C7A000C3F3072383EA111343EA012383EAC10396
:10C7B0001BB25A4082EA0212D2B2C3F3072383EAC1
:10C7C000121343EA022383EAC2031BB288EA030876
:10C7D00088EA08185FFA88F8C3F3072383EA181376
:10C7E00043EA082383EAC803A17CE27CDFF8748172
:10C7F0001BB2594081EA0111C9B2C3F3072383EA8E
:10C80000111343EA012383EAC1031BB25A4082EAAF
:10C810000212D2B2C3F3072383EA121343EA0223BC
:10C8200083EAC2031BB283F0270787EA0712D2B25A
:10C83000C3F3072787EA121747EA022787EAC207E6
:10C840003FB20CF10103BAB25FFA87F94FF0310C35
:10C85000FE200C2184F87E31C8234FEA122E22805C
:10C8600084F807C0A070E170A37184F81490049F4D
:10C8700084F815E07968BA68FB683868B7F810C0C2
:10C88000A8E80F0028F803CB84F8BBE184F8BA913C
:10C890001AF8011F28680BF093FFD045F8D194F8DF
:10C8A0007671002F41F031802C4B94F87E81B3F9E2
:10C8B0000010B3F90220B3F904309FED296A6771C3
:10C8C00007EE103A029B1B680C9388F06A0383EA18
:10C8D000031306EE901AD9B20B0983F0D50343EA8D
:10C8E000012383EAC1031BB283EA03115242C9B296
:10C8F00007EE902AC3F3072383EA111343EA0123C7
:10C90000F8EEE77AF8EEE66AB8EEC77A83EAC10392
:10C910001BB267EE867A66EE866A27EE067A0020FC
:10C9200083F0C80ECDED0E7ACDED0D6A8DED0F7A48
:10C930001090119012908EEA0E1C0DF130095FFAE2
:10C940008CFCC3F3072EB9E80F000DE0322900205C
:10C95000FB2A002060430020382900200096002098
:10C9600088C3E43AD82A00208EEA1C1E4EEA0C2E18
:10C970008EEACC0EDFF888C40FFA8EFEACE80F000A
:10C980008EF01E0799E8070087EA071A5FFA8AFA0D
:10C99000CEF3072787EA1A1747EA0A278CE8070029
:10C9A00087EACA071C214FF0050A4FF01E094FF015
:10C9B000FE0EC82208F10103E17084F876A184F824
:10C9C000079084F802E0ACF11001A2710CF10C0C9C
:10C9D00084F80480278084F87E3111F8013B7B4085
:10C9E00083EA0313DBB21A0982EA172242EA03221E
:10C9F00082EAC3031BB29FB261452780EDD183F069
:10CA0000270383EA0313DBB21A0982EA172282EAB8
:10CA1000032282EAC3031BB21FFA83FCDFF8E4831C
:10CA2000A4F800C05FFA83FE4FEA1C2C84F825C0EE
:10CA300084F824E008F5D37904F1220AD8F800003C
:10CA4000D8F80410D8F80820D8F80C304F460FC793
:10CA500008F11008D045B946F0D1E04FB8F80030E1
:10CA6000A9F8003007F1240884F8CAE184F8CBC1A2
:10CA700017F8011F28680BF0A3FEB845F8D194F809
:10CA800077A1BAF1000F40F03A87D54B1B68052219
:10CA900084F877219A0641F17380D24ADFEDD27A89
:10CAA000D18907EE101AB8EEC77A13F0140F27EEEB
:10CAB000277A01F0C084CD4BDFEDCB6AD3ED007A4D
:10CAC000F8EEE77A67EEA67A94F87EC1C84BC94AB9
:10CAD000B3F90410B2F90620C74FC8488DED0D7A9E
:10CAE0008CF0220383EA03135FFA83FE4FEA1E13DE
:10CAF00083F0590343EA0E23B2F5FA6F83EACE03BB
:10CB00001BB2A8BF4FF4FA6283EA0318B2F57A7F2A
:10CB10005FFA88F8C3F3072EB8BF4FF47A72A2F514
:10CB20007A728EEA181E642303FB02F34EEA082E83
:10CB300087FB03278EEAC80EDA17C2EBA71280FB29
:10CB400001300FFA8EF7CB174FF0000BC3EBA003A9
:10CB500087F0C8080DF13009CDED0E7AADF842200E
:10CB6000ADF84030CDF830B0CDF83CB0CE4688EAD4
:10CB70000818BEE80F005FFA88F8C7F3072787EAAE
:10CB8000181747EA082787EAC8089D4FDEF800E033
:10CB900084F804C00FC70FFA88F888F04A0383EAC4
:10CBA0000310C0B2C8F3072383EA10133A460CF10E
:10CBB000010143EA002383EAC00342F810E90020A0
:10CBC0004FF04A084FF0FE0C4FF0140E84F87E111F
:10CBD000C82160712380043784F8078084F802C07C
:10CBE00084F803E0A171184612F8011B414081EA64
:10CBF0000111C9B20B0983EA102343EA012383EA36
:10CC0000C10109B288B2BA422080EDD181F014018D
:10CC100081EA0111C9B24FEA111E8EEA102E8EEA86
:10CC2000012E8EEAC10E774B0FFA8EFE1FFA8EFC94
:10CC30001F464FEA1C2B5FFA8EFE84F81DB084F865
:10CC40001CE0596838689A68DB68A4F800C007F5EA
:10CC5000D37CACE80F0038697969B7F8188004977D
:10CC6000ACE8030004F2A717ACF8008084F8C3B165
:10CC7000B84684F8C2E104F2C31B18F8011F286803
:10CC80000BF09EFDC345F8D15F4B604A1B781278CC
:10CC9000013B12F00100DBB214BFC0214021172B71
:10CCA00003D85B4A134493F80CA05A4B1A88930795
:10CCB0001ABF002341F01001012312F4027F18BFB4
:10CCC000022312F0100F18BF062312F0200F18BF16
:10CCD0001023002841F03C814FF0030894F87EC1F6
:10CCE0000C938CF0460383EA0313DAB2130983F042
:10CCF000920343EA022383EAC2031BB283EA0310CE
:10CD0000C0B2C3F3072282EA101242EA002282EA8A
:10CD1000C00212B282F0C80E8EEA0E1E00235FFA25
:10CD20008EFE0320C2F307228DF834A08DF83780E1
:10CD300082EA1E128DF835308DF836108DF83800E5
:10CD400042EA0E2899E8070088EACE0E0FFA8EF81C
:10CD5000DFF8ACA0E37188EA0819AAE803005FFADB
:10CD600089F9C8F3072888EA191848EA092181EAED
:10CD7000C90994F808808AF800200FFA89F988EA2E
:10CD8000090282EA02185FFA88F8C9F3072282EAE8
:10CD9000181242EA0822607AA17A94F80B90637123
:10CDA00082EAC80212B2504080EA0010C0B2C2F358
:10CDB000072282EA101242EA002282EAC00212B27C
:10CDC000514081EA0111C9B2C2F3072282EA11126D
:10CDD00042EA012282EAC1021EE000BFD72A0020F7
:10CDE000F4950020409F00200AD7233CF8950020AE
:10CDF0000096002008470020D34D621067666666E3
:10CE00003829002032290020404000201C770020D3
:10CE1000A84704085096002012B289EA020989EA5C
:10CE200009195FFA89F9C2F3072282EA191242EA64
:10CE3000092294F80C80607BA17B84F804C082EA0C
:10CE4000C90212B288EA020888EA08185FFA88F86C
:10CE5000C2F3072282EA181242EA082282EAC802D2
:10CE600012B2504080EA0010C0B2C2F3072282EA38
:10CE7000101242EA002282EAC00212B2514081EA54
:10CE80000111C9B2C2F3072282EA111242EA012259
:10CE900082EAC102E17B94F8109013B281EA0302A6
:10CEA00082EA0212D2B2C3F3072383EA121343EADF
:10CEB000022383EAC2031BB289EA030282EA021256
:10CEC000D2B2C3F3072383EA121343EA022383EAAD
:10CED000C2031BB283F0320282EA0212D2B2C3F35F
:10CEE000072383EA121343EA022383EAC2031BB235
:10CEF0009AB24FF0FE085FFA83FE0920C8210CF1B8
:10CF0000010C84F802804FEA1228E070A17184F8C5
:10CF10007EC1228084F8128084F811E0049B186896
:10CF200059689A68B3F80CB00AF5CC7CACE80700F5
:10CF30000AF5D47A8CF80290ACF800B084F8B88185
:10CF400084F8B7E117F8011F28680BF039FCBA45DF
:10CF5000F8D1039BC4F86831FEF73ABEDFF83C8392
:10CF6000BF4FDFF83CA3412027F0C6F8B8F90220F4
:10CF700087FB0230D217C2EBA00080B227F0A0F8E6
:10CF8000B8F9002087FB0230D217C2EBA00080B2B4
:10CF900027F096F8B8F9042087FB0230D217C2EBCD
:10CFA000A00080B227F08CF89AF80010D9F80000A1
:10CFB0000BF006FC94F8608118F0010700F0338450
:10CFC000A84F3A68910640F18180A74ADFF8D482E1
:10CFD0001278920740F1678798F81420042A8CBFD2
:10CFE000032302230393472027F086F8D8F8000094
:10CFF00027F032F8D8F8040027F02EF8B8F80E2001
:10D000009A49D9F80000A1FB0232C2F34712114637
:10D0100004920BF0D5FB9AF800003968049A11F0DD
:10D02000140F82EA00028AF8002040F09786B8F8D0
:10D030000820642000FB02F027F00EF898F8147026
:10D04000039BD9F8000043EA8707FFB239460BF08B
:10D05000B7FB9AF80020D9F80000574039468AF803
:10D0600000700BF0ADFB94F86081B8F1000F2DD18A
:10D070007F4F4F2027F040F8386826F0EDFF7868A2
:10D0800026F0EAFF404626F0E7FF0121D9F800002C
:10D090000BF096FB744A9AF800701278D9F80000E9
:10D0A00002F00108414687F001078AF800700BF092
:10D0B00087FB9AF80020D9F8000088EA020211469E
:10D0C0008AF800200BF07CFB94F86081694AC4F870
:10D0D0005CB108F10103DBB2A2FB0312D20802EB40
:10D0E0008202A3EB420384F86031FEF751BD624B2C
:10D0F00062491868FEF79EF900232370FEF7F1BD20
:10D100005F4F386800283EF430AD4FF0000ADFF87A
:10D1100098815C4CAB465546FEF7C0F9F8B1F5B9BD
:10D120004FF00109AA463868FEF7B0F983B27E2BAA
:10D1300000F05D8398F80120002A49D194F84C1141
:10D14000B1B11B2B84F84C2100F02B830D2B45D063
:10D15000386888F80190FEF7A1F90028E3D1AA46C3
:10D1600050460CAA48495D462EF0CAF8FEF7FDBCB1
:10D170007D2B00F0F18494F8502122B180F020033F
:10D18000DBB284F8501194F84B21062A10D8B4F879
:10D190004E1138681944A4F84E11A118013281F8D3
:10D1A000543184F84B21FEF779F90028BBD1D6E73A
:10D1B000B4F84E2188F8019013449BB21A0A52FA2F
:10D1C00083F3FF2BA4F84E31386802D12F4DA3E72B
:10D1D0003868FEF763F90028A5D1C0E73868A4F8DD
:10D1E0004E21FEF75BF900289DD1B8E794F8BC32D8
:10D1F000C4F8B862012B40F2988494F8BD22244907
:10D20000981801EB8001013202F001024F6A84F8A4
:10D21000BD22BFB11F4D0D950DF15009123DA52343
:10D2200049F8205D802284F81031152331464846A4
:10D2300084F8112184F81231B847002840F0F683B1
:10D2400094F8BC32144A013382FB0312A2EBE3725E
:10D2500002EB42029B1A84F8BC32FEF7C9BC00BF45
:10D2600067666666F4950020529600201F85EB5194
:10D2700060430020CDCCCCCC90970020B896002005
:10D2800060960020302900207A2A0020842A00207D
:10D29000A8470408552A00205655555500960020E9
:10D2A000607A0020409F002004000020C54AC64B41
:10D2B00092F80BE0029AD4F8381110681B88C34A20
:10D2C000401A4FF47A71DFB201FB0EF11B0A977717
:10D2D000177588424FF00007D37753759770177111
:10D2E00080F00F84BA4BDFF814C31B68B949BA4FFA
:10D2F0000868DFF80C9389683F688CFB038EDB17A6
:10D30000C3EB6E1303F5FA739BB293761B0AD376C5
:10D3100089FB00A389FB01A9C017C917C0EBA300B3
:10D32000C1EBA90107F5EA43DFF8D8E21077303303
:10D33000001282F8201009121B12DFF8CC829EF82E
:10D3400000E0507782F821108CFB0790F917C1EBB1
:10D35000601182F82330A14B98F814A083F81AA02A
:10D36000783130371EF0020F82F8241082F82270D4
:10D3700000F0C483D8F800E0994AD8F80400DFF838
:10D380008CB282FB0E714FEAEE77C7EBA15103918D
:10D3900082FB0092C117C1EBA25203990BFB01E182
:10D3A00001EB410149000F460BFB020B0497B94604
:10D3B0000BEB4B0B8B4F4FEA4B01059187FB099B06
:10D3C00087FB01194FEAA949CDF81C90B8F80E90D7
:10D3D0000399B8F8088002EB820209EBC90902EB55
:10D3E0008202089201EB81074FEA890205990392B4
:10D3F00007EB8707049A0697CF17C10F0991049886
:10D4000079494FEAAB4BD2174FEADE7E83F809E049
:10D41000ABEB020E01FB1E020798069908F5FA789D
:10D42000BAF1050F1FFA88FAA0EB0708059F6E48AE
:10D4300083F815A04FFA8EF909EB8109414600FBEC
:10D4400018789DF8240098730898684FDFF8C0E1B9
:10D4500049B201EB80018CFB020B4FEAE2720492AD
:10D46000039ABEF800E08CFB08C087FB02C74FEAB6
:10D47000E27C049AC2EB6B1203925D4A1FFA89F9AF
:10D480001288ADF8102083F80A90039A83F813E00D
:10D4900089B24FEAE8784FEA112BC8EB6010CCEB69
:10D4A000A7174FEA1A284FEA192C4FEA222A9DF8AB
:10D4B0000C2083F810B04FEA202983F80BC0D973F1
:10D4C000C7F3072C4FEA1E2134BF4FF0320B4FF049
:10D4D000330B1A739DF8102083F80DA0587483F84D
:10D4E000129083F81680DF7183F808C0197583F8ED
:10D4F0001BB01A77C4F83461FEF7C9BADFF814918B
:10D50000D9F80000FDF7BAFF00283EF44FABD9F878
:10D5100000000121FDF7AEFF0222002387F87420EE
:10D5200088F80030FEF742BB5E209047D9F8003003
:10D5300030209847284BD3F800805FFA88F02EF00F
:10D540008BFAC8F307202EF087FA94F82C3113F0E9
:10D55000030800F0B783D9F80020FEF781BADFF89E
:10D56000B8809FED248A4FF0240A5E2090475046F1
:10D57000D9F800309847204BF8EC016A9B8A07EEF7
:10D58000103AF8EEE66AB8EEC77A0AF1010AC6EE7A
:10D59000877A5FFA8AFA67EE887AFDEEE77ACDED50
:10D5A000027ABDF908B05FFA8BF02EF055FACBF392
:10D5B00007202EF051FABAF1270F00F0ED80D9F8CC
:10D5C0000020D2E79078002088780020349700204F
:10D5D000F8950020CC950020FC9500206097002055
:10D5E0006BCA5F6B83DE1B4340420F00D34D62105A
:10D5F000EC53002000007A44089600201F85EB5170
:10D600006766666652960020409F0020806967FF2B
:10D610005C9600201C330020389600205E20904746
:10D62000D9F8003002209847FF2026F065FA0378E9
:10D63000FF2B00F0358490F901304FEAE3785FFA70
:10D6400088F8D8B22EF008FA40462EF005FAD9F83C
:10D6500000305E209847D9F8003003209847FF201B
:10D6600026F04AFA0378FF2B00F01584B0F9083051
:10D67000D8B2C3F307282EF0EFF940462EF0ECF9AC
:10D68000C84B1B78042B7DD0DFF854B3B4F82E11AF
:10D690009BF80020DFF834A391FBF2F302FB131395
:10D6A0009BB2BAF80010A4F82E314FEA03181FFA03
:10D6B00088F8642303FB01235200B3FBF2F348EA2A
:10D6C0000328C3F303225E20D9F800301FFA88F83C
:10D6D00048EA02089847D9F80030062098475FFAD0
:10D6E00088F02EF0B9F94FEA18202EF0B5F9AE49BE
:10D6F000B4F82E214B7ABAF800A00132012BA4F81D
:10D700002E2100F082864A7B0AEB8A031FFA83FAF5
:10D71000002A40F02784D9F800305E209847D9F8D5
:10D7200000303A209847A14BA3FB0A384FEA58181B
:10D730001FFA88FB5FFA8BF02EF08EF94FEA1B2060
:10D740002EF08AF9D9F800305E209847D9F80030D9
:10D750003B209847642303FB18A39BB294480533EE
:10D7600080FB0320DB17C3EBA000C0B22EF074F9DE
:10D7700000202EF071F9DFF86C8298F80630002B4B
:10D7800040F0AD833B68980600F1058294F82C3197
:10D79000D9F80020FEF768B93968D9F80020FEF7FB
:10D7A00059B93868FDF77AFE00287FF4D1AC3868A3
:10D7B00084F84A9188F80190FDF770FE00287FF404
:10D7C000B2ACCCE4FDF780FB7A4B1B68A0EB030BFB
:10D7D00040F6B8339B4500F2B481774B1A793A2A68
:10D7E00000F03C85002388F80030FEF7DFB9386888
:10D7F00084F84AA184F84BA184F84C9188F801A0E0
:10D80000FDF74CFE00287FF48EACA8E494F8481194
:10D8100094F8493169484A1CFEF793B9013A84F8F3
:10D820006F21FEF721BD664A1288D30513D4D006B6
:10D8300000F14183910600F1D585530600F102867F
:10D84000100700F10286D10700F1418612F0020FA5
:10D850000CBF04270C275B495B4A0B78D27803F096
:10D8600001030AB143F002035320039326F044FC62
:10D87000564A128802EB820202EB8202900080B2CA
:10D8800026F01EFC002026F01BFC514A514912884C
:10D89000D9F80000C2EBC212520081FB02311144E0
:10D8A0004FEAE278C8EB61285FFA88F841460AF04F
:10D8B00087FF9AF80020039BD9F800001F4388EAED
:10D8C000020800218AF800800AF07AFF3946D9F868
:10D8D00000000AF075FF9AF80020D9F800007A409D
:10D8E000D2B211468AF800200AF06AFF94F86081EB
:10D8F000FFF7BBBB013B84F86E31FEF78DBB0AF12D
:10D90000FF3A84F877A1FFF724BB013F84F87671D2
:10D91000FFF7B5B8013B84F87231FEF7C0BF4FF096
:10D92000000A5E201F6884F82CA19047D9F80030C7
:10D93000DFF8B4801720984750462EF08DF8264B1C
:10D94000A3FB07239B0BA8FB03125209C2EB021295
:10D95000A3EB8203D8B22EF07FF8D9F800305E2016
:10D960009847D9F80030182098471C4BA3FB072391
:10D970009B09A8FB03125209C2EB0212A3EB82031C
:10D98000D8B22EF069F850462EF066F8D9F800208B
:10D99000FEF76FB80024DFF8548027464FF0500A96
:10D9A00029E000BF4C450020907800201F85EB51F6
:10D9B0006766666600320020E83100206496002029
:10D9C000509600201C7700203041002088780020ED
:10D9D000384700200308208073B2E745D34D62101A
:10D9E0009E780020E495002089888888C1BB0308C0
:10D9F000DBB283F3118815F804B0601C5946284443
:10DA000026F028FA002840F0A2810BF101031C4403
:10DA1000EFF311838AF312882A6E9442E8DB002226
:10DA2000DBB22A6683F31188FEF7E0B90C9EAE42A2
:10DA30004FF000014FD941F2210015F8013B81EA76
:10DA400003235A0013F4004F80EA020192B289B214
:10DA500008BF11464A0080EA020311F4004F99B250
:10DA600093B218BF0B46590080EA010213F4004F2D
:10DA700089B293B208BF0B465A0013F4004F80EAF4
:10DA8000020192B289B208BF11464A0080EA02033D
:10DA900011F4004F99B293B218BF0B465A0013F419
:10DAA000004F80EA020192B289B208BF11464B00D2
:10DAB00011F4004F80EA03029BB292B208BF1A46EB
:10DAC000530080EA030112F4004F9BB289B208BFF1
:10DAD0001946B542B1D148460CF0D4F8A1490C9D85
:10DAE000A1486D1A152DA8BF15252A4635F03CFC16
:10DAF0009E4A94F8BC321570FFF7A4BB2D22DA764B
:10DB0000F8E49B4B02991B780968C4F83811013B73
:10DB1000012B3FF6E7AB1021022391701371FFF741
:10DB2000E1BB2DF07BFFFEF714B8924A02EB8302B3
:10DB3000576AFFF76EBB2DF061FF01233B70FDF7C5
:10DB4000C5BF8D4AB2F8623100210133A2F86231BB
:10DB500088F80010FEF72AB8386884F85091FDF76D
:10DB60009DFC00287FF4DFAAFFF7F9BA014684463E
:10DB7000074682460490804605900246FEF783BA27
:10DB80009FED7E7A13F0140F08BFF0EE477A7EF413
:10DB900092AFFEF799BFDFF8FCA19AF80030990721
:10DBA00000F10C82DFF8F0810027BB46D9F8003085
:10DBB0005E209847D9F800300120984758462DF04C
:10DBC0004BFF38462DF048FFD9F800305E209847CB
:10DBD000D9F800300920984700202DF03DFF0020A3
:10DBE0002DF03AFFB8F8123098F81470B3F5967F1C
:10DBF0000AD994F82C2102F00F02072A04D842F225
:10DC00000F779F4228BF1F46D9F80030DFF88CB14C
:10DC10005E209847D9F80030052098479BF80830D7
:10DC2000002B00F0EB83A7F1200307EE903A9FED65
:10DC3000547AF8EEE77AF6EE006A67EE877ABEEE7F
:10DC4000007AF5EEC07AF1EE10FA58BFB0EE667ABF
:10DC500077EE877AFDEEE77ACDED027ABDF90870AE
:10DC6000F8B22DF0F9FEC7F307202DF0F5FE9AF873
:10DC7000002000230A930B93930700F1258194F869
:10DC80003031012B00F02081BBF90030DFED3D6A1F
:10DC900007EE103ABBF9023007EE903AB8EEC77AB9
:10DCA000F8EEE77A27EE267A67EEA67ABDEEC77A17
:10DCB000FDEEE77A0CA88DED0C7ACDED0D7A2DF006
:10DCC000EDFE63E53049D4F82821304B8A421868CC
:10DCD00040F23A8180EAE073A3EBE0732C4A1BB276
:10DCE00082FB03124FEAE37BCBEB621B4FF064082D
:10DCF00008FB1B380FFA88F80FFA8BFB5FFA88FADB
:10DD00005FFA8BF2C8F30728CBF3072BD9F8003062
:10DD100002925E209847D9F8003010209847029A66
:10DD200010462DF099FE58462DF096FED9F8003099
:10DD30005E209847D9F800302120984750462DF0B2
:10DD40008BFE40462DF088FE94F82C3103E44146CA
:10DD50003A2025F0DBFF0743FFB256E60B4A106876
:10DD6000FFF76AB9402A0020AC920020C19200203F
:10DD70004C450020A847040830290020000000007E
:10DD8000E4380E3F0050C3473F4B4C00F89500204D
:10DD90001F85EB5152960020409F00209078002074
:10DDA000CC49CD4B0093A1F13F07CC4BCC4A0B9112
:10DDB00001F8404C0CA8CB490A970CF03BF80A9F9D
:10DDC0007B1C0A933C700A9B2922591C0A911A70E9
:10DDD0000A9BEA22591C0A911A700A9BC822591CF4
:10DDE0000A910CA81A7034F033FB00F101080CA959
:10DDF00042460A9835F0B8FA0A9A02EB0803013352
:10DE00000A9302F808400A9B5A1C0A921C700A9B4B
:10DE10005A1C0A921C700A9B5A1C0A921C700A9B7C
:10DE20005A1C0A921C700A9B5A1C0A921C700A9B6C
:10DE30005A1C0A921C700A9B5A1C0A921C700A9B5C
:10DE40005A1C0A921C700A9B5A1C0A921C700A9B4C
:10DE50005A1C0A921C700A9B5A1C0A921C700A9B3C
:10DE60005A1C0A921C700A9B0122991814A80A9144
:10DE70001A7050F8283DDB1B3B702DF087FE9A4B43
:10DE80002C70C3F8B062FDF7A7BEC4F83C6187F8F8
:10DE90000080FDF71BBE4FF000084046FFF7EBBBCC
:10DEA0004046FFF7CFBB01230393FFF79CB8FDF774
:10DEB000E1FAFDF720BE3427CDE48C4B1F6807EB59
:10DEC00087077F00FEF7DDBA98E80C0001210AA859
:10DED00084F830110A920B932DF0E0FD56E4D9F846
:10DEE0000030DFF828A2DFF820B25E209847D9F88A
:10DEF000003028209847DAF800308BFB032BDB1723
:10DF0000C3EBAB0B5FFA8BF02DF0A6FDCBF3072034
:10DF10002DF0A2FDD9F800305E209847D9F80030E6
:10DF200004209847B8F80830002B40F05E82DAF8F9
:10DF3000083083F310085FFA88F02DF08DFDC8F3E8
:10DF400007202DF089FD1DE4C246C3464246DDE6AA
:10DF5000674AD278002A0CBF4FF004084FF005083A
:10DF6000FEF7BCBE9BF800309AFBF3FAFFF7D3BB79
:10DF70000123D9F800003B70FDF788FA0746D9F86D
:10DF80000000FDF783FA7F067DF4A0AD8A2800F03B
:10DF90008D828E287DF49AAD9AF80030002B7DF4A6
:10DFA000B1AD5448544B03602D2384F840310768C9
:10DFB000FDF790BD4FF00109FEF772B9DFF850810F
:10DFC000D9F800304D4F5E209847D9F80030112025
:10DFD0009847B8F80E204FF4F36B0BFB02F287FB67
:10DFE0000237D217C2EB6737F8B22DF035FDC7F311
:10DFF00007202DF031FDD9F800305E209847192018
:10E00000D9F800309847B8F80E303D4A0BFB03F3BF
:10E0100082FB0301DB17C3EB611382FB0321DA17D9
:10E02000C2EB6112642101FB1233D8B22DF014FD52
:10E0300000202DF011FD9AF80030B8F808709A070A
:10E040007FF5B2AD5FFA87FB3F0AAFE5214A2D4B62
:10E050000D920DF15008A2F13D0048F8200D1988ED
:10E06000DFF8A890A2F1400300204FF00A0E02F85A
:10E07000400C082283F801E040469A700BF0DCFD6A
:10E08000D9F800302049DA1781FB0313C2EBA30350
:10E0900099B240460BF0D0FD22F02CFCD9F8089044
:10E0A0000C9B4FEA1942591C0C911A700C9B4FEAB9
:10E0B0001922591C0C911A700C9B5A1C0C9283F853
:10E0C00000900C9B5A1C0C92187040462DF05EFD7F
:10E0D000FDF72ABEB89600207E590020547A040825
:10E0E0005C7A0408687A040830290020F89500203A
:10E0F000304100206C9600203497002089B5F81438
:10E100001F85EB518878002067666666CC950020F5
:10E11000409F0020DFF884939FEDCF8AB9F9023049
:10E12000CE4A0D9207EE903AF8EEE77A0DF15008DC
:10E1300067EE887AA2F14003FDEEE77AA2F13D0195
:10E1400048F8201D02F8400C0822CDED027A5A70E2
:10E150001E229A70BDF8081040460BF06DFDB9F90B
:10E16000003007EE903AF8EEE77A404667EE887A9C
:10E17000FDEEE77ACDED027ABDF808100BF05CFDFC
:10E18000B9F9043007EE903AF8EEE77A404667EEC8
:10E19000887AFDEEE77ACDED027ABDF808100BF033
:10E1A0004BFD40462DF0F2FCFDF7BBBDAB4B0D9394
:10E1B000A3F1400900222121A3F13D0A03F8402CDC
:10E1C00089F8021089F80120CDF830A030F04CFF1A
:10E1D000A34BA44A1B88A44900280ABF11464FF04C
:10E1E00003084FF004085A0500F12181D80700F117
:10E1F0002F8103F002039D4A002B1CBF4FF0030840
:10E20000114642469A4835F0AFF80AEB080314A8C5
:10E21000984A013340F8203D9B1A00220AF8082052
:10E2200089F801302DF0B2FCFDF781BD924B934A85
:10E230001B88927903EB830303EB83034FEA830884
:10E240001FFA88F8002A00F045818D4B1B680FFAF1
:10E2500083FA22F04FFB40B2FDF719BE9978039381
:10E26000184613F0BDFF00287FF4BCAA8249854FF1
:10E27000834A09888448854CF961DFF82492116843
:10E2800003689268F962B4F86211C7F86CB0FB6376
:10E29000FA64D9F80000F965FBF78EFA8346002886
:10E2A0007DF47FAC5146D9F80000FDF7E3F8039BFD
:10E2B00094F86421DB780493642A4FF0040387F810
:10E2C000743040F02B8194F86531DFF8D8A1072B2A
:10E2D00008BF84F865B194F86521069207EB021B2C
:10E2E000DBF804100591084634F0B2F8DBF808308A
:10E2F00003935FFA80FB184634F0AAF8C3B20BEB25
:10E300000300069A0599059308308AF8070022F061
:10E310000F008AF80A0002F00F0203EBCB008AF824
:10E320000D208AF80E005A460AF10F0035F01CF84D
:10E33000059B03990BF109001A460AF106031844DC
:10E3400035F012F89AF8073003F1010BD3B1013B15
:10E350005FFA83FC0CF1080CDFF84CE1D4440AF1BD
:10E360000700002310F8011B59408B00CA0883EAFC
:10E37000410302F018024B404EFA02F2534084452A
:10E38000DBB2EFD1424A04980BF8023034F0C8FFF8
:10E3900094F865310022013384F8653184F86421F2
:10E3A0009AF802305BB11AF80510D9F800000AF0AB
:10E3B00007FA01359AF80230EDB2AB42F3D894F87F
:10E3C00064310322013384F8643187F8742088F8BB
:10E3D0000020FFF795B811469446174692460492DE
:10E3E000FDF751BE2427FFF736BA22F083FA2DF04D
:10E3F00033FB00202DF030FBFFF7C4B9F8B22DF04D
:10E400002BFB380A2DF028FB31E4D9F800305E20D0
:10E410009847D9F80030392098475FFA8AF02DF0F4
:10E420001BFB4FEA1A202DF017FBFFF7A4B94FF0A2
:10E4300003081849E5E6138907EE903AF8EE677A83
:10E44000FEF742BB1027FFF706BA2027FFF703BAF3
:10E4500011494FF00408D4E658A08B41B89600202B
:10E4600050960020387A0408407A0408507A04084C
:10E470007B9600207996002088780020E495002083
:10E48000CC95002004000020F895002030290020C1
:10E4900082B10020447A0408487A040800960020DB
:10E4A0001C3300207CB100200007090E614B1B6863
:10E4B00098067DF50BAB9AF80030002B7DF422AB6B
:10E4C0005D485E4B03602D2384F840316FE50827DB
:10E4D000FFF7C1B94FF0FF33B9E6594B8046B3F9A6
:10E4E00000A06420FDF7D3BC11469446174692461F
:10E4F00004929046FDF7C7BD1146FDF7C4BD114615
:10E500009446FDF7C0BD114694461746FDF7BBBDC6
:10E510001146944617469246FDF7B5BD97F87530FB
:10E52000DFF82CA1474905951A0704BF0133DBB278
:10E53000072B28BF01234FEA031B07EB0B02107CBC
:10E5400000228AF80A2011F800C05FFA8BF20392C9
:10E550000AF10D02039D07EB0B012843BCF1010FEB
:10E560001070C96802F101000ED9ACF10205EDB2DC
:10E5700005F1020E9644024602F8011B72454FEA6D
:10E580001121F9D101352844BB4421F06002013347
:10E590009BF81110DBB20A43082B027000F1010254
:10E5A00044D04FEA031B07EB0B00264D007C2649A5
:10E5B00015F800C0039D511A05F1100E01EB0C0572
:10E5C00006955FFA8EF50395069D132DC2DD059D18
:10E5D000DFF880E0C9B28A1DD2B242F040008AF86A
:10E5E000070002F1010BCAB14A1DD2B208325244EF
:10E5F00003920EF1010C00221CF8010B5040820026
:10E6000082EA4002C1084240104801F0180140FA75
:10E6100001F14A4003996145D2B2EDD104980BF85B
:10E620000E2087F8753034F07BFEB9E60649059D6B
:10E63000511ACDE7F49500206C96002060970020D9
:10E64000CC950020A847040889B100200007090ED6
:10E650007CB1002082B100202DE9F047C44B1C683A
:10E6600062072DED028B03D4BDEC028BBDE8F08771
:10E67000C04D2B78002BF7D06E6846F2A713861B8F
:10E680009E42F1D9DFF850936860B9F80070DFF866
:10E690004C83002F40F0A68198F80620AB689FEDD0
:10E6A000B60ADFEDB60ADFF8F492013AB3FBF2F3F3
:10E6B00007EE903AF8EE677AB7EE008A27EE800A06
:10E6C00035F0EEF8DFEDAE7A38EE400A20EE270A9C
:10E6D00035F01EF8B8F80830DFEDAA6A07EE103AF8
:10E6E000EB68C01AB8EEC77A07EE900AA7EE668A02
:10E6F000B8EEE70AD9ED097AF8EEE77A20EE080AD3
:10E7000067EEA67AA7EE270A35F002F89E4BC9F805
:10E71000240002461860A30740F1AA81DFF8C0E296
:10E720009A4CDEED007A9FED9A5A2168F8EE677AEE
:10E7300027EE855A002900F0BB81964B07EE101A90
:10E74000D3ED026AB8EEC77AF8EEE66A86EE878AFB
:10E75000914991ED004AB8F80C10D5ED054ADFED6E
:10E76000895A95ED066A67EE847A06EE901A67EE8E
:10E77000887A8A49B6EE004AF8EEE66AF0EE643A24
:10E78000E7EE843A66EEA56A91ED097A7E49F7EEE6
:10E79000005A75EEE65AB8EEC77AA3EE856A77EEB0
:10E7A000A47A27EE257AC5ED057AF0EE477AE6EEF3
:10E7B000267ABDEEE77AC5ED067A81ED007A7849D2
:10E7C0000978122900F05B81002119605960996075
:10E7D0002160CEF80010002F7FF446AFE869EA61AF
:10E7E000121A07EE102ADFED6F6A6F4B07EE906A80
:10E7F000B8EEC77AF8EE677A27EE267A40F2DC5256
:10E80000C7EE276A0A21FDEEE67A17EE900A9042DB
:10E81000A8BF10469842B8BF18460BF055FCB8F890
:10E820000A309FED586AD5ED056A07EE103AB8EE4A
:10E83000C77AF7EE007AE7EE467A05EE900AF8EE30
:10E84000E55A66EE866A67EEA57AE7EE267AB0EEBE
:10E85000670AC5ED057A34F05BFF052106460BF02B
:10E8600033FC524A5249B2F90040086084EAE4732A
:10E87000A3EBE473B3F5487F74DAB2F9022082EABD
:10E88000E273A3EBE273B3F5487F6BDA494B1B7875
:10E89000002B40F01181484B3B4A1B6812684748E7
:10E8A0009B1AB3F5FA7FA8BF4FF4FA739842B8BF2A
:10E8B00018460A210BF008FC414B1C68637A00FBE8
:10E8C00003F00028B8BF7F30C211B2F5967F3D4BF0
:10E8D000A8BF4FF496729A42B8BF1A463A48E37EF0
:10E8E000076895ED087ADFED396A911B01FB03F3A8
:10E8F000227F344E002B01FB0272B8BF1F335B1125
:10E90000B2F5C81F3249A8BF4FF4C812B3F5967FBD
:10E91000A8BF4FF496738A42B8BF0A46617F02606F
:10E9200007EE901A37EE087AF8EEE77A27EE267AA5
:10E93000B34267EE877AB8BF3346002AB8BF02F504
:10E94000FF52FDEEE77AB8BF1F3203EB623317EEDA
:10E95000902A962A6FF09501A8BF96228A42ACBFF2
:10E960009F1A5F1A1B4A85ED088A17607CE600BF74
:10E97000F4950020F42B002008942537B1DC423EAA
:10E98000D048874A6F12833AF89500207C9E002079
:10E99000BD3786356C9E0020809E0020643B0020A1
:10E9A000CD8900200024744924FAFFFF009600203E
:10E9B000FC950020F42F0020EC2F00200CFEFFFF20
:10E9C00054960020D4FEFFFFE42F00200000003BFF
:10E9D0000000E7FFDC2F0020A69E002018980020F2
:10E9E000789E0020374998F806A00A68AB689FED2A
:10E9F000360ADFED360A002A0AF1FF3AB3FBFAF3D2
:10EA00009246B8BF02F1070AA2EBEA0203EB020A40
:10EA1000BAF1000F5346B8BF0AF10703DB1007EE47
:10EA2000903AF8EEE77AC1F800A027EE800A34F0B9
:10EA300037FFF7EE007A77EEC07A9FED257A2B69E3
:10EA400067EE877A9A4518BF07F1FF33FDEEE77A44
:10EA500014BF9FB200274FF00003C5ED037A18BF23
:10EA6000C5F810A0A9F800706B61AB61002252E6F6
:10EA70009FED188ADFF870E0174C184B9FE695ED74
:10EA8000057AD5ED067ADFF864C02068996891FBB5
:10EA9000F0F1BDEEC77AFDEEE77A17EE100A17EE39
:10EAA000909AACF80200ACF80010ACF804908BE639
:10EAB0009FED088A094B4BE6094A0A4B12681C680D
:10EAC0000CE700BF7C00002008942537B1DC423EF3
:10EAD000D048874A000000007C9E00206C9E0020E9
:10EAE000F02F002054960020789E0020D08900202E
:10EAF0002DE9F843304B1B685B0701D4BDE8F88370
:10EB00002E4C2F4D94F82490B9F1010F48D1EB69A8
:10EB1000284698472B69284698472B6A04F12C0011
:10EB200004F128019847274B276B9B79A668E06A78
:10EB300007F101089845636B08BF84F8009003F162
:10EB4000010208BF4FF00008032A1FD01E4962636C
:10EB500094F8382041F82300FAB904EB870704EB56
:10EB60008803F863DA6BAB89C4F83080B61A304496
:10EB70000022A06084F82420002BBFD0134A0A2B67
:10EB80001268B8BF0A231361BDE8F8830E4B012257
:10EB90009860002384F83820636331F043F8DCE7A1
:10EBA0006B6928469847AB69284698470122EB894C
:10EBB00084F82420E0E700BFF4950020F42B002027
:10EBC000643B002018980020009F00203898002007
:10EBD0002DE9F04F2DED028B9F4BA04A1C7897B08A
:10EBE00000F59C41203181460A911160002C00F013
:10EBF00006859B4A1268904240F28380994A0792A8
:10EC000016689949994A0691013C1C70984B0492E8
:10EC100006F480560993002E40F08180954B1B78B6
:10EC2000022B00F06587042B00F05487012B00F0C5
:10EC30000887914B9945099B9B7800F2B083002B84
:10EC400040F0B1838D4B0893079B1E6816F48057E4
:10EC500040F0A384DFF85492049BB3F90610069B9E
:10EC60005C8BA142B4BF00240124854B1B6813F0C8
:10EC700080535ED0089A127812F001025FD0069895
:10EC8000408C884241F38E80002C5ED17D4D95F8FA
:10EC90008811002959D17C487C49006890F82D00E2
:10ECA00000250D604D608D60794900284ED10870B7
:10ECB000002A4FD0F1064DD5764A1278D20649D4B3
:10ECC000002F47D1002B45D1750243D4724B1B78DE
:10ECD000002B01F06587714B9B78002C42F000807F
:10ECE0003BB16F4A6F4B12681B689B1A002BC2F234
:10ECF0000C801020634D2DF039FF012385F88931F8
:10ED000028E0584B07931E68584B574A049306F463
:10ED10008056574B06920993002E3FF47FAF002197
:10ED200057480BF0A3FC00287FF478AF10F0D4FC18
:10ED300074E770029ED4089A127802F00102514DD5
:10ED4000002185F88811002CA5D0514901200870B8
:10ED5000002AAFD1544B1A78002A40F0B3800699AC
:10ED6000049D488BB5F90070898BB5F90250874234
:10ED7000CCBF8026002646F040038F42A8BF334612
:10ED80009B0843F080068542C8BF3346049F43F08A
:10ED900040068D42B8BF33469B08B7F90450B7F917
:10EDA000066043F080078542C8BF3B4643F04007FA
:10EDB0008D42B8BF3B469B0843F08007314D8642E9
:10EDC000C8BF3B4643F0400795F88AE18E42B8BF82
:10EDD0003B469E4501F01982A5F88C2185F88E21CD
:10EDE0002D4985F88A310E78002E01F040815F2B85
:10EDF00001F0B5816F2B01F0D081089B1B78DB07F8
:10EE000060D495F88E1100295CD1B5F98C31322B84
:10EE100058DD95F88A210120572A85F88E0101F0E6
:10EE20003985079B1B685C0741F153805A2A41F0E2
:10EE3000508095F89031002B41F0C28695F89231C0
:10EE400083F0010385F89231002B41F03A870C20C2
:10EE50002DF08CFE01F097B91C950020B493002092
:10EE6000189500205C6200201891002008470020BF
:10EE70003041002016940020404B4C001C770020AD
:10EE8000343B0020F42B0020549600204C3B002003
:10EE9000942F002052960020A4220020BC9D002028
:10EEA00034C80020CC3000206F360020D032002043
:10EEB0000F202DF05BFEB5F88C3185F88E41FA3BC2
:10EEC000A5F88C31079BB24A1B680592B14C5F07CD
:10EED00000F18D840DF1500ADFF8E0820A940022DF
:10EEE000CAF804204546149240F6330B192740F225
:10EEF0008336049C02E004354D4522D0A978EB7896
:10EF0000994217FB0160F6D295F801E00EF1040E6C
:10EF100017FB036134F91E305B45A8BF5B46B3F5B0
:10EF2000617FB8BF4FF461739842E4DA9942E2DB43
:10EF300029782729DFD8504604350BF087FB4D454B
:10EF4000DCD1954A0A9C1378944A9AE8030082E837
:10EF50000300002B40F01781914B1F78002F00F029
:10EF6000BF8301218D480BF081FB002840F04A81CE
:10EF7000099BDB78002B40F0458123881DB225F0EA
:10EF80000105AEB2B342268000F0D785854D022739
:10EF90000E204FF014094FF0FF082F7085F80190F4
:10EFA00085F802802DF0E2FD39467C4826880BF07A
:10EFB0005DFB002841F0A48026F002039BB2B3421F
:10EFC00023800AD0774B1421FF2202250E201D70CA
:10EFD00059709A702DF0CAFD2688DFF8E4B1DFF889
:10EFE000E4A19BF80010DAF80400B50708BF81F02F
:10EFF0000201C1F3400109F0E5FF242167480BF04D
:10F0000035FB30B9089A1378590744BF23F004033D
:10F010001370059B1B6813F00A0F1DD005215F4874
:10F020000BF024FB002800F0938625886F0741F140
:10F0300033805A4806210BF019FB002800F0758632
:10F040006E0641F12180072154480BF00FFB002888
:10F0500040F0CE85059B1B689D0600F11283268833
:10F060004E480C210BF002FB002800F0E68046F42D
:10F070008073B342238009D04A4B02251421FF221A
:10F080000E201D7059709A702DF070FD464B1B7844
:10F09000082B00F0DE800E2B00F0DB80079B1B6846
:10F0A0005D0548D5414B1B79002B00F08F80142162
:10F0B0003A480BF0DBFA002840F08D802CF0C0FDC0
:10F0C00001202DF095FC002835D0DFF8FC800025CC
:10F0D0004FF0CC0902E0DDB2022D2CD809FB05F778
:10F0E0006B1C58F80760002EF5D1032290F902300E
:10F0F00002960192C2782E4951F8222000921846B9
:10F100003246334601212DF0A7F8034605EB4500B2
:10F1100000EB0010069353B1314608EB8000CC227F
:10F1200035F0B3FA069B48F807300135EDB21FF011
:10F130008DF90028D0D1089B1B78D80740F19C801E
:10F140009BF800101B4A1C4DDAF80000012301F067
:10F15000010113702B7009F035FF059B1B685A07DE
:10F1600000F1FE8017B0BDEC028BBDE8F08F98F87F
:10F17000022098F803309A42C0F0A08608F10408F3
:10F1800045453FF4E9AE98F800102329F6D1EEE7A3
:10F19000F49500205096002080640020343B00202D
:10F1A0001C360020C83A0020404000209078002003
:10F1B000086D0408003000201D77002080320020F8
:10F1C000FCC7002000C8002008BA0020089B1B785C
:10F1D000D9077FF573AF4FF40F7030F0DDFE0028D4
:10F1E000A9D021F01FFF4FF40F7030F077FE0028F8
:10F1F000A1D021F017FF4FF40F7030F06FFE002800
:10F20000EFD198E7059B1B689A077FF5B6AE268875
:10F21000F3073FF5D1AE46F001039E4223803FF451
:10F22000CBAEB74B1421FF2202250E201D70597062
:10F230009A702DF09BFC2688BEE626F480739BB264
:10F24000B34223807FF418AFAE4B1B78082B7FF4BA
:10F2500022AF228822F040039BB29A4223803FF4DF
:10F260001DAFA74B02251421FF220E201D705970DF
:10F270009A702DF07BFC11E7A34B1E78002E65D110
:10F28000A24B1B68002B61D0DFF8CC82DFF8CC9258
:10F2900018F8030C99F804704146A8F103052FF003
:10F2A000B9FE002800F0A985002F40F0FA8505F18D
:10F2B000080168792FF0AEFE002841F04E84944991
:10F2C000A87A2FF0A7FE002800F0AA85022F41F0AF
:10F2D00040849049E87B2FF09DFE002841F0358462
:10F2E0008D49287D2FF096FE002800F0AA85042F76
:10F2F00041F04A848949687E2FF08CFE002841F055
:10F300003F848749A87F2FF085FE002800F0AA855A
:10F31000062F41F03184834995F823002FF07AFEBF
:10F32000002841F02584804995F828002FF072FECE
:10F33000002800F0AA85082F41F003847B4995F846
:10F340002D002FF067FE002840F0AA85784B01229F
:10F350001A7030F0E9F8059B1B685A077FF502AF79
:10F3600003202FF08FFE002800F06787238813F01A
:10F3700008047FF4F7AE08200CF022FC049E6D48D0
:10F380006D4D6E496E4A6F4BF68800682E8008609E
:10F3900014601C6017B0BDEC028BBDE8F08F13B990
:10F3A000099A01239370684B099A1D7892F82140BD
:10F3B00008931B202FF066FE012C05F00108814602
:10F3C00000F0E88605F00205099A604E92F82030B8
:10F3D000DFF88CA15E4F05959346052B00F232872E
:10F3E000DFE813F0C00084000600FE000001F30017
:10F3F000012C04BF05238BF82030B8F1000F12D088
:10F40000069B3088B3F918100022134661F30F02EF
:10F4100060F31F4261F30F03049861F31F4303601D
:10F420000323426005934B4DDBF814102A68914288
:10F4300080F00D8647F230510322CBF81C108BF878
:10F44000202002200CF0D4FB10F046F92968DBF8EC
:10F450001C200A440421CBF818208BF82010012C22
:10F4600040F066872A68DBF81810914280F0EA863F
:10F470009AF8000020B92FF005FE002840F0E2863F
:10F480003A6822F002023A602A687388642101FB1C
:10F4900003234FF480600022CBF810308BF820203B
:10F4A0008BF803200CF074FB9BF8203095E72FF0CD
:10F4B000EFFD012807D1274D72882B68642101FBDD
:10F4C0000233CBF81030B9F1000F02D0B379002B22
:10F4D0007DD1012C00F0B6861E4DDBF810102A6895
:10F4E0009142C0F01A8701238BF82030012C6CD098
:10F4F000F379012B78D02FF04BFD9BF820306CE78F
:10F50000C83A0020404000201D77002020770020CE
:10F51000A03A0020A53A0020AA3A0020AF3A0020E5
:10F52000B43A0020B93A0020BE3A0020C33A002085
:10F5300000300020F8950020E02F0020EC2F002064
:10F54000E42F0020DC2F00201C770020849E002068
:10F550004C96002034C80020963A00207C00002001
:10F56000A4220020B8F1000FA1D1059D4FF48060C6
:10F57000B9F1000F00F0FF820CF022FB099A002382
:10F580001361002D3FF460AB28462DF0EFFA079B86
:10F590001E6816F480573FF45DAB1D21A6480BF0A2
:10F5A00065F800287FF456ABA44B03F1500903E043
:10F5B0000433994500F04C861A78262AF8D19978B8
:10F5C000DA789142F4D2FFF747BB9D4D5CE72FF00C
:10F5D000DFFC03224FF47A738BF82020CBF81C3029
:10F5E000974D2EE7964D3AE72FF0D2FC032240F6D6
:10F5F000B8338BF82020CBF81C30914D21E7914F88
:10F600003B78002B01F0AA818F4BDFF87082DFF886
:10F6100070B2DFF870A2069345465E4604909946A4
:10F620000EE019F804109847032C28DC88B93B78C1
:10F630002AF8020F01349C4205F1040580F22A8168
:10F64000072CE1B23046DBF80430EADD984700B21F
:10F65000EDE738F824206B88801A4FF47A719B1AF2
:10F6600001FB00F040F6CA0290FBF3F00844904220
:10F6700040F2EE23A8BF10469842B8BF184600B229
:10F68000D5E7724B1B78980704D5714D2B7D042B61
:10F6900000F25B86268816F0300F3FF4E1AC1020B4
:10F6A0000CF076FA20200CF073FA6A4B26880022C0
:10F6B0001A70694A69486A4F6A4D002111606A4AA6
:10F6C0003960002329604160816103608360436188
:10F6D000C36113605160936053619161D361BFE472
:10F6E000DFF8A4A1DFF8A481604D0AF15A064FF0BB
:10F6F000010951461AF8010C2FF08CFCF8B19AF868
:10F7000004009AF802309AF803E000EB400105EBA0
:10F710008101013BD1F89C2103EB43034344934215
:10F720000DD095F8C82181F898E109FA00F022EA95
:10F730000000C1F89C31C1F8A07185F8C8010AF138
:10F74000060A5645D5D14A493D4A4A4B09681B78B5
:10F75000D2F80080DFF838910B910A934FF0FF3B0D
:10F760004FF0000AD9F80430002B37D01E78002E55
:10F7700034D0D9F80820A8EB0202002A11DB3B4D57
:10F78000012195F8C82101FA0AF122EA010285F85F
:10F79000C821394A08F5FA704FF0FF31C9F808005E
:10F7A00011600A9AD2B199F8002059780432D2B285
:10F7B000002940F0FD8206990498098B30F9122047
:10F7C00001F1C800824240F37985284D9A7895F876
:10F7D000C83143FA0AF3D80740F1F7850AF1010A64
:10F7E000BAF1040F09F10C09BCD1FFF7BABB1F4DE8
:10F7F00095F892315BB1089B1B78DE0707D5049B17
:10F80000B3F90620069B5B8B9A4200F3CD8511214C
:10F8100009480AF02BFF002800F0B28295F89631D3
:10F820002BB995F8903113B93223A5F894310123FF
:10F8300085F89631FFF74EBB343B00208032002024
:10F8400034C8002044330020189100205296002034
:10F85000409F00206C4300205844002008440020B2
:10F86000682F00205C30002030440020F42B002062
:10F870005896002024410020040100206433002019
:10F88000A0930020EE2C0020AD390020DC470408B6
:10F890008C2D0020DDF81090B84AB9490792126803
:10F8A000A1FB091B42F2010111404FEA9B1B0F9182
:10F8B00000F06382B34DB448B44CB5492E7800785B
:10F8C000267008701EB1B2490E7886F00106B14D5F
:10F8D0000F2185F82011002B00F0E683AE4B069C2B
:10F8E0000E93B4F824E0B4F826C0069CCDF82CC0E2
:10F8F0001846248B0078A94B1294A94C0D900494BF
:10F900000446A3FB00035B0803EB4303E31ADBB2EB
:10F9100095F82181099302F4805205F592700BF558
:10F920009673119597F800A0DFF8BCC29C4C0C911F
:10F930007546DDF83CE01392002108930596CDF85A
:10F940004090059B002B00F02583964B33F9113036
:10F950001FFA83F9A9454FEA410203D30B9EB14533
:10F9600040F25C835CF821309B4580F01C83A35EF1
:10F97000BEF1000F40F0318301315145A35200F137
:10F980000600DEDB0C9A119D874B85F820210F2A9B
:10F990000CBF01220022DDF8409085F821811A7009
:10F9A00000F08983814B7849794ADFF840B20993A6
:10F9B0001C46042001230B7013700CF019F9DBF8BE
:10F9C0000030A1686268E3605B1A934284BF002341
:10F9D00084F82130079B3C781E68002C00F0DA8701
:10F9E000069A734DB2F824E0178B6D4916F48056D1
:10F9F000284640F0968332460EE0437803EB8303BB
:10FA000003EB830303F2EE239BB20132A24221F8FF
:10FA1000023B00F102000ED015F81230002B00F06E
:10FA20000183022BE9D001320B8821F8023BA2426C
:10FA300000F10200F0D10E9A137801331370FFF732
:10FA4000EAB8544DD5F88431A9EB0303002BFFF637
:10FA5000F0A8584A584B527C069933F812308A7DE8
:10FA6000DFED566A9FED566AC97D9BB207EE102AFC
:10FA700007EE903AB8EEC77AF8EEE77A27EE267AE4
:10FA800067EE867A0A9AC5F88421C7EE876A40F243
:10FA9000FF32FCEEE67ACDED057ABDF814309342E4
:10FAA00028BF134609B1D31A9BB24648464D017888
:10FAB000464C35F81160226825F81130921B13442A
:10FAC0000131434D236001F00F021B0902702B80AE
:10FAD000FFF7AFB8FBF7F8F93E4B3F4A1B68C31A74
:10FAE00093427FF7A6A83A4B00221A80FFF7A1B8ED
:10FAF000069A0499537DD27D013B31F913301AB136
:10FB0000C3F53B6308331BB2A3F57A7307EE903A53
:10FB10009FED327A2E4AF8EEE77A40F2FF3167EE37
:10FB2000877AFCEEE77ACDED057ABDF814308B428A
:10FB300028BF0B461380FFF77CB8022128480AF043
:10FB400095FD00283FF438AA2580B7073FF545AA60
:10FB500046F00203B34223803FF43FAA214B022028
:10FB60001421FF2218700E2059709A702CF0FEFF9D
:10FB70002688FFF732BA0CF00BF8FFE45C62002035
:10FB8000D34D62107C930020D41D0020244100201E
:10FB9000D51D0020F42B002037320020ABAAAAAAE2
:10FBA00008470020F02C00203C3B00203041002082
:10FBB00098330020D4C70020F4C700200000C842BA
:10FBC00000008044179400201C940020189400200A
:10FBD00038470020102E002060E316006F12833F8C
:10FBE000343B0020C83A00203832002034C80020BE
:10FBF000CB4AB2F90030002BB8BF5B42B3F5E17FCE
:10FC0000BFF628AAB2F90230002BB8BF5B42B3F5A9
:10FC1000E17FBFF61FAAC34B93ED057AD3ED077AB8
:10FC2000D3ED096A93ED030A77EEA67A30EE070A60
:10FC3000F7EE000AB0EE007AE7EEC70A30EE000AEF
:10FC40000AF060FAB6EE008A20EE488A9FEDB60A06
:10FC500038EE000AFDEEC07A17EE903A2033402BC2
:10FC600040F2B0839FEDB10AB14ADFEDB07A82ED88
:10FC7000000ABDEEC87AC2ED017A17EE103A2033C1
:10FC8000402BC2ED027A49D8DFEDAA7AB4EEE78ABA
:10FC9000F1EE10FA40F38087DFEDA76A9FEDA77AB7
:10FCA00001E0B0EE678AB4EEC78AF1EE10FA78EEA2
:10FCB000667AF6DC9FEDA27AF4EEC77AF1EE10FADE
:10FCC00040F166879FED9C6ADFED9E6A01E0F0EEF1
:10FCD000477AF4EEE67AF1EE10FA37EE867AF6D449
:10FCE000DFED917AB4EEE77AF1EE10FA40F329866F
:10FCF000DFED907A37EEC77A27EE076ADFED925A8A
:10FD0000DFED926ADFED927AE6EE256A67EE065A3B
:10FD1000E6EE267AA5EEA77AF0EE477A0A20C2ED43
:10FD2000037A2CF023FFFFF795B925F040039BB22F
:10FD3000AB4223803FF487A9864B02251421FF2282
:10FD40000E201D7059709A702CF010FFFFF77BB9D0
:10FD5000238823F00405ADB2AB4225803FF469A9A6
:10FD60007C4B02251421FF220E201D7059709A70C1
:10FD70002CF0FCFE2588FFF75CB977490E78A1E5E9
:10FD800095F89031002B3FF4A5A8089B1B7813F041
:10FD900001037FF49FA8012285F8903185F8912115
:10FDA000FFF798B86D4D012185F88811FEF7CDBF9A
:10FDB000012900F02B85BBF1FF3F684D0BD01B786C
:10FDC0000C2B08D0664B674A03EB8606664BC3F8DC
:10FDD00000B0736C136095F8C821012303FA0AF38D
:10FDE0000AF1010A1343BAF1040F85F8C83109F189
:10FDF0000C097FF4B7ACFFF7B4B808F105016879D6
:10FE00002FF008F900283FF45AAA012F40F0A586E8
:10FE100005F10D01A87A2FF0FDF8002840F0998631
:10FE20005249E87B2FF0F6F800283FF459AA032F37
:10FE300040F08B864E49287D2FF0ECF8002840F0EA
:10FE4000A3864C49687E2FF0E5F800283FF459AAB4
:10FE5000052F40F095864849A87F2FF0DBF8002851
:10FE600040F08A86454995F823002FF0D3F8002802
:10FE70003FF459AA072F40F07B86414995F82800A6
:10FE80002FF0C8F8002840F05C863E4995F82D0018
:10FE90002FF0C0F800283FF459AA092F3FF456AAC2
:10FEA0000926334603EB83031D44374B6978AA7850
:10FEB00089F8046019705A70FFF748BA33480AF09D
:10FEC000D5FB00283FF448A814202CF04FFEFFF784
:10FED00043B85D2A00F07E825B2A00F048855E2AE6
:10FEE00000F0A085562A00F01286972A00F01E86A0
:10FEF000A72A00F08B85264C23889B0740F04E856F
:10FF0000A2F1B703072B00F28F82DFE813F087021C
:10FF10008D028D028D0281028D027302730200BF79
:10FF2000009600206C220020DB0FC93F000000007B
:10FF300088000020DB0F4940DB0FC940E4CB1641AD
:10FF4000DB0F49C0E4CB16C192E741B99730083CBA
:10FF500015A82ABEC83A002024410020F42B002016
:10FF6000DC4704080454002004010020A53A0020C6
:10FF7000AA3A0020AF3A0020B43A0020B93A002053
:10FF8000BE3A0020C33A002024770020343B0020F2
:10FF900050960020002D3FD05CF821309B454FEA61
:10FFA0004102FFF4E4ACB34BB24E9B5C06EB02099A
:10FFB000002B00F09980022B47D199F8013003EB18
:10FFC000830303EB830303F2EE239BB2032933DDA8
:10FFD0001BB2BEF1000F3FF4CFAC099E20F81630E3
:10FFE000B8F1000F03D10D9E022E7FF6C5AC4388F9
:10FFF000B0F80090B0F804804B4498449E4B0FFA40
:020000040801F1
:1000000088F883FB08639D4EA3EBE87326F8028013
:100010001BB24FF00108AFE42B464A00089E4CF893
:100020002160A5E4D3B2022B04D9032B7FF4FBACEF
:100030007346EAE43B46E8E4012606FA01F90C9E21
:1000400026EA09061BB20C9692E4A35ABEE78C4A34
:100050001278002A7FF4EEA9B8F1000F3FF4EAA964
:10006000012C40F0EF809BF82030FFF7B6B9314605
:1000700084480AF0FBFA002800F0A38085F88F611D
:100080000FF05AFFFEF7B9BE45F04003AB422380A4
:100090007FF452AEFEF7D7BF45F004039D422380A4
:1000A0007FF45EAEFEF7C5BF774B784A0E92012211
:1000B0001A70774B04931B2172480AF0D7FA002874
:1000C0007FF470AC734BDFF8F0B109931946DBF89D
:1000D0000030CA688B609B1AC82B00F24C84079BC7
:1000E0001E6806F48056A6E4CBB2022B40F28B8346
:1000F000032BAAD1129B139E002E08BF2B4665E747
:1001000026F001039BB2B34223803FF41EAD0E20C4
:100110002F7085F8019085F802802CF027FD268845
:1001200013E500220FE0437803EB830303EB830323
:1001300003F2EE239BB20132A24221F8023B00F10E
:1001400002003FF478AC15F812301BB1022BEAD054
:100150000B88F0E7D3B2032BFAD83B46EBE7B2F5B6
:10016000FA7FFEF6AFAE95F88E31002B7EF4AAAE84
:10017000089B1B78012213EA020485F88E213EF4C5
:1001800097AE0FF0A9FA444B0593079B434C1B68AD
:10019000FEF79DBE0025FFF717B9B2F5FA7FFEF610
:1001A00091AE95F88E21002A7EF48CAE089B1B78C8
:1001B000012185F88E11D90700F1BA830FF0BCFE3A
:1001C000E1E7089B364A1B781060D8077EF519AE28
:1001D000344B1B78002B3EF475AE099BDB78002B6B
:1001E0007EF470AE95F88F310133DBB2032B85F8C6
:1001F0008F317EF667AE2C4B5B7813B9002C7EF402
:1002000061AE0FF069FAFEF7F8BD284A2849106878
:10021000B5F98C21C66981FB06018911F617701AA0
:1002200000F5FF407F3082423EF7DAAD891B0A4479
:1002300012B2A5F88C21FEF7D3BD08200BF0A8FC64
:10024000FEF790BF059D002D3EF4FEACFFF79CB974
:10025000184A069BD488049A1B8BB2F906101A1B05
:10026000914240F39E8023449942B4BF002401246C
:10027000FEF7FBBC9833002056555555602D0020E5
:10028000842F0020343B00203C3B002037320020EC
:100290000847002030410020F495002050960020AF
:1002A000D030002024410020BC9D00203898002040
:1002B000D34D6210A089002034C80020C8398A427A
:1002C000BD4D5FDA9A7895F8C83143FA0AF3D90739
:1002D0003FF584AA524201200C922CF06DFD731E52
:1002E0000C9A162B00F28A83DFE813F0B101980113
:1002F0007E01DE01CA010B02210156023C026D02A1
:100300004C018803DE018B020B02210156023802E8
:100310008702DA000C01F300C2002EF039FE03213F
:1003200040F6B8328BF82010CBF81C20FFF789B8C4
:10033000AB460999DBF80020CB69059D13448B611E
:10034000002D3EF481ACFFF71FB90A202EF09AFE73
:1003500026880746002800F0BC82F10640F1C683DB
:10036000954D95F8D071002F7EF47AAE0D202CF0CB
:10037000FDFB012385F8D0312688002F7FF499A951
:10038000FEF76EBE95F8C831012202FA0AF223EA9E
:10039000020308F5FA7285F8C831C9F80820FFF79A
:1003A0001DBA0124FEF761BC002184480AF05EF901
:1003B00000287FF42CAA322385F89201A5F8943105
:1003C000FFF725BA09F014FE4EE4002A0CBF012005
:1003D000022081E77A4B002201207A497A4C0B6097
:1003E0007A4B227005932CF0E7FC079B784C1B6836
:1003F000FEF76DBD774A7849734B116002225A703F
:10040000724B05932EF0A0FE079B1B68FEF75FBDA5
:10041000704A724911606C4B0022F0E76D4A7049D6
:100420001160694B0122EAE79E2A00F03D849D2A73
:1004300000F00784AE2A00F0FC83AD2A00F0F283BE
:10044000EF2A00F0EC83FD2A00F0D783FB2A00F0AE
:100450004184FE2A00F03B84F72A00F035847B2A91
:1004600000F0B783079B594A1B680592FEF72FBD22
:10047000D5F8CC015B4F90F836B0BB789344BBF114
:10048000640FA8BF4FF0640B2BEAEB7B80F836B00B
:10049000002B40F0118426F0A7F9D9F804308EE43F
:1004A000D5F8CC014F4F90F802B09344BBF1C80F80
:1004B000A8BF4FF0C80B2BEAEB7B80F802B0BB78EB
:1004C000002BE8D0142059462EF024FED5F8CC019C
:1004D000E1E7D5F8CC01434F90F837B0BB789344AF
:1004E000BBF1FE0FA8BF4FF0FE0B2BEAEB7B80F8B1
:1004F00037B0002BCFD0162059462EF00BFED5F882
:10050000CC01C8E70B99374F91F801B09344BBF584
:10051000967FA8BF4FF4967B2BEAEB7B81F801B066
:10052000BB78002B40F0F983D5F8CC01B3E7D5F8C0
:10053000CC012C4F90F804B0B9789344BBF1C80FAC
:10054000A8BF4FF0C80B2BEAEB7B80F804B0002962
:1005500040F0F283102E9ED090F801B09344BBF18E
:10056000C80FA8BF4FF0C80B2BEAEB7B80F801B097
:10057000BB78002B8FD0132059462EF0CBFDD5F839
:10058000CC0188E7D5F8CC01164F90F808B0BB78BD
:100590009344BBF1C80FA8BF4FF0C80B2BEAEB7B0D
:1005A00080F808B0002B3FF476AF0B2059462EF0B0
:1005B000B1FDD5F8CC016EE7F42B0020343B0020D0
:1005C0003A5600205496002078590020F4950020D7
:1005D00050960020589600205E5700204657002075
:1005E00052570020145400200B99CA4F91F804B0C0
:1005F0009344BBF1640FA8BF4FF0640B2BEAEB7B75
:1006000081F804B02EF0A0FDBB78002B8CD0032025
:1006100059462EF07FFDD5F8CC013CE70B99BD4F34
:1006200091F802B09344BBF1640FA8BF4FF0640B84
:100630002BEAEB7B81F802B0BB78002B3FF474AF60
:10064000022059462EF066FDD5F8CC0123E70B9920
:10065000B04F91F800B09344BBF1FA0FA8BF4FF030
:10066000FA0B2BEAEB7B81F800B0BB78002B3FF450
:100670005BAF012059462EF04DFDD5F8CC010AE7BD
:100680000B99A44F91F807B0BB7893448BF3080BF8
:1006900081F807B0002B3FF447AF052059462EF0F4
:1006A00039FDD5F8CC01F6E60B989A4F90F806B0D4
:1006B000B9789344BBF1640FA8BF4FF0640B2BEAE9
:1006C000EB7B80F806B0002940F02F830D2E3FF41D
:1006D0002BAF0B99BB7891F805B09344BBF1640F35
:1006E000A8BF4FF0640B2BEAEB7B81F805B0002B21
:1006F0003FF41AAF0E2059462EF00CFDD5F8CC0170
:10070000C9E6D5F8CC01834F90F803B0B97893448B
:10071000BBF1C80FA8BF4FF0C80B2BEAEB7B80F8EA
:1007200003B0002940F0E8820F2E3FF4B4AE90F8F9
:1007300000B09344BBF1C80FA8BF4FF0C80B2BEA21
:10074000EB7B80F800B0BB78002B3FF4A4AE122006
:1007500059462EF0DFFCD5F8CC019CE6D5F8CC014B
:100760006C4FE4E7D5F8CC016A4F90F806B0BB783F
:100770009344BBF1C80FA8BF4FF0C80B2BEAEB7B2B
:1007800080F806B0002B3FF486AE092059462EF0C3
:10079000C1FCD5F8CC017EE6D5F8CC015D4F90F8D0
:1007A00005B0B9789344BBF1C80FA8BF4FF0C80B90
:1007B0002BEAEB7B80F805B0002940F0C682112EB1
:1007C0007FF471AE67E6D5F8CC01524F90F807B0D0
:1007D000BB789344BBF1C80FA8BF4FF0C80B2BEAFE
:1007E000EB7B80F807B0002B3FF455AE0A2059464A
:1007F0002EF090FCD5F8CC014DE6D5F8CC01454F54
:10080000AAE6444F65E7129BFFF7E0BB049993F813
:1008100002B031F91220B2F5617F4FF4966191FB7D
:10082000FBF16DDB40F6330B9345A8BF93460C2ECE
:10083000ABF5617B9BFBF1FB5FFA8BFB00F0058165
:10084000182E40F091805A46C82AA8BFC822324DBF
:10085000D5F8CC1191F817E0D0B270453FF4AFAAAB
:10086000B2EB0E022B4FC87548BF0732D210B978D1
:10087000531CDBB239B913B118462CF09DFAD9F8E4
:100880000430FFF79CBA594618200C932EF042FC16
:100890000C9BF0E7214B22491A684FF47A73B3FBA3
:1008A000F2F3C3EB431203EB8202079B1B68D200F7
:1008B0001F06A1F8A82000F1B9801A4A0592126813
:1008C00055077EF503AB184A184C0A211180FEF734
:1008D000FEBAF20600F102810B202EF0D3FB0028B5
:1008E00040F0C680B30600F13C810B4D95F8D03145
:1008F000002B3FF43BAD002F7EF4DBAEFEF7B0BB28
:100900000C2E00F00181182E2CD14FF0000B5A460E
:100910009DE700BF14540020F42B00204C620020FF
:10092000705A0020F4950020A69E002050960020CA
:10093000C849079B0A60C84A1B680592C74CFEF766
:10094000C6BADFEDC77AB4EEE77AF1EE10FA44BF2B
:10095000DFEDC47A37EEC77AFFF7CEB9C24A069206
:10096000FEF79ABF4FF0000BC04DFFF728BAC04BFF
:100970000122022031E5BF4A079B1E68136823F05D
:1009800004031360099A012306F4805682F821308B
:10099000FFF751B806F48056FFF74DB80023BB2A85
:1009A000149300F02781B72A00F02081BE2A00F0BE
:1009B0001B81BD2A7FF438AD4FF6FE71AE4AA648C2
:1009C000D68905909089334401449181D38129F0DF
:1009D000B9FF08F03BFE29F09DFFF9F79DFA0120D1
:1009E0002CF0EAF9B5F88C21079BFA3A00211B6834
:1009F000A5F88C2185F88E11FEF769BAD5F8CC01DF
:100A000025F0F2FE4FF0FF3BFFF7E5B99B49079B4E
:100A10000A7891481B68059042F004020A708F4CD6
:100A2000FEF755BA964B02220320D6E4934A127879
:100A300096077FF542AF934A127D042A7FF63DAFB9
:100A400019F016FC079B1B6837E75D468E4A527803
:100A5000AA4289D08D4F284610F042F9BB781BB1CD
:100A600059460C202EF056FB6B1CDBB27F4D02E783
:100A7000874A884B528993ED007A07EE902AF8EE68
:100A8000E77AB0EEC77AB4EEE77AF1EE10FA7FF5C6
:100A900029AF93ED017AB0EEC77AF4EEC77AF1EEA2
:100AA00010FA7FF71FAFB3063FF51FAF20200BF002
:100AB00087F895E80C0078490A60084641F8043F39
:100AC00012F0DAFF754B01221A70684D95F8D0319B
:100AD000002B00F002812688FEF7EBBD10200BF002
:100AE00057F86E4B26881F700127F5E610200BF093
:100AF00067F820200BF04CF86949081F12F0BCFF82
:100B0000664B02221A70E0E70025AB469EE729F00B
:100B100019FF08F09BFD29F0FDFEF9F7FDF9012012
:100B20002CF04AF995F88A21FFF7DFB94A495D4A66
:100B3000079B05914FF4C8711B681180474CFEF765
:100B4000C6B908263346FFF7ADB903263346FFF78B
:100B5000A9B902263346FFF7A5B901263346FFF7A8
:100B6000A1B920200BF014F84C4B00221A70ACE70E
:100B700007263346FFF796B906263346FFF792B9A4
:100B800005263346FFF78EB904263346FFF78AB9A8
:100B9000B0EE677AFFF7A4B8F0EE487AFFF78AB8AC
:100BA000002C3EF4A6A8314D95F88931002B3EF477
:100BB000D1A82BF0BFFF002385F88931FEF7CAB812
:100BC000254B85F8901185F891010593234CFEF78C
:100BD0000FBE4FF4FA6102200FF0ACFF1E4B0593DD
:100BE000079B1B68FEF773B90221E7E619464FF62B
:100BF000FE73E3E619460223E0E6002101200FF030
:100C000099FFB5F88C21079B13491B680591963A0B
:100C1000A5F88C21002285F88E21FEF758B9002115
:100C20000846ECE7FF21002022F00BF895F88A2116
:100C300006E40121002022F004F895F88A21FFF74C
:100C4000FCBB0021FF2021F0FCFF95F88A21FFF773
:100C5000F1BB00BFD0300020F4950020509600205A
:100C6000DB0FC9BFDB0F49C018910020F42B002017
:100C7000885600204C9600209C9D00205296002013
:100C8000D6560020409F00207859002014540020A0
:100C9000FC430020A0780020F42D00206C430020AD
:100CA00064430020A89E00200021012021F0C9FFFC
:100CB00095F88A21FFF7BBBB594617202EF02AFA78
:100CC00032E40B20FEF7C4B80021042097E700218E
:100CD000032094E70021022091E70127FFF746BB9C
:100CE000002B3FF460AF1D491D4A09684FF47A702C
:100CF00000FB0313136056E70F2059460C922EF0A9
:100D000009FAD5F8CC010C9A0EE5164D0EF0E4FC6C
:100D1000002385F88931FEF71DB8152059462EF0BD
:100D2000F9F9D5F8CC01FFF7B6BB59460D200C9266
:100D30002EF0F0F90C9AC9E4102059460C922EF0CE
:100D4000E9F9D5F8CC010C9A04E4112059460C922B
:100D50002EF0E0F9D5F8CC010C9A30E534C800202B
:100D6000CC300020F42B00202DE9F047C74C6368FD
:100D700020469847002800F0C380C54B1B7801220D
:100D8000042B84F83C2000F0BD80B4F91610B4F9AF
:100D90001820B4F91A3021636263A363BD4B1B882A
:100DA000002B69D0BC4DD4ED0C7AD5ED004A95ED01
:100DB000050A95ED015A95ED067AD5ED035A95EDA4
:100DC000026AF8EEE76AD5ED047AA4EEA60AA5EE6B
:100DD000267A67EEC07AA5EEC07AE6EE267A85ED31
:100DE000057AC5ED067A32F093FCD4ED0D6AD5EDA7
:100DF000094A95ED0E0A95ED0A5A95ED0F7AD5ED53
:100E00000D7AD5ED0C5A95ED0B6A2063F8EEE66A83
:100E1000A4EEA60AA5EE267A67EEC07AA5EEC07A01
:100E2000E6EE267A85ED0E7AC5ED0F7A32F070FC8B
:100E3000D4ED0E6AD5ED124A95ED170A95ED135AC9
:100E400095ED187AD5ED167AD5ED155A95ED146A0B
:100E50006063F8EEE66AA6EEA40AA6EE857A67EE6F
:100E6000C07AA0EE657AE6EE867A85ED177AC5ED52
:100E7000187A32F04DFCA063884FA17F884816F0A5
:100E800029FC3B88002B40F08480864ED6F8D45154
:100E9000854B1B685B0743D4B5F90070216B636B0E
:100EA000A06B824A824E92ED026AD2ED006AD2EDC8
:100EB000015AC91B2163B5F90270DB1B6363B5F9E5
:100EC00004703568C01B07EE900AB8EEE75A07EECB
:100ED000901AB8EEE77A07EE903AF8EEE77A36EE37
:100EE000056A36EE877A77EEA57A0135A06382ED42
:100EF000026A82ED007AC2ED017A3560BDE8F087C2
:100F0000BDE8F0876B4BB4F91600B4F91810B4F9CA
:100F10001A2018802063598061639A80A2633DE79C
:100F2000B6F89421322A00F08880002A66D196F81B
:100F30009131002BB0D06048D6F8F0215F4980FB9A
:100F40000273D217C2EB23122A80D6F8F42180FB59
:100F50000273D217C2EB23126A80D6F8F831A78A3F
:100F600080FB0302DB17C3EB2213DB1BAB800023E8
:100F7000CB6086F8913129F0E5FC08F067FB29F099
:100F8000C9FCF8F7C9FF01202BF016FFD6F8D451A1
:100F900082E7444E226BD6F8D451B3F5C87F4FF0A8
:100FA000000323632B80398818BFD6F8D801B7F81F
:100FB000008008BF0020B1F5C87F18BFD6F8DC312B
:100FC000616B02440B440020B8F5C87F6063C6F82B
:100FD000D821C6F8DC31688052D0D4F838E0D6F891
:100FE000E011A0637144B8F1010FA880C6F8E011C8
:100FF00068D008F1FF38A7F8008049E7D6F8F0017B
:10100000236B00210344C6F8F03121632980D6F810
:10101000F401636B61630344C6F8F4316980A36B28
:10102000D6F8F801A1630344012AC6F8F831A98073
:1010300075D0013AA6F8942179E72B8820491F48FA
:10104000276BA6F8E4310023B5F802E0B5F804C038
:10105000C0684B608B602363C6F8F0712B80616BB6
:10106000C6F8F41163636B80A16BC6F8F811A36333
:10107000A6F8E6E1A6F8E8C1C6F8EC01AB80D8E72F
:10108000A36BC6F8E031A063A880B2E70896002001
:10109000CD890020A8940020AC940020A89E0020B8
:1010A00038960020F42B00205C620020389E00203F
:1010B000349E0020D08900201F85EB519C9D00208C
:1010C000E42D0020DFF88CC0DFF884E0C8328CFB10
:1010D00002A9C833D217C2EBE9128CFB03A9DB17B4
:1010E000C3EBE913C8316B802A808CFB013CA28AD8
:1010F000CB17C3EBEC139B1AAB80CEF80C0029F096
:1011000021FC08F0A3FA29F005FCF8F705FF40469A
:101110002BF052FEB7F80080D6F8D45169E70B20C7
:1011200086F8961186F890212BF020FDD6F8D45140
:10113000074BB6F8E421B6F8E671B6F8E801D6F840
:10114000EC112A806F80A880B6F89421D96070E7EE
:101150009C9D00201F85EB512DE9F047B0F9085008
:101160000D81EDB2442D92B00C46174600F0C382BB
:10117000064642D9812D00F0008200F29580542D60
:1011800000F0C98040F2E6816E2D00F08282802D51
:1011900040F01D81BD4B93F8009009F1020919F050
:1011A000FF0900F09580BA4BBA4FBB4EDFF824A37D
:1011B000994403F101080A2516E0322D00F0CA8295
:1011C000A5F13C00C0B2132840F2CA820023226875
:1011D000511C216015702268C14502F10101216096
:1011E000137075D018F8015B0A2DE6D1BAF80030FB
:1011F000FF2BA8BFFF23DBB2E9E7052D00F06982D2
:101200001ED8022D7FD040F29281032D00F038824B
:10121000042D40F0DC802A46A049204608F0EAFC74
:101220000021204608F02EFD22680221531C0125D2
:10123000236028462B461170638112B0BDE8F08709
:10124000242D5ED040F20381282D00F0DE81382D60
:1012500040F0BD800A68924B0125511C2160157039
:101260002268052150192060117022680A21501946
:1012700020601170226800215019206011702268CE
:10128000197850192060117022685978501920601F
:10129000117022689978531923602B4611702846E3
:1012A000638112B0BDE8F087A02D18D040F2148100
:1012B000B82D00F0E381FE2D40F08980794D05F1D5
:1012C000080635F8021B204608F0DCFCAE42F8D1D7
:1012D00001252B462846638112B0BDE8F087724B8A
:1012E0000846196808F0B6FC704B2046196808F0EB
:1012F000B1FC6F4B19682046012508F0ABFC2B466A
:10130000E8E76C4BF6E704226B492046012508F01C
:1013100071FC2B46C3E70B68684A694F581C1121C2
:101320002060197023681278591C21601A70236894
:1013300097F85520591C21601A70236897F854209B
:10134000591C21601A70B7F85010204608F09AFC1A
:1013500023680022591C21601A7023682822591C16
:1013600021601A70B7F85210204608F08BFCBD1EA1
:1013700007F14E0635F8021F204608F083FCAE4206
:10138000F8D122684F4B0D21501C20605D18117060
:10139000226813F8011F501C9D4220601170F7D184
:1013A00023680222591C21601A70B7F85610204693
:1013B00008F068FCB7F85810204608F063FC0125D7
:1013C000B7F85A10204608F05DFC2B4667E7214627
:1013D000284609F02DFB00287FF47AAF742D00F029
:1013E000BF80772D0CD1336872689A421BBF5A1C9C
:1013F000326001461978344A20462BF097FD67E7A2
:10140000F52D01F05582762D00F07D81392D326861
:1014100000F0168200F2FC81212D01F02982292D95
:1014200040F03F82531C336013780A2B01F0CE82C8
:10143000502B40F04284304608F0CAFB234F3880DE
:10144000304608F0C5FB012578802B4627E7202D84
:10145000BDD10B681E4D591C6A7821601A70236833
:101460002A78591C21601A702368AA78591C2160B7
:101470001A702989204608F005FC23686A79591CEE
:1014800021601A702268A979D0E600BF7177002028
:101490008448040867666666606800207E590020FC
:1014A00025560020D0890020107AFF1F147AFF1FD4
:1014B000187AFF1F98570020E07B0408DC89002081
:1014C000E04400203D45002089C103084868002011
:1014D000E495002088680020822D7FF478AF0B68A7
:1014E000B74AB84D1178B84A581C20601970118954
:1014F000204608F0C7FBB54B22681B88FF2B02F182
:101500000101A8BFFF2321601370A96881F31001B6
:1015100089B2204608F0B6FB296801F30F0189B2B1
:10152000204608F0AFFBAA4B226819787EE6012D11
:101530007FF44DAF0B680022591C21601A7023689C
:101540005A1C22601D7022682521531C23602B46E3
:101550001170A4E6522D7FF43AAF2268002165E6AF
:10156000336872689A421BBF5A1C32600146197870
:10157000984A20462BF0DAFCAAE6974B1E780336F1
:1015800016F0FF063FF4A4AE944B954F1E4403F1B2
:1015900001094FF00A0820E0B8F1500F00F0D880A0
:1015A000B8F1320F00F0F180A8F13C00C0B213286E
:1015B00040F2EE800025294623685A1C226020460E
:1015C00083F8008008F05EFB2946204608F05AFBAD
:1015D000B1453FF47DAE19F8018BB8F10A0FDBD1AC
:1015E000804B9D68196805EB85054FF6FF736D000C
:1015F0009D42A8BF1D469942A8BF194625EAE57538
:1016000021EAE171ADB289B2D6E70B68DFF8FC815F
:10161000754E591C022221601A70236806275A1C35
:1016200022601F7023680A22591C21601A702368E7
:1016300001255A1922601D70B8F80010204608F0E4
:1016400021FBB8F80210204608F01CFB23685A1949
:1016500022601F7023685022591921601A70236874
:101660000022591921601A703188204608F00AFBBF
:101670007188204608F006FB2B4610E65B4B39E6E6
:101680000B685A1C0A601D700B685A1C0A601D709A
:1016900063E74E4B0A681B884A4DFF2BA8BFFF2308
:1016A000511C21601370A96881F3100189B2204692
:1016B00008F0E8FA4E4B2046198808F0E3FA29684A
:1016C00001F30F0189B22046012508F0DBFA2B4611
:1016D000E5E50B224749204608F08CFA08224649E6
:1016E000204608F087FA012507224449204608F0E1
:1016F00081FA2B46D3E5002A3FF4EAAD404B136054
:1017000001252B46CBE533685A1C32601B78002B31
:1017100001F05281102B01F05481054601462268E8
:10172000501C20601370204608F094FA2946204689
:1017300008F090FA334B2046196808F08BFA2046DF
:10174000002108F09FFA0021204608F09BFA04E7E8
:101750002D4B46E73388FF2BA8BFFF23DBB236E5CE
:1017600022F0CAF900283FF431AD03780A2B25D8BE
:10177000B0F9023087FB0312DB17C3EBA2039BB265
:10178000FF2BA8BFFF23DBB221E597E822002AE761
:1017900022F0B2F900283FF40DAF03780A2B3FF690
:1017A00009AFB0F90430B0F9061003EB830383F3FB
:1017B000500521EAE171ADB289B2FDE60023E2E70E
:1017C0009E780020CC950020E495002088780020A9
:1017D0004C45002031C2030871770020944804086A
:1017E000586800201468002048680020A0390020B4
:1017F00038470020E87B0408F47B0408007C0408D8
:1018000075A70108EC2F00204C6800208C9D00205B
:10181000552D25D0572D44D1531C336012F8370B6A
:101820000DF107010133336013F8015C01F8015F2A
:101830009342F7D102A90125F7F7B8FB2B462EE515
:10184000531C336013780A2B01F0C680304608F031
:10185000CBF9304608F0C8F9304608F0C5F937E54D
:10186000531C33601778FF2F01F02681FE2F01F003
:10187000EB80304608F0ACF996E80C009B1A002B80
:1018800006DD531C3360137813B90C2F41F24081ED
:10189000272F00F2E384F74B012523F817002B468E
:1018A000FDE471680B3D8B1AEF2D00F2D78401A087
:1018B00050F825F0DD2401085D2201085D220108B1
:1018C0005D2201085D2201085D2201085D220108F8
:1018D0005D2201085D2201085D2201085D220108E8
:1018E0005D2201085D2201085D2201085D220108D8
:1018F0005D2201085D2201085D2201085D220108C8
:101900005D2201085D2201085D2201085D220108B7
:101910005D220108832401085D2201086924010871
:101920005D220108472401085D2201085D220108AB
:101930005D2201086D2501085D22010813250108BB
:101940005D220108952501085D2201082124010876
:101950005D220108B72201085D2201086722010803
:101960005D220108152201085D2201085D2201089F
:101970005D2201085D220108D11201085D220108E3
:10198000E92101085D2201085D22010819230108EF
:101990005D220108791C01085D2201085D22010811
:1019A0005D2201085D2201085D2201085D22010817
:1019B0005D2201085D220108332301085D22010830
:1019C000FB1F01085D2201085D2201088721010833
:1019D0005D2201085D2201085D2201085D220108E7
:1019E0005D2201085D2201085D2201082321010812
:1019F0005D220108B32001085D220108452001088D
:101A00005D220108912301085D220108C12101081E
:101A100073230108DF1F01085D2201085D22010810
:101A20005D2201085D2201085D2201085D22010896
:101A30005D2201085D2201085D2201085D22010886
:101A40005D2201085D2201085D2201085D22010876
:101A50005D2201085D2201085D2201085D22010866
:101A60005D2201085D2201085D2201085D22010856
:101A70005D2201085D2201085D2201085D22010846
:101A80005D2201085D2201085D2201085D22010836
:101A90005D2201085D2201085D2201085D22010826
:101AA0005D2201085D2201085D2201085D22010816
:101AB0005D2201085D2201085D2201085D22010806
:101AC0005D2201085D2201085D2201085D220108F6
:101AD0005D2201085D2201085D2201085D220108E6
:101AE0005D2201085D2201085D2201085D220108D6
:101AF0005D2201085D2201085D2201085D220108C6
:101B00005D2201085D2201085D2201085D220108B5
:101B10005D2201085D2201085D2201085D220108A5
:101B20005D2201085D2201085D2201085D22010895
:101B30005D2201085D2201085D2201085D22010885
:101B40005D2201085D2201085D2201085D22010875
:101B50005D2201085D2201085D2201085D22010865
:101B60005D2201083F1F01085D220108291F0108AD
:101B7000B51F01085D2201085D2201085D220108F0
:101B80005D2201085D2201085D2201085D22010835
:101B90005D2201085D2201085D2201085D22010825
:101BA0005D2201085D220108CF1E01087D1E01088B
:101BB000451E01085D220108A91D01088F1D0108AD
:101BC000731D01085D220108591D0108F31C01085D
:101BD000CB1C0108C11C0108132801085D22010863
:101BE000E52701085D2201085D220108C3270108DD
:101BF000952701088127010859270108392701087D
:101C000017270108EB2601085D2201085D22010863
:101C10005D2201085D2201085D2201085D220108A4
:101C20005D2201085D2201085D2201085D22010894
:101C30005D2201085D2201085D2201085D22010884
:101C40005D220108D12601085D2201085D220108FC
:101C5000772601085D2201085D2201085D22010846
:101C6000112601085D2201085D2201085D2201089C
:101C7000C7250108E0440020531C3360BA4B12789A
:101C8000BA4F1A7000233B60304607F089FF326874
:101C90003B68B749B74D0343501C3B603060137835
:101CA0000B72304607F094FF2860304607F090FF33
:101CB0006860304607F08CFFA860304607F088FF68
:101CC000304607F085FFFFF703BB531C33601078E5
:101CD000060600F1DA87A84B1B78DD073FF5F8AA66
:101CE000032828BF00200125F8F748F82B46FFF706
:101CF000D6BA531C3360304692F8009007F050FF7C
:101D00008046304607F04CFF0546304607F048FF56
:101D10000746304607F05CFF304607F059FF304673
:101D200007F062FFB9F1000F00F09A87B9F1100FC8
:101D30007FF4CEAA914BC3F804809D600FB1904B05
:101D40001F609049904B0222081F01251A7011F064
:101D500093FE2B46FFF7A3BA874B1B78D8073FF5B6
:101D6000B7AA0125F8F7B4FAF8F7D6F82B46FFF72B
:101D700096BA814B1B78DA073FF5AAAA834A1378F3
:101D8000012543F0040313702B46FFF788BA7A4B02
:101D90001B78D9073FF59CAA7D4B4FF4C8720125EB
:101DA0001A802B46FFF77BBA092B40F35782794FF5
:101DB0001346511C3D68316013F8021B29703360D3
:101DC0005378AB70D31C33609378642B02F1040119
:101DD000A8BF64236B713160D378642B02F10501D5
:101DE000A8BF6423AB7131601379EB71931D33602D
:101DF0005379642B02F10701A8BF64232B72316071
:101E00009379EB7002F108033360D3792B7130467C
:101E100007F0DEFE726833686881D11A00290BDD95
:101E2000591C38683160521A002A1978417203DD52
:101E30009A1C32605B78437001252DF085F92B46A2
:101E4000FFF72DBA544B1868D31C014621329D1E52
:101E5000356013F8035C0D705D1E356013F8025C8D
:101E60004D70336013F8015C8D7003339A4201F1B9
:101E70000301ECD124F0B8FCFFF72ABA531C3360FD
:101E800013784249002B00F00B870B7843F00203D4
:101E9000901C0B70414D306053782B75304607F025
:101EA0007FFE2860304607F07BFE6860304607F012
:101EB0008FFE2881304607F08BFE394AE88113787F
:101EC000012543F0020313702B46FFF7E8B9C3F373
:101ED0004705122D00F2C281B5B112AB0DF1060912
:101EE00003EB4507C846423F304607F071FE28F82D
:101EF000020FB845F8D12B4B39F8022F23F8022FE7
:101F0000C845F9D1112D09D8274A6B00023B13446B
:101F10000021223223F8021F9A42FBD1234A0123D7
:101F20001D461370FFF7BBB9214F002330463B60BD
:101F300007F036FE012538602B46FFF7B0B913468F
:101F4000511C316013F8025B3360D31C507833604E
:101F50009178002D00F0A986012D7FF4B9A90EF02B
:101F6000A3FE2B46FFF79BB9404000209857002066
:101F700018910020947600201C770020F02D00207E
:101F8000EC2F0020F82D00206C43002052960020FA
:101F9000A89E00205896002054960020409F0020C4
:101FA0006A43002002310020043100202831002043
:101FB000A0390020531CC4483360017813780029ED
:101FC00040F0B38504220270C04A9B001380F8F7EA
:101FD0007BFFBF4B012518622B46FFF760B9531CEE
:101FE00033601378002B00F0F8854FF40040012592
:101FF00009F0FEFD2B46FFF752B9531C33601778EA
:10200000112F00F22B81931C3360B24D537805F8E9
:102010001730304607F0DCFD40F6CA039842A8BFEF
:10202000184640F2EE23984205EB4701B8BF184628
:102030000125A0F2EE222B46192092FBF0F24A7005
:10204000FFF72DB9531C3360A34DA44F13787B7158
:102050003046D5F8008007F0BBFDA8F820003046D8
:10206000D5F8008007F0B4FD72683368A8F81E0048
:10207000D11A072900F37585D11A032900F3658564
:10208000D21A002A05DD591C2A6831601B7882F8B3
:102090002630F7F799FE1CF049FC914B1B68002B8A
:1020A00000F079852868012523F0CEFF2B46FFF745
:1020B000F6B81346511C3160884F13F8021BB970F3
:1020C0003360884953780B70D31C3360864D937806
:1020D0002B71131D3360D378092BA8BF0923304619
:1020E000AB7007F075FD336872682880D11A01293A
:1020F00005DD304607F06CFD33687268E8819A426E
:1021000040F05485F7F760FE336872689A423FF4F6
:10211000DFA85A1C32601B78EB7001252B46FFF7B5
:10212000BEB8724B1B68002B3FF4D2A811F09CFD87
:10213000FF283FF4CDA8304607F04AFD3F2840F283
:102140003E856B4F00253D7033687268B880D21AA7
:10215000012A7FF7BDA81A46591C316012F8021BEC
:10216000B97012A8326000225D7800F8402D11F09D
:102170004DFD9DF80830AB423FF4AAA8284611F067
:1021800069FDFFF7A5B85B4B1B78012B3FF6A0A8B4
:102190001046531C3360584F10F8023BBB70306040
:1021A000D31C50783360CB1A012B917840F31E85F5
:1021B000304607F00DFD012538802B46FFF76FB83C
:1021C0001346511C31604D4913F8020BC87033603F
:1021D0004B4953784B71D31C33604A4B9278DA7079
:1021E00001252B46FFF75BB81346501C306046486C
:1021F00013F8025B85703360557845708B423FF46D
:1022000067A8D31C3360324B92781A7401252B4691
:10221000FFF745B80721B3FBF1F1C1EBC1055B1B2B
:102220001CD1C9B201F1FF385FFA88F800293FF4E8
:102230004FA8DFF8D8A008F101081D46531C3360F1
:1022400092F90010314B002793F902208A4203F1E2
:10225000080300F00C840137062FF5D14FF0FF354D
:102260002B46FFF71CB8531C336013780E2BF5D8A0
:10227000911C31605578032DF0D82548062101FBCB
:1022800003F14318D71C5D71376095784554111DD3
:102290003160D1785970511D316011799970911D5B
:1022A00031605179D970D11D316092791A7101254F
:1022B0002B46FEF7F4BF531C3360164B12785A7549
:1022C00001252B46FEF7EBBF16940020384700206F
:1022D000F02D002098330020549600205C5A0020F6
:1022E0003C400020909D00205C640020207700206E
:1022F000247700207C570020145400209C9D00204F
:1023000018980020AC9D0020BC9D00204491002026
:10231000AC39002018910020B14B02F108010132C4
:10232000326012F8010C03F8010F9142F7D1FEF769
:10233000CFBF1346511CAB4D316013F8021B2971FE
:10234000336053786B71304607F042FC3368288065
:102350005A1C32601B78AB71304607F039FC336889
:1023600068805A1C32601B78EB7101252B46FEF702
:1023700096BF9D4B1B7813F001017FF46FAF531C88
:102380003360107801250EF0D5FB2B46FEF787BF92
:10239000304607F01DFC304607F01AFC304607F0C7
:1023A00017FC304607F020FC3368904D1946581C46
:1023B0002A68306011F8020B82F82C0031605978DD
:1023C00082F83610D91C31609B7882F8373030465D
:1023D00007F00AFC304607F007FC304607F004FC23
:1023E00030462F6807F0F4FB788730462F6807F0F7
:1023F000EFFB336872683887D11A01290ADD591C4E
:102400002A6831601B7882F82E30304607F0ECFBEA
:1024100033687268D31A032B00F38C83286829E58C
:10242000511C316015781F2D3FF618AF052B7FF436
:1024300015AF304607F0B4FB6D4B43F8250017F09D
:1024400087FEFEF745BF304607F0C2FB694F386094
:10245000304607F0BDFB7860304607F0B9FB012538
:10246000B8602B46FEF71BBF634F00233B6030462E
:1024700007F096FB3B68012503433B602B46FEF7C4
:102480000EBF531C33601578132D3FF6E7AE931C37
:102490003360507801922AF083FD00283FF4DEAECD
:1024A000019A564B017803F82510D11C316003EBDB
:1024B000850391785970111D3160D1789970511D43
:1024C00031601279DA7000202CF080FD4C4B80F0E6
:1024D0000100012518702B46FEF7E1BE494A102B7A
:1024E0004FF0000128BF1023116051609160D1604E
:1024F0001174002B3EF4ECAE3168013A0B4401310B
:10250000316011F8010C02F8010F9942F7D1FEF782
:10251000DFBE531C3C4D336013782B72304607F0FE
:1025200057FBA883304607F053FB2883304607F05B
:102530004FFB32686883531C33601278EA74726808
:10254000D31A032B00F36D833368D11A052900F3E6
:102550005883D21A002A7EF7BBAE5A1C32601B7811
:1025600085F8213001252B46FEF799BE531C3360B8
:10257000264815780570C91A00297EF7A9AE931C64
:1025800033605378003318BF0123012543702B4675
:10259000FEF785BE164D05F14007304607F018FBE3
:1025A0003368A5F88000591C1A46316012F8021BE6
:1025B00085F8821032605B7885F883300435BD423F
:1025C000EBD1FEF785BE084B1B78DB073FF546AE27
:1025D0000125F7F7EFFBF7F79FFC2B46FEF75FBEF1
:1025E00017910020849E00201C7700205496002024
:1025F0006C450020947600209857002080320020FF
:10260000A4220020EE53002018910020404000201A
:10261000304607F0DDFA3368ADF808001A46591C59
:10262000316012F8021B32608DF80A105A788DF86A
:102630000B20DA1C32609A788DF80C201A1D32605B
:10264000DA788DF80D205A1D32601B798DF80E3026
:1026500002A80023ADF8103007F012FAC24AC34BAB
:102660001268801A4FF0010561F10001C3E906010B
:102670002B46FEF714BE531C336013780F2B3FF626
:10268000EDAD911C3160C3EBC303B9495078C85418
:10269000D01C30600B4491785970111D3160D17895
:1026A0009970511D31601179D970911D3160517946
:1026B0001971D11D31609179597102F108013160B0
:1026C000D2799A71012523F029FC2B46FEF7E7BD4C
:1026D000304607F07DFAA74FF881304607F078FAC8
:1026E0000125B8812B46FEF7DABD1146531C336035
:1026F000A14B11F8020B1870316051785970D11C40
:10270000316091789970111D3160D278DA700125AD
:102710002B46FEF7C4BD304607F05AFA974F388271
:10272000304607F055FA7882304607F051FA012515
:10273000B8822B46FEF7B3BD1346511C316013F827
:10274000020B3360D31C51783360927819F0F0F8A3
:1027500000287EF4BDAD81E51346511C31608849E7
:1027600013F8020B08703360824953788B70D31CC6
:102770003360844B92789A7001252B46FEF78FBD0B
:10278000814B824918684E22012530F0EDFD2B4621
:10279000FEF785BD1146531C33607D4B11F8020BCB
:1027A0001870316051785970D11C316092789A70EC
:1027B000304607F00DFA774B0125D8802B46FEF7FF
:1027C0006EBD304607F004FA724F3880304607F08D
:1027D000FFF97880304607F0FBF90125B8802B46D9
:1027E000FEF75DBDDFF8C48198F80030002B3EF4A1
:1027F0006FAD694F0025304607F0EAF924F04AF939
:1028000098F80030A7EC010A01359D42F3DBFEF792
:102810005FBD0D2B7FF422AD531C33601578072D5F
:102820003FF61CADDFF8888130460C2707F0D0F961
:1028300007FB05F708EB0705A880304607F0C8F945
:10284000E880304607F0C4F9336828811A46591CDD
:10285000316012F8021BA97232605B78EB7230466D
:1028600007F09EF9012548F807002B46FEF717BD33
:102870001346511C3160494D13F8021B69703360D7
:1028800053782B70D31C33609378AB70304607F0CD
:102890009FF933682881591C1A46316012F8021BCF
:1028A000697132605B78AB7101252B46FEF7F7BC8E
:1028B000336872689A4240F0A0802C4BFF221A7055
:1028C0004FF00009364D0CF0CBFE4946202235482A
:1028D00085F8009031F0D9FE8DF808909DF8083009
:1028E000072B00F22081DFF8CC802E4E4A469DF85F
:1028F000083003EB430308EBC3035B7CE3B19DF8B3
:10290000083003EB430308EBC30320215B699BB151
:102910009DF8083003EB430308EBC303586946F8FE
:10292000220006F08BFA2B7856F8230006F044FBC1
:102930002A780132D2B22A709DF808300133DBB216
:102940008DF808309DF80830072BD0D92368591C22
:1029500021601A70002F3EF4BBAC134B3B60012585
:102960002B46FEF79CBC00BF34C80020F02D002091
:10297000B43800209C9D00205C4100205C64002055
:102980005C5A0020AC9D002054960020606A040828
:10299000949D0020A0890020C8360020E4950020E6
:1029A0004F33002004320020FD25020871770020FB
:1029B000F43700209C630020BF4A92E82200FEF713
:1029C000AEBEBE4A51689568FEF7A9BE304607F014
:1029D000FFF8BB4FFEF733BD931C3360B94B517802
:1029E0001970D11C316091785970111D3160D27805
:1029F0009A7001252B46FEF752BC5A1C19463260CC
:102A0000AE4811F8022B027031605B784370042AE3
:102A100003D9FF2A7EF4A1AD52E7AB490978994268
:102A200005D8022A7EF499ADFF2B7EF496AD23687B
:102A300001255A1922601D70002F3EF449ACA34BAA
:102A40003B602B46FEF72BBC931C33605578022D60
:102A50003FF604AC304607F0BBF89D4B03EB450353
:102A60004FF0FF35A3F856002B46FEF718BC0AEBD3
:102A7000C709304689F8021007F0AAF833682AF827
:102A800037001A46591C316012F8021B89F80310EE
:102A900032605A7889F80420DA1C32609A7889F812
:102AA00006201A1D32600135DB7889F80530A8450B
:102AB0007FF4C4ABFEF70CBC931C3360854B51789C
:102AC0001970D31C3360824F937887F85530131DEB
:102AD0003360D37887F85430304607F079F8A7F898
:102AE0005000304607F074F8304607F071F896E869
:102AF0000C009B1A012BA7F852007EF7E9AB304679
:102B000007F066F80125A7F85A002B46FEF7C7BB69
:102B10006F4B00301F4418BF0120012587F85E006D
:102B20002B46FEF7BCBB4A4610E704297EF4D0AB27
:102B3000FFF74ABA30462F6807F04AF878863046E1
:102B40002E6807F045F8B08668E4304607F040F894
:102B5000F881304607F03CF8336872683882FFF736
:102B60008FBA304607F034F87881304607F030F8F5
:102B7000B8813046D5F8008007F02AF8A8F822007E
:102B80003046D5F8008007F023F833687268A8F85B
:102B90002400FFF771BA50485049514A514B036025
:102BA00001250B6013602B46FEF779BB5A1C32607F
:102BB0001B78003318BF0123FB71FFF7A3BAC508C8
:102BC00000F0070301350133EDB2474F284619469F
:102BD0007B7020F0FBFEFFF7B6BA444A136801256C
:102BE00023F4004313602B46FEF759BB404B1A8871
:102BF000012512FB00F22B4692FBF1F23A80FEF720
:102C00004EBB5A1C32601B78EB72304606F0C8FF90
:102C10003368E8605A1C32601B782B743368726822
:102C200097E4304606F0D4FFA884304606F0D0FF83
:102C300033687268E884D11A03297FF786AC1A4694
:102C4000591C316012F8021BA97732605B7885F855
:102C50002030304606F0BCFF33687268688474E444
:102C6000154B1020C3F800805D6008F091FF214AE9
:102C7000137843F001031370002F3EF429AB1E4B71
:102C800001251F602B46FEF70ABB00F07F000328DA
:102C900028BF002001250EF023F82B46FEF7FFBACF
:102CA0000B7803F0FD03FFF7F3B8012523F020FCB8
:102CB0002B46FEF7F4BA00BF60430020F02D002041
:102CC0008C9D0020255600207177002081A70108E7
:102CD000E0440020DC890020448400209884002007
:102CE0009888002015860108247700204C96002043
:102CF0006C9D002052960020EC2F00202DE9F04F13
:102D00002DED0C8B364C95B06368049020469847A7
:102D1000002800F07D82B4F8A870002284F85120C9
:102D2000002F67D1B4F93860206AA16AB4F93A205B
:102D3000656AB4F93C30DFF8B4A0301A5B1A521B54
:102D4000E06294F85210636304F12C00226314F0E3
:102D5000C1FCDAF80030990042F10782D4ED0C5A38
:102D6000DFF88CB0D4ED0B7A1E4A9BED406ADBEDA8
:102D7000416A9BED427ADBF80C311268B8EEE58AC5
:102D8000D4ED0D5AF8EEE77AF8EEE58A013377EEE6
:102D9000867A38EE268A78EE878A9342CBED407A9F
:102DA0008BED418ACBED428ACBF80C3101F00C85DA
:102DB0000D4B029393F800E0BEF1140F03F00B8665
:102DC000DBF814210025062A01F27386DFE812F0F1
:102DD0002819151984175A18DA0DC218E61700BFFA
:102DE000705A0020C83B0020CD8900205C62002082
:102DF000202E0020D44BD549059391F801901B68F3
:102E0000D348DFF8A08302904FF47A71B1FBF3F35B
:102E1000C3EB431603EB8603DE00B6B2B742057878
:102E2000B8F9060003F0E182D4F87CE0B4F9382068
:102E3000236E0EF1010107EE902A13440129E16788
:102E40002366F8EEE77A03F0DA82D4ED1B5AD4ED6C
:102E50001D6A07EE101A37EEE56AB8EEC75A012F61
:102E600086EE057A37EE257A77EEC77A84ED1C7AFE
:102E7000E7EE866A84ED1B7AF0EE667AC4ED1E6A90
:102E8000C4ED1D6A03F0CF86D4F890E0B4F93A207F
:102E9000636E0EF1010107EE902A13440129C4F874
:102EA00090106366F8EEE77A03F0C182D4ED205A01
:102EB000D4ED226A07EE101A37EEE56AB8EEC75A6B
:102EC000012F86EE057A37EE257A77EEC77A84ED04
:102ED000217AE7EE866A84ED207AF0EE667AC4ED18
:102EE000236AC4ED226A03F0C686D4F8A4E0B4F9DC
:102EF0003C20A36E0EF1010107EE902A1344012934
:102F0000C4F8A410A366F8EEE77A03F0A982D4ED22
:102F1000255AD4ED276A07EE101A37EEE56AB8EEA7
:102F2000C75A012F86EE057A37EE257A77EEC77AF3
:102F300084ED267AE6EE276A84ED257AF0EE667A4D
:102F4000C4ED286AC4ED276A03F0BD86DFF858B2E5
:102F5000A8F80600B4F8A830029A013B1578A4F846
:102F6000A83005990023072D4B608B60CB6040F0A3
:102F70005781F7F7A9FF029BDFF828821D78049B91
:102F8000C01A9BF82131A8F800000693002B40F0EE
:102F90004D816E4B5B79002B01F00B836D4B1B78E1
:102FA000013BDBB2072D8BF8213102F06284002354
:102FB0000893694ADBF82C31D2ED006A674A9FED2D
:102FC000686AD2F800A0604A0592049ADBED4AAA2A
:102FD000DFF8D8819BED499A9FED62AADFED62BAD6
:102FE0009FED62CA9FED62BADFF8C491614FCBF8E2
:102FF0002C21D31A07EE903AF8EE677AB7EE007AF2
:10300000C6EE279A08F11C03002507935A4B039339
:103010002E4677EE6A8A68EEA68AF4EEC78AF1EE4B
:1030200010FA88BFF0EE478A544B98ED008A2B4483
:10303000D3ED007AF5EE407AF1EE10FA17D0504B4E
:103040002B4493ED007A78EE476AB0EEE66AF4EE30
:10305000C67AF1EE10FA08D5F5EEC06AF1EE10FA74
:10306000CCBF37EE878A37EE678A83ED008A454BFF
:103070001A8893073FD0022E3DD0434B9AF82E106A
:1030800033F9163007EE103A079B07EE901A2B44DF
:10309000F8EEE76AB8EEC77AD3ED007A4B42A6EEB7
:1030A000A77A700007EE903AF8EEE77AB4EEE77A86
:1030B000F1EE10FA0AD407EE901AF8EE677AF4EE01
:1030C000C77AF1EE10FA88BFF0EE477A2F4B3049FD
:1030D0000344085EB3F90C30C01A07EE100AB8EECC
:1030E000C77AD007E7EE4A7A41F1F981294B93ED8F
:1030F000008A27EE888A059B9BF864212B4493ED78
:1031000001DA78EE4DCA002A00F0E780224BDBF8A6
:10311000682104991B688A1A9A4240F3DE809AF863
:103120004830022B02F0F683022E04F06A871B4B14
:103130001B68990700F19280194B87ED00CA1B6844
:103140009342C0F2C48035E04C6200205C5A0020FB
:10315000CD890020909D0020EC880020549600200E
:1031600000247449CDCCCC3DAE47813F0000000027
:103170000000C8424C3B0020403B0020E08800207B
:103180005C2F002050960020682F00209C9D00207E
:1031900000960020C8880020F4880020F4950020C4
:1031A000F0880020D0890020202E0020502F002001
:1031B000583B0020F7EE007AF4EEE7AAF1EE10FAA1
:1031C00040F18B8005991F4BD1ED017A93ED007A88
:1031D000F0EEE77AF4EEC77AF1EE10FA7DD5D1ED94
:1031E000027AF0EEE77AB4EEE77AF1EE10FA74DDE7
:1031F000D1ED037AF0EEE77AB4EEE77AF1EE10FA69
:103200006BDD114B1B689A0761D51049104B45E0E7
:10321000104BDFF844B01D780293072D3FF4A9AEA0
:103220009BF821310693002B3FF4B3AE581E8BF868
:103230002101012D01F0B68415B0BDEC0C8BBDE869
:10324000F08F00BFFC880020F4950020009600203D
:103250009C9D0020CD890020202E0020D74BD849EE
:10326000DFF8CCE331F916C09EED008ADFF8C4E345
:1032700087ED00CA03EB460028EE0A8AB0F90C007D
:10328000A0EB0C0007EE900AF8EEE77ADEF80000FB
:1032900027EE888A904278EE4DCA8BDAB3F90C207B
:1032A000B1F900E0C748AEEB020E00688EEAEE729C
:1032B000A2EBEE72824210DAB3F90E30B1F90220BD
:1032C000D21A82EAE273A3EBE273984205DD00238F
:1032D00018468BF86431F7F755FFBB4B2B4493ED41
:1032E000000A039B29EE000A022E20EE2C0AA3EC12
:1032F000010A039304F04286B44BD7ED006A93EDC4
:10330000007AB34BD3ED007AB24B93ED006AB24B27
:1033100067EE277A2B4427EEA87AD3ED007A67EE82
:10332000277AF0EE665AECEEA75AB1EE467AB4EE82
:10333000E57AF1EE10FA08DCB4EEE56AF1EE10FA87
:103340008CBFB0EE657AB0EE467A9BED4A6AF7EE36
:10335000007AB4EEE76AF1EE10FAACBF0123002365
:1033600043B1F0EEE66AF0EEC77AF4EEE67AF1EEFB
:1033700010FA01D587ED007A022E04F0BF85974A36
:10338000974B52F826001B68B0EE4D0A9847954AB5
:10339000954B52F826001B6898479AF8373023B1AE
:1033A000924B1B88002B01F00781B0EE4C8A904BAA
:1033B00038EE400A2B4493ED008A83ED000A9AF818
:1033C000483030EE480A20EE298A53B3894B1B78E7
:1033D000DB0741F17780F7EE007AF4EEE7AAF1EE31
:1033E00010FA9BF86431C1F28687002B01F08981C5
:1033F000DBF86831049AD31A7F4A12689A4210DDCA
:103400007E4BD3ED007AF0EEECCAF4EEE7CAF1EEB3
:1034100010FA42F18882002318468BF86431F7F7DE
:10342000B1FE774B9BF874212B4493ED000A29EEF3
:10343000000A20EE088A89ED008A32B9039B87EDE5
:1034400000CA03ED01CA89ED00CA0136032E08F156
:10345000040809F1040907F1040705F104057FF4E4
:10346000E3AD029B1B78072B01F04A87012B02F08A
:10347000ED81002307939BF87C31002B41F0C5833D
:10348000604BDFF8B4A11E68DAF8003096F82C70B3
:10349000D80401F1AC805C4B5C4A039319465C4B49
:1034A000498B5C4DD2ED005AD3ED004A5A4A5B4B32
:1034B000D5ED036A93ED005AD2ED007AD2ED013AD0
:1034C00092ED026ACBED635A07EE101AB8EEC77A96
:1034D00034EEE54A012336EEC77ACBED615A8BED27
:1034E000604ACBED644A8BF89431C7EE055A338DB0
:1034F0005A4206EE902A4A4ADFED4A4A92ED005AB5
:10350000494A92ED004AB7EE007AF4EEC75A35EE1A
:10351000045AF1EE10FA88BFF0EE475A35EE275AFA
:10352000F8EEE66AF4EEE45AF1EE10FA07EE903A9D
:10353000B4EEE65AB8BFF0EE645AF1EE10FACBEDF5
:10354000675AB8EE677A01F14585B4EEC75AF1EED5
:1035500010FA88BFB0EE475A314BDFED344AD3ED55
:10356000017A314B93ED014A77EE847A25EE245AA5
:1035700077EEA37AF4EEE76AF1EE10FA08DCB4EE27
:10358000E77AF1EE10FA8CBFF0EE676AF0EE476A68
:10359000234A738DD2ED027A9FED247A5A4204EECB
:1035A000102A76EE277AB8EEC44A66EE876AF4EE01
:1035B000C47AF1EE10FA4CD440E000BF9C9D00208C
:1035C00000960020F88800209C88002084000020BD
:1035D0004084002010890020A88800204884002012
:1035E000448400209C840020988400205096002071
:1035F0008C2F00201C770020F488002000890020F8
:10360000B488002054960020189100207C9D002052
:10361000809D0020A07800204C3B0020A88900203D
:10362000403B002000000000583B00206F12833A0E
:10363000C8880020F08800205C62002007EE103A65
:10364000B8EE474AB4EEE74AF1EE10FA88BFB0EEA2
:10365000674AEA4BDFEDEA7A5B7824EE274A0BB93A
:10366000B1EE444A002F42F09680B7EE003AE54FA3
:103670003A78002A03F08C81E34B9FEDE46AD3EDA6
:10368000024A93ED017AD3ED037A66EEA44AE5EEA1
:10369000074AE4EE274A63EE244AF4EEC64AF1EE06
:1036A00010FAB4BFF0EE463AF0EE643A98BFB0EECE
:1036B000646A012ACDED0C4A03F0A081D3ED067AAD
:1036C000D3ED052A93ED077A66EEA77AE5EE227A26
:1036D000E4EE077A23EE277AB4EEC67AF1EE10FA1A
:1036E000B4EEE37A8CBFF0EE467AF0EE477AF1EE74
:1036F00010FA98BFB0EE676AB4BFF0EE637AF0EEEE
:10370000477A022A8DED0D7A00F0DE8093ED0A7A79
:10371000D3ED092AD3ED0B3A26EE877AA5EE227A6D
:10372000A4EE237A23EE077AB4EEC67AF1EE10FA0D
:10373000B4EEE77A8CBFF0EE463AF0EE473AF1EE9F
:1037400010FA98BFB0EE636AA8BFF0EE477A032A7A
:103750008DED0E7A00F0B88093ED0E7AD3ED0D2A40
:10376000D3ED0F3A26EE877AA5EE227AA4EE237ADD
:1037700023EE077AB4EEC67AF1EE10FAB4EEE77AE9
:103780008CBFF0EE463AF0EE473AF1EE10FA98BFF1
:10379000B0EE636AA8BFF0EE477A042A8DED0F7A87
:1037A00000F09280D3ED123AD3ED112A93ED137A03
:1037B00066EEA33AE5EE223AE4EE073A63EE233AE8
:1037C000F4EEC63AF1EE10FAF4EEE73A8CBFB0EE42
:1037D000467AB0EE637AF1EE10FA98BFB0EE476A1F
:1037E000A8BFF0EE637A052ACDED103A6CD0D3ED88
:1037F000163AD3ED152A93ED177A66EEA33AE5EE65
:10380000223AE4EE073A63EE233AF4EEC63AF1EEDA
:1038100010FAF4EEE73A8CBFB0EE467AB0EE637A77
:10382000F1EE10FA98BFB0EE476AA8BFF0EE637AE7
:10383000062ACDED113A47D0D3ED1A3AD3ED192A25
:1038400093ED1B7A66EEA33AE5EE223AE4EE073AF0
:1038500063EE233AF4EEC63AF1EE10FAF4EEE73AEC
:103860008CBFB0EE467AB0EE637AF1EE10FA98BFF4
:10387000B0EE476AA8BFF0EE637A072ACDED123AA0
:1038800022D093ED1E7AD3ED1D2AD3ED1F3A26EEFA
:10389000877AA5EE227AA3EE847A27EE037AB4EE35
:1038A000C67AF1EE10FAB4EEE77A8CBFF0EE466A13
:1038B000F0EE476AF1EE10FA8DED137A98BFB0EE94
:1038C000666AA8BFF0EE477A77EEC67AF7EE006A2E
:1038D000F4EEE67AF1EE10FACBED4A7A44F360802A
:1038E00086EEA77A022ADDED0D7A67EE244A67EEAE
:1038F000877ACDED0C4ACDED0D7A2DD0DDED0E7A27
:1039000067EE877A032ACDED0E7A25D0DDED0F7AAA
:1039100067EE877A042ACDED0F7A1DD0DDED107A9F
:1039200067EE877A052ACDED107A15D0DDED117A94
:1039300067EE877A062ACDED117A0DD0DDED127A89
:1039400067EE877A072ACDED127A05D0DDED137A7E
:1039500027EE877A8DED137A2D4B1B6813F0805973
:1039600001F08084F6EE005ACBED675A002A02F08F
:10397000D487284B28499BED646A0878D978089148
:1039800026490591B1F906109BF9943109910399E3
:10399000DFF894E09BED635A214E498B9EF800803E
:1039A0000A91BDEEC66A07EE103ADAF800300899BF
:1039B000D6ED004ADBED606ADBED617A16EE10EAC7
:1039C000BDEEC56A00F0010C03F4805603F0100050
:1039D00003F480030B93B8EEC77A16EE103A002971
:1039E00041F0C481002841F09E8507489DED0C5AA6
:1039F00090ED006A0B4925EE866A17E040400020F2
:103A00006F12833A717700201889002000000000AF
:103A1000343B0020304100201C7700200847002064
:103A200014890020A03B002080640020A5EE076AD6
:103A3000B0EE675AA6EE265ABDEEC56A16EE108A9B
:103A400016EE106AF045A8BF76464345C8BF1E462D
:103A500006EE106AB8EEC66A012A81ED006A00F02F
:103A6000DC8090ED046A9DED0D5A25EE866AA5EE88
:103A7000076AB0EE675AA6EE265ABDEEC56A16EE84
:103A8000108A16EE106AF045A8BF76464345C8BFB7
:103A90001E4606EE106AB8EEC66A022A81ED016A79
:103AA00000F0BB8090ED086A9DED0E5A25EE866A07
:103AB000A5EE076AB0EE675AA6EE265ABDEEC56AB5
:103AC00016EE108A16EE106AF045A8BF76464345FA
:103AD000C8BF1E4606EE106AB8EEC66A032A81ED1C
:103AE000026A00F09A8090ED0C6A9DED0F5A25EE67
:103AF000866AA5EE076AB0EE675AA6EE265ABDEEB4
:103B0000C56A16EE108A16EE106AF045A8BF764612
:103B10004345C8BF1E4606EE106AB8EEC66A042AC0
:103B200081ED036A79D090ED106A9DED105A25EE73
:103B3000866AA5EE076AB0EE675AA6EE265ABDEE73
:103B4000C56A16EE108A16EE106AF045A8BF7646D2
:103B50004345C8BF1E4606EE106AB8EEC66A052A7F
:103B600081ED046A59D090ED146A9DED115A25EE4D
:103B7000866AA5EE076AB0EE675AA6EE265ABDEE33
:103B8000C56A16EE108A16EE106AF045A8BF764692
:103B90004345C8BF1E4606EE106AB8EEC66A062A3E
:103BA00081ED056A39D090ED186A9DED125A25EE27
:103BB000866AA5EE076AB0EE675AA6EE265ABDEEF3
:103BC000C56A16EE108A16EE106AF045A8BF764652
:103BD0004345C8BF1E4606EE106AB8EEC66A072AFD
:103BE00081ED066A19D090ED1C6A9DED135A65EEC1
:103BF000865AE7EE055AE6EEA57AFDEEE77A17EE6D
:103C0000900A8645A8BF86468342D8BF734607EE12
:103C1000903AF8EEE77AC1ED077ABCF1000F01F0B7
:103C2000B381E44B1B68002B41F0BB81E24B1B7856
:103C30009BB1387870B1DFF8A883DFF8A89300262D
:103C4000F0B2D9F80030B8EC010A9847387801365C
:103C50008642F5DBD94B1B689847029B1B78072BE4
:103C600001F0638300230793DAF8008018F4806F73
:103C700041F0B481D24B059A1C68B2F90670628992
:103C8000974280F265864FF07E53CBF82431DFF8FF
:103C90005893059A039BB2F900001E8B99F90430E2
:103CA00099F8001099F801E0002BA0EB060383EAD5
:103CB000E37CACEBE37C14BF01224FF0FF32BCF598
:103CC000FA7FA8BF4FF4FA7C614580F23D86ACEBE9
:103CD000010307EE903AF8EEE77A8642C5ED007AE6
:103CE00003DDF1EE677AC5ED007A059BB3F90200BA
:103CF000831B83EAE37CACEBE37CBCF5FA7FA8BFD3
:103D00004FF4FA7C614580F21B86ACEB010307EEB1
:103D1000903AF8EEE77A8642C5ED017A03DDF1EEDE
:103D2000677AC5ED017A059BB3F904108B1B83EA12
:103D3000E370A0EBE370B0F5FA7FA8BF4FF4FA7020
:103D40007045CCBFA0EB0E0E4FF0000E02FB0EFE36
:103D500007EE90EAF8EEE77AB142C5ED027ABCBF11
:103D6000F1EE677AC5ED027A18F4805A00F0C38547
:103D7000B7F5FA6F3A46A8BF4FF4FA62B2F57A7F08
:103D80009BF8A431B8BF4FF47A72A2F57A72002B77
:103D900040F0CA858B49DFF854E281FB0230D3172B
:103DA000C3EB6013581C6FF0630C3EF910003EF932
:103DB00013E00CFB0323A0EB0E0003FB00F381FBDD
:103DC0000321DB17C3EB61139E440FFA8EFE07EE4F
:103DD00090EAB8EEE78A85ED038ABAF1000F41F068
:103DE0006881794B1E8816F04003059300F0DD8052
:103DF000764B774993ED019A93ED026A91ED020AB1
:103E000091ED043AD3ED030AD3ED003AD1ED038AE4
:103E1000D1ED015AD5ED011A95ED002A6D4B30EE2A
:103E2000435A39EE467A73EEA07A25EE077A75EE9C
:103E3000E84A73EEE09A35EEA8AA24EEA71AB0EE8F
:103E4000474AAAEE294A16F00302B0EE415A79EE2B
:103E5000067A70EE036AAAEE295AA6EEA74AA6EEE3
:103E6000E75AF0EE474AD6EEA74A34EE014AF6EE9C
:103E7000006A73EE89AA26EEC44A35EE475A35EE3B
:103E8000807AF0EE647AEAEE694AA7EE2A4A77EE83
:103E9000C17A36EE607A73EE68AA25EE265AEAEE0B
:103EA000297AAAEE875A74EE814A24EE047A73EED8
:103EB000C93A33EE283A64EEA64A75EEC05A36EE99
:103EC000206A67EEA66AF0EE477AE3EE234AD5EE63
:103ED000057AA5EE057AE5EE866AF1EE648AB0EE23
:103EE000476AB0EE677AF1EE663AA8EEA47A64EE1D
:103EF000260A26EEA43AA3EEA66AB1EE450AE3EE40
:103F0000A67AF0EE609AB0EE431A64EE243AA6EE7A
:103F1000A67AE5EE249AA0EE041AF0EE665AA8EE10
:103F2000A46AF0EE638A71EEA16AE0EE240AE5EE7F
:103F3000258A27EE217A32EE029AA5EE043A61EE46
:103F4000211A66EEA96AE4EEA47AE0EE253A0CBFE7
:103F5000D5ED022ADFED202A83ED005AE2EE066A53
:103F6000A9EE207AE2EE281A33EE033A67EEA27A3F
:103F700073EEA33AB0EE006AA2EE837AE2EEA36A91
:103F8000E1EE867A8BED6C7A85ED017ACBED6B6A8A
:103F9000C5ED006ACBED6D7A83ED014AC3ED025A9F
:103FA000C3ED034A0AB9C5ED027A0C4B1B6813F046
:103FB000140F1DE03C840020A86700207C640020D2
:103FC000589600201F85EB51509600205C2200205F
:103FD000840000209422002000000000F4950020BE
:103FE000A03B002074640020949D00208C9E002043
:103FF00003D016F4027F41F0C580DA4A12789AB1F4
:10400000039A528BBA420FDBD74A1278012A01F089
:104010004584192A01F042840E2A05D0082A03D0CB
:104020000022AA60CBF838219BF8DA7117B1B207E9
:1040300041F0F2839BF8E071002F40F0DB87039A98
:10404000927F002A00F04F84022A01F0D983032ACC
:1040500041F0D283039A92F82020C2EB421102EB86
:104060008101C90089B2039AD27F0232D2B2002FF5
:1040700000F0E385002900F0E085BC4B1B68B1FB34
:10408000F3F10FFA81F8ABF81082AAB307EE908A29
:10409000F8EEE77AF7EE006A86EEA77A012AD5ED08
:1040A000007ADBED896A77EEE67A67EE877ACBED08
:1040B000857A21D0D5ED017ADBED8A6A77EEE67A52
:1040C000022A67EE877ACBED867A15D0D5ED027A93
:1040D000DBED8B6A77EEE67A032A67EE877ACBED23
:1040E000877A09D0D5ED037ADBED8C6A77EEE67A34
:1040F00067EE877ACBED887A029B1B78092B03F059
:10410000AF82B8F1000F40F3F4839AB39BED897A44
:10411000DBED857A77EE877A012ACBED897AC5EDDA
:10412000007A21D09BED8A7ADBED867A77EE877A6A
:10413000022ACBED8A7AC5ED017A15D09BED8B7AF8
:10414000DBED877A77EE877A032ACBED8B7AC5EDA4
:10415000027A09D0DBED8C7A9BED887A77EE877A4C
:10416000CBED8C7AC5ED037A013A022AB8BF022260
:10417000D3B20693002F069818BF02202378DFEDF4
:10418000806AA27807EE903AF8EEE77AB0EE007A0D
:1041900067EEA67A029BF4EEC77AF1EE10FA197870
:1041A00040F30387DFED736A37EEC77AB0EE676AD4
:1041B000A7EE266AF0EE466A95ED007A9FED6E6AEC
:1041C00027EE066AF0EEC65A8BED536ACBED565ACF
:1041D0009AB107EE102AB8EEC75A9FED697A66EEDB
:1041E000064A25EE075AB7EE007A37EE457A64EEB6
:1041F000A54AA4EE857A26EE076A9FED607A637978
:1042000026EE877A27EE067ACBB1DFED5D6A9FED69
:104210005D6A65EEA65A06EE903AF8EEE66A66EE3C
:10422000A56AF4EEC66AF1EE10FA01F38482F7EEA5
:10423000005A75EEE66A85EEA66A27EE067A0C2924
:104240009FED518ADFED516A01F01B80B4EEC87A10
:10425000F1EE10FA98BFB0EE478AB4EEE68AF1EEBE
:1042600010FAB8BFB0EE668A8BED4C8A002800F0D9
:10427000F580B0EE007AF4EEC77AF1EE10FA05DDC3
:1042800037EEC77ADFED3B6AE7EE267A95ED017AE5
:10429000DFED396A27EE267AF0EEC75A8BED547AB5
:1042A000CBED575A9AB106EE902A9FED356AF8EE9B
:1042B000E66A27EE075A66EE866AB7EE006A36EEC1
:1042C000666A25EE255AA6EE856A27EE067ADFEDA8
:1042D0002B6AA37967EEA67A67EE877AABB107EE11
:1042E000103AB8EEC77A9FED266ADFED266A27EE10
:1042F000257A27EE067AB4EEE67AF1EE10FA41F36B
:104300003382DFED1B6A67EEA67A0C2900F0D487B2
:10431000DFED1D6A9FED1D7AF4EEE67AF1EE10FAFC
:1043200088BFF0EE667AF4EEC77AF1EE10FAB8BF05
:10433000F0EE477A0128CBED4D7A40F38F80637819
:10434000DFED0F6A07EE903AF8EEE77AB0EE007A0A
:1043500067EEA67A637AF4EEC77AF1EE10FA1DDD05
:1043600016E000BFA4220020404000203C40002076
:104370000000C842D7A368416F12033B00004843C6
:104380000AD7233CA4707D3F00C0F94400C0F9C4A3
:1043900037EEC77A5FED096AE7EE267A95ED027A85
:1043A0005FED0B6A27EE267AF0EEC75A8BED557A51
:1043B000CBED585A9BB106EE903A1FED0F6AF8EE1E
:1043C000E66A27EE075A66EE866AB7EE006A36EEB0
:1043D000666A25EE255AA5EE266A27EE067A5FED77
:1043E000196AE37967EEA67A67EE877AFBB107EE82
:1043F000103AB8EEC77A1FED1E6A5FED1E6A27EE0F
:10440000257A27EE067AB4EEE67AF1EE10FA01F399
:104410009681B5EEC07AF1EE10FA02F16584B7EE3E
:10442000006A36EE477AC6EE076A67EEA67A0C296E
:1044300000F01F875FED2C6A1FED2C7AF4EEE67A10
:10444000F1EE10FA88BFF0EE667AF4EEC77AF1EE7C
:1044500010FAB8BFF0EE477ACBED4E7A092900F09A
:10446000F386039B93F82140002C40F0A886BA4BBA
:1044700000221B688BF8E0219A0607D516F0300F52
:1044800004D0B64B1B78DB0702F1AD8114F04EFA75
:10449000002840F09483B24B1B7823B9B14B9B7832
:1044A000002B41F0CE81029B1D78072D7EF4C1AE1A
:1044B000F6F70AFD029AAC4B1578079A801AD88055
:1044C000FEF7B7BE9BF86431002B3EF4AAAF002381
:1044D00018468BF86431F6F755FEFEF7A2BFB1F926
:1044E00000209BED567AB1F90200DBED576A9F4937
:1044F00082EAE273A3EBE273F4EEC76A80EAE07249
:10450000F1EE10FAA2EBE072B4BFB0EE476AB0EE83
:10451000666A9342B8BF134607EE103A0B78B8EEBE
:10452000C77A27EE0A7A002B40F0BC80904BD3ED7F
:10453000005AF4EEEB5AF1EE10FA41F16881B7EE51
:10454000005A75EE654ADFED8B6A9FED8B5A8B4BF7
:1045500036EEC77A24EE855AD3ED006AE7EE055AA7
:1045600065EEA65AF5EEC05AF1EE10FA40F27686E4
:10457000CBEE256AB7EE007AF0EE475AE6EE665AC1
:10458000F0EE656AF4EEC76AF1EE10FA88BFF0EE5D
:10459000476AF5EEC06AF1EE10FAB8BFF0EE4C6A69
:1045A000774B93ED007A67EE877AA7EEA68AFEF73F
:1045B000A2BD0123FEF7F6BC724B734A2B4493ED68
:1045C000007AD2ED007A714B67EE277AF7EE006A37
:1045D000F4EEE67AF1EE10FA93ED007A88BFF0EE91
:1045E000667A67EE877A27EE888AFEF7E0BE684B28
:1045F000684D1B78D5ED037A13F0010F664B0393DA
:1046000004BF1B8BABF88831644B1B8807EE103A54
:10461000B8EEC77AF4EEC77AF1EE10FA42F28D8066
:104620005F4A128807EE102AB8EEC77AF4EEC77A0E
:10463000F1EE10FAC1F239815A4B5B4A93ED006AF0
:10464000D2ED006A9BF99431CBED636A76EE665A3F
:10465000012BCBED616ACBED605A8BED646A01F002
:10466000BE86049BCBF89831002237EEC77AFCEE69
:10467000E77A4E498BED677A17EE903AABF88831BE
:10468000012391ED005A8BF89431494B9A4242F242
:104690004180484BD3ED007AD3ED013A93ED026AA5
:1046A000FEF723BF354B93ED005AB5EEC05AF1EE3D
:1046B00010FA40F3D385404BD3ED006AF5EEC06AA3
:1046C000F1EE10FA40F3CA8536EEC77A66EE4B5A21
:1046D00087EE266AC5EE856AB7EE007AB4EEC76A41
:1046E000F1EE10FA88BFB0EE476AB5EEC06AF1EE9F
:1046F00010FA76EE876AB8BFB0EE4C6A66EE266AAC
:1047000040E72E4AD2ED007AB0EEC87AB4EEE77AEE
:10471000F1EE10FA7EF785AE294AD2ED007AB0EEBE
:10472000EC7AB4EEE77AF1EE10FA7EF77AAE254A2B
:10473000D8ED007A92ED007AF0EEE77AF4EEC77ADF
:10474000F1EE10FA7EF56DAE01220499CBF86811F6
:104750008BF86421FEF750BEF4950020529600209D
:104760001C36002014540020D0890020D48800205A
:10477000DC88002000003443610BB63BD088002069
:10478000CC880020782F0020C4880020C08800201A
:104790001C770020A078002018910020AC89002010
:1047A000AE890020809D002098890020B4890020D7
:1047B0008FD003004C3B0020D888002004890020C3
:1047C0000089002008890020E34A029207EE103A8F
:1047D0001278DFF8C483CBF80C71B8EEC77AF7EE25
:1047E000006A132A86EE879AB8F90400BBF81051C4
:1047F00094ED070A01F07F85D84BD94A93ED001A52
:10480000D3ED053A93ED122A93ED173AD3ED091A39
:10481000D3ED0E4A93ED016A93ED064A93ED0A7AC1
:10482000D3ED0F5AD3ED132AD3ED186A93ED045A42
:10483000D3ED030A67EE897A69EE288A29EE088AA1
:10484000E1EE273A02EB85060021A2EE283ACBF8EA
:104850000011CBF80411E1EE884AA6EE274AE7EEF4
:10486000085A93ED167A93ED0D6A93ED021AD3ED83
:104870000C1AC6ED003AE2EEA86A25EE635A27EE5E
:10488000437A93ED0B2AD3ED152AC6ED204AA0EE0C
:10489000E34A26EE646AD3ED143A83ED054AA1EEAD
:1048A000275AF0EE477AE1EEE45AA2EE086AE2EE09
:1048B000C36AE3EEA87A83ED065AC3ED0E5A83ED80
:1048C0000F6A86ED403AC3ED176AC3ED187ACBF84C
:1048D00008116B1C03F01F03ABF81031A8F804009B
:1048E000029BFEF767BAABF810229046002F3FF408
:1048F000C3AD022042E4039B5A8B9742C0F23F842F
:10490000B7F5FA6FD4BFC2EB0703C2F5FA634FF4F1
:104910007A7101FB03F19BF8A401C2F5FA63B1FBC4
:10492000F3F200283FF436AA9BF8A5318D4902FB2B
:1049300003F281FB0213D217C2EB6312FFF72ABA0C
:10494000DFED897AFFF7E7B9DFED877AFFF7C5B9C1
:10495000B7F5FA6F80F20E84217ABB1A03FB01F3DC
:10496000C2F5FA6293FBF2F3C3F1640307EE903AE7
:104970009FED7E7AF8EEE77A67EE877ACBED497A9B
:10498000FFF785B97A4B1978DBF81871DFF80CC29C
:104990009FED757AFE000CEB060383ED007A00298B
:1049A0007BD07448B0EE476AF0EE476A0023F0EC23
:1049B000017A013367EEA77A05EE903AB4EEE77A12
:1049C000F1EE10FAF8EEE55AB8BFB0EE677A8B4216
:1049D00076EEA76AA7EEA56AE9D1F5EEC06A0CEB00
:1049E0000603F1EE10FA83ED007A56DDC6EE265A84
:1049F000614B62490988F7EE007A75EEE75AD3ED0C
:104A0000007A65EEA77AFDEEE77A17EE903A812BF1
:104A100042F376818B42A8BF0B4607EE903AF8EE40
:104A2000E77A574BF01903EB800393ED057AD3ED4A
:104A3000003A93ED066A93ED014AD3ED046AD3ED93
:104A4000034A93ED025AA3EEA77AA4EE276A66EE14
:104A5000C76AA7EE646ABDEEC77AE5EE276A17EE6D
:104A6000100A812883ED056AC3ED066A42F3458189
:104A70008142A8BF014607EE901AF8EEE77AFCEEF5
:104A8000E77ACDED037ABDF80C300CEB06018B8094
:104A90001FB9BEF1130F02F06F87BEF1150F41F081
:104AA0006E816644DFF8F080B38828F81730DBF8B1
:104AB0001421344B013283FB02139918D317C3EB33
:104AC000A103C3EBC303D21ACBF814212E49DBF8A0
:104AD0001C21049D2D480B680078CBF81C51AA1AA4
:104AE00013440B60002840F0B88007EE902A284E4F
:104AF000DFF8AC90274FB8EEE78A06F2447506F56A
:104B0000F668F6EC017A94ED070AD4F86C37F8EE03
:104B1000E77A284627EE800A9847A5F1E000D4F806
:104B20008C369847A5F17000D4F8FC369847D6F833
:104B30005006D4F8AC309847D7ED007AA9EC010ABA
:104B4000E0EE087A2435A845E7EC017AD9D1029B3A
:104B50001D78FEF762BB00BFCD890020583E0020C3
:104B6000EC3B00201F85EB51000000000AD7233CDE
:104B7000CE3B0020202E0020D03B0020CC3B00204C
:104B8000EC3D002093244992249E0020C03B00204D
:104B90009C5A0020289E0020D0890020C43E00207E
:104BA00050620020614B624A19681288614BC969E2
:104BB00019805A8015B0BDEC0C8BBDE8F08F5E4CAF
:104BC00013F070FD6378022B00F05886032B7FF4FE
:104BD00062AC41F2B813E35C002B41F0878341F2F1
:104BE000A403E35C002B41F07C8341F2E803E35C27
:104BF000002B41F0718341F22C13E35C002B3FF456
:104C00004AAC4E4820F0C1FB45E44D4B4D4F1B785C
:104C1000DD0700F1B3833A78002A00F0B3854A4BF0
:104C20004A494B48039392002EF09EFB494BDFF814
:104C300034A1494D0593FEF7F4BFBBF8108208F18B
:104C4000FF380FFA88F8B8F1000FABF810823FF781
:104C50005CAA002F7FF44DAE0EE407EE902A3F4D84
:104C60003F4BDFF8D080DFF80091CDF80CB0F8EEC4
:104C7000E78A05F2D46600279B46CDF81880029B90
:104C8000D4ED077A1B78172B00F0988195ED007A08
:104C9000B8EEC78A082B28EE278A07D1B0EE480A5B
:104CA00005932EF035FD059BA8F80000DAF80020EA
:104CB00092000BD5002F03F0F181B0EE480AD4F832
:104CC0006C3706F170009847B0EE408AB0EE480AA3
:104CD000D4F88C36A6F170009847D4F8FC363046EC
:104CE0009847029B1B78032BB0EE408A00F061814D
:104CF000D5F85406D4F8AC30B0EE480A9847D9ED50
:104D0000007AABEC010AE0EE287A0137032F06F1B6
:104D1000240608F1020805F10405E9EC017AAED198
:104D2000029BDDF80CB01D78FEF777BA38980020AA
:104D3000C6360020D0890020589F002084B0002073
:104D40001C7700207177002018910020C8360020C1
:104D5000A03B002008470020A07800209C5A00209B
:104D6000506200205C620020289E0020002800F095
:104D7000C986D548BCF1000F42F00083B8F1000F9E
:104D800042F0A68190ED006A9DED0C5ACF4925EEC8
:104D9000866AFDEEE44AA5EE076AB0EE675AA6EE13
:104DA000265A14EE903ABDEEC56A16EE10CA16EEFB
:104DB000106AF445A8BF76466345C8BF1E4606EE96
:104DC000106AB8EEC66A012A81ED006A00F0DF8041
:104DD00090ED046A9DED0D5A25EE866AA5EE076AF0
:104DE000B0EE675AA6EE265ABDEEC56A16EE10CA98
:104DF00016EE106AF445A8BF76469C45B8BF1E461D
:104E000006EE106AB8EEC66A022A81ED016A00F069
:104E1000BE8090ED086A9DED0E5A25EE866AA5EEDD
:104E2000076AB0EE675AA6EE265ABDEEC56A16EEC0
:104E300010CA16EE106AF445A8BF76469C45B8BF66
:104E40001E4606EE106AB8EEC66A032A81ED026AB3
:104E500000F09D8090ED0C6A9DED0F5A25EE866A5C
:104E6000A5EE076AB0EE675AA6EE265ABDEEC56AF1
:104E700016EE10CA16EE106AF445A8BF76469C4599
:104E8000B8BF1E4606EE106AB8EEC66A042A81ED67
:104E9000036A7CD090ED106A9DED105A25EE866A6B
:104EA000A5EE076AB0EE675AA6EE265ABDEEC56AB1
:104EB00016EE10CA16EE106AF445A8BF76469C4559
:104EC000B8BF1E4606EE106AB8EEC66A052A81ED26
:104ED000046A5CD090ED146A9DED115A25EE866A45
:104EE000A5EE076AB0EE675AA6EE265ABDEEC56A71
:104EF00016EE10CA16EE106AF445A8BF76469C4519
:104F0000B8BF1E4606EE106AB8EEC66A062A81EDE4
:104F1000056A3CD090ED186A9DED125A25EE866A1E
:104F2000A5EE076AB0EE675AA6EE265ABDEEC56A30
:104F300016EE10CA16EE106AF445A8BF76469C45D8
:104F4000B8BF1E4606EE106AB8EEC66A072A81EDA3
:104F5000066A1CD090ED1C6A9DED135A65EE865AC8
:104F6000E7EE055AE6EEA57AFDEEE77A17EE900A2F
:104F70008645A8BF86468342D8BF734607EE903A5F
:104F8000F8EEE77AC1ED077A002A3EF44AAE9200C5
:104F90004F494E482EF0E8F94E4B1B68002B3EF46B
:104FA00045AE20F0EDFBFEF741BEF0EE676AFFF77D
:104FB00003B92EF0ADFBA8F8000099E695ED007A54
:104FC00004EB4702B8EEC78A128FA8F8002028EE3B
:104FD000278A6BE6B0EE665AFEF7BEBAA368002BCE
:104FE0003EF448AE3C49A1F14C009847DAF8008005
:104FF000FEF740BE39493A4AD1F8EC10126844F63F
:1050000020608142A8BF0146B1F57A7FB8BF4FF456
:105010007A7189B2D006ABF8E21145D5BAF1000F2A
:1050200001F072862F4AD2F800C0BCF832E04FEA95
:105030005E0E2D48DBF8E421D5ED037AA0FB0101DB
:105040008809642191FBF0F11429BDEEE77A0BEB9E
:105050004208A8BF142101328A42CBF8E42117EE9E
:10506000109AA4BF0022CBF8E4210BEB4202A8F86F
:10507000E891B2F9E82107EE102AB8EEC77A77EE88
:10508000C77AFDEEE77ACDED087ABDF9201081EA06
:10509000E172A2EBE172724501F3E98713494FF027
:1050A0007E520A60FEF7CBBF18F0805FB6D1FEF7E4
:1050B000C6BF1D210A4805F0D9FA002841F06D83CA
:1050C0000B4B03F1500219E018890020A03B00208F
:1050D000C83600203C840020BC5A0020E41D00207B
:1050E000343B002054960020D34D621084000020F1
:1050F0008032002004339A423EF473AE1978262998
:10510000F8D193F802E0D8788645F3D28F4BDB785C
:10511000002B7EF466AE8E4805F0A8FADFED8D7A9E
:105120008D49002802F0048438EE678AC6F57A7249
:10513000FDEEC87A12B2CDED057ABDF914301B032D
:1051400081FB0301DB17C3EBA11302FB03F343F362
:105150000F33334407EE903AB8EEE78A012385ED2A
:10516000038A8BF8A031FEF73CBE7C4B0293DFF83C
:1051700008B2ABE4237AC3F16403FFF7F7BB5146EF
:10518000FFF7C9BB764A127812F0100201F0A08333
:105190009BF8B811DBF8BC2195ED017A00290CBF12
:1051A00001214FF0FF3102FB01F207EE902AF8EEE9
:1051B000E77A77EE877AC5ED017AFEF71EBF1E21EA
:1051C000634805F053FA00283FF451A9059B002BD2
:1051D0007FF44DA99BF83432A34242F06082614BC8
:1051E0009BED8E0AD3ED058ADBED4E5A9FED5E6A8C
:1051F000DFED5E6A20EE657A68EE007AA8EE287A26
:10520000E5EEA87AB4EEC67AF1EE10FA88BFB0EEF9
:10521000467AB4EEE67AF1EE10FAF4EEC67AB8BF4A
:10522000B0EE667AF1EE10FA88BFF0EE467AF4EE50
:10523000E67AF1EE10FAB8BFF0EE667A8BED4C7AB2
:10524000CBED4E7AFFF713B9FDEEC87A484A17EE58
:10525000903AA2F80480D380FFF703B9DFED456AE6
:10526000FFF79EB9DAF8003059023EF57BABFEF746
:105270007DBBBDEEE77A3E4B17EE102A9A80FFF712
:10528000D9B8B4EEC87AF1EE10FA98BFB0EE478AFA
:10529000BDEEC77AB4EEE68A354FF1EE10FA17EE9E
:1052A000103AB8BFB0EE668A8BED4C8A3B8000287E
:1052B0007EF4DFAFFFF7D5B89FED2B7ADFED2B6AD9
:1052C0002B4AF4EEC77AF1EE10FA98BFB0EE677A87
:1052D000FDEEE77AB4EEE67AF1EE10FA17EE903AC8
:1052E000B8BFB0EE667A01288BED4D7A53803FF758
:1052F00026A8FFF7B6B8002B3EF493A8FEF778B8BF
:10530000F5F7E2FD029B089A1B78DFF86480801AAB
:10531000012BA8F8020000F09B82072B7EF4A9A8BD
:10532000F5F7D2FD0790FEF7A6B8F5F7CDFD029B85
:1053300007991B780E4A401A072B90807EF492AC96
:10534000F5F7C2FD0790FEF78FBC00BF304100208B
:10535000343B002000007A44D34D6210CD890020F8
:10536000529600208400002000C0F94400C0F9C417
:10537000D089002000000000202E00203B78002B68
:1053800000F00082DBED573A9BED566ADBED617A67
:10539000ED4A9BED607AD2ED005A9BED544ADBED6D
:1053A000534AEA48EA49F4EEC63AF3EE046AF1EEEB
:1053B00010FA37EEA65A00F1C58290ED026A26EE89
:1053C000446AF0EE674AE6EE074AF4EEC54A34EE68
:1053D000E66AF1EE10FA48BFB0EE656A012B81ED86
:1053E000006A00F0CF8190ED066A26EE446AF0EE86
:1053F000674AE6EE074AF4EEC54A34EEE66AF1EE95
:1054000010FA48BFB0EE656A022B81ED016A00F028
:10541000B98190ED0A6A26EE446AF0EE674AE6EE3C
:10542000074AF4EEC54A34EEE66AF1EE10FA48BFD8
:10543000B0EE656A032B81ED026A00F0A38190ED66
:105440000E6A26EE446AF0EE674AE6EE074AF4EE8C
:10545000C54A34EEE66AF1EE10FA48BFB0EE656A6E
:10546000042B81ED036A00F08D8190ED126A26EE27
:10547000446AF0EE674AE6EE074AF4EEC54A34EEB7
:10548000E66AF1EE10FA48BFB0EE656A052B81EDD1
:10549000046A00F0778190ED166A26EE446AF0EE19
:1054A000674AE6EE074AF4EEC54A74EEE66AF1EEA4
:1054B00010FA48BFF0EE656A062BC1ED056A00F0F0
:1054C0006181D0ED1A6A66EEC46AF0EE674AE6EED4
:1054D000874AB3EE046AF4EEC54A74EEC66AF1EE8A
:1054E00010FA48BFF0EE656A072BC1ED066A00F0BE
:1054F0004981D0ED1E6A974B039326EEC44A964B22
:10550000DFF860A2954D0593E4EE077AF4EEC57AD4
:1055100077EEC67AF1EE10FA48BFF0EE657AC1ED8B
:10552000077AFEF77EBB89489DED0C5A90ED006A24
:10553000BCF1000F41F0748225EE866A8449A5EE25
:10554000076AB0EE675AA6EE265ABDEEC56A16EE99
:1055500010CA16EE106AF445A8BF76466345C8BF68
:105560001E4606EE106AB8EEC66A012A81ED006A90
:105570003FF40DAD90ED046A9DED0D5A25EE866A5F
:10558000A5EE076AB0EE675AA6EE265ABDEEC56ACA
:1055900016EE10CA16EE106AF445A8BF76466345AB
:1055A000C8BF1E4606EE106AB8EEC66A022A81ED32
:1055B000016A3FF4ECAC90ED086A9DED0E5A25EEC1
:1055C000866AA5EE076AB0EE675AA6EE265ABDEEC9
:1055D000C56A16EE10CA16EE106AF445A8BF7646E4
:1055E0006345C8BF1E4606EE106AB8EEC66A032AB7
:1055F00081ED026A3FF4CBAC90ED0C6A9DED0F5A41
:1056000025EE866AA5EE076AB0EE675AA6EE265A20
:10561000BDEEC56A16EE10CA16EE106AF445A8BFB4
:1056200076466345C8BF1E4606EE106AB8EEC66AE7
:10563000042A81ED036A3FF4AAAC90ED106A9DED57
:10564000105A25EE866AA5EE076AB0EE675AA6EEF6
:10565000265ABDEEC56A16EE10CA16EE106AF4455B
:10566000A8BF76466345C8BF1E4606EE106AB8EE70
:10567000C66A052A81ED046A3FF489AC90ED146A8C
:105680009DED115A25EE866AA5EE076AB0EE675ABF
:10569000A6EE265ABDEEC56A16EE10CA16EE106AC0
:1056A000F445A8BF76466345C8BF1E4606EE106A9D
:1056B000B8EEC66A062A81ED056A3FF468AC90ED43
:1056C000186A9DED125A25EE866AA5EE076AB0EEBD
:1056D000675AA6EE265ABDEEC56A16EE10CA16EE39
:1056E000106AF445A8BF76466345C8BF1E4606EE5D
:1056F000106AB8EEC66A072A81ED066A3FF447AC25
:1057000090ED1C6A9DED135A65EE865AE7EE055A38
:10571000E6EEA57AFDEEE77A17EE900A8645A8BF79
:1057200086468342C8BF9E4607EE90EAF8EEE77AC7
:10573000C1ED077A28E49FED0A6AFEF77EBDDFED32
:10574000086AFEF772BE00BF148900201889002085
:10575000A03B00201891002008470020A0780020DE
:105760000000C8425C620020B5EEC07AF1EE10FA8B
:1057700001F1B682B7EE006A36EE477AC6EE076AE6
:10578000FEF7C1BDCA4B0393CA4BDFF870A3CA4DE5
:105790000593FEF746BAC94A5379002B3DF465AF2D
:1057A000C74B1B78002B3DF460AF1278DFEDC54A84
:1057B00007EE902AC44AB8EE677A128807EE903A4C
:1057C00006EE102AF8EEE77AB8EE466A67EE277A18
:1057D000B7EE007A87EE863AB4EEE43AF1EE10FACC
:1057E00088BFB0EE643AB4EEC73AF1EE10FAB8BF33
:1057F000B0EE473AFDF73BBFB44A5188FEF733BCE1
:10580000BBF8E21101F57A7189B2FEF72CBCB04BFE
:10581000D3ED005AFEF7A6BEAE4A9FEDAF7AD2EDA9
:10582000087AF4EEC77AF1EE10FA00F2DD849FED0B
:10583000AB7AD5ED037A77EE877AC5ED037AFEF77A
:10584000F9BB049827F050FDFEF72DBEDFF8B082BB
:10585000F5F73AFBA24ADBF8783112680790C31AD1
:105860009A1ACBF87801A8F80430A8F80620FDF7BA
:1058700002BEF5F729FB0890FDF79BBBA3784FF01C
:105880000109072B3EF607AEDFE813F07206210789
:105890000A071607A806570661066E06914A927B0C
:1058A000002A3EF4BDABFEF7BFBBBBF888219A428D
:1058B00000F2E984262029F089FB002840F0E384E7
:1058C000894B8A4AD3ED007A894B92ED007A1B7896
:1058D000CBED637A8BED647A002B01F0C28377EE17
:1058E000676A9BF99431CBED606A0133CBED617A45
:1058F00001F08B86049BCBF8983100229FED777ADC
:105900007C498BED677AFF2391ED005A8BF8943137
:10591000FEF7BBBE0120F5F735FCDBF86821049BE0
:105920009A1AFDF701BC744BD8ED007A93ED007A1A
:10593000F0EEE77AF4EEC77AF1EE10FA7DF771AD8A
:10594000FDF769BD90ED016A26EE646AB0EE674A24
:10595000A6EE074AB4EEC54A34EE666AF1EE10FAD6
:1059600048BFB0EE656A012B81ED006A3FF40AAFD3
:1059700090ED056A26EE646AB0EE674AA6EE074A25
:10598000B4EEC54A34EE666AF1EE10FA48BFB0EEE6
:10599000656A022B81ED016A3FF4F4AE90ED096A6D
:1059A00026EE646AB0EE674AA6EE074AB4EEC54A30
:1059B00034EE666AF1EE10FA48BFB0EE656A032B6A
:1059C00081ED026A3FF4DEAE90ED0D6A26EE646A68
:1059D000B0EE674AA6EE074AB4EEC54A34EE666AF0
:1059E000F1EE10FA48BFB0EE656A042B81ED036A50
:1059F0003FF4C8AE90ED116A26EE646AB0EE674AD5
:105A0000A6EE074AB4EEC54A34EE666AF1EE10FA25
:105A100048BFB0EE656A052B81ED046A3FF4B2AE73
:105A200090ED156A26EE646AB0EE674AA6EE074A64
:105A3000B4EEC54A74EE666AF1EE10FA48BFF0EEB5
:105A4000656A062BC1ED056A3FF49CAED0ED196A7C
:105A500066EEE46AB0EE674AA6EE874AB3EE046AE1
:105A6000B4EEC54A74EE466AF1EE10FA48BFF0EEA5
:105A7000656A072BC1ED066A3FF484AED0ED1D6A5E
:105A80000B4B039366EEE44A0A4BDFF870A00A4D15
:105A90000593E4EE877AF4EEC57A77EEC67AF1EEF6
:105AA00010FAB8BFF0EE657AC1ED077AFEF7B9B823
:105AB0001891002008470020A0780020E4950020DD
:105AC0009E780020713DAA3F88780020A093002096
:105AD000D0880020FC9D00208FC2753C0000000093
:105AE0003C400020885900207C9D00209C8900209B
:105AF00080640020B0890020088900205C620020BA
:105B0000D0890020D648B8F1000F41F01B8190EDFC
:105B1000006A9DED0C5AD34925EE866AFDEEE44AF3
:105B2000A5EE076AB0EE675AA6EE265A14EE903A32
:105B3000BDEEC56A16EE108A16EE106AF045A8BFD3
:105B400076464345C8BF1E4606EE106AB8EEC66AE2
:105B5000012A81ED006A3EF460A890ED046A9DED93
:105B60000D5A25EE866AA5EE076AB0EE675AA6EED4
:105B7000265ABDEEC56A16EE108A16EE106AF0457A
:105B8000A8BF76469845B8BF1E4606EE106AB8EE26
:105B9000C66A022A81ED016A3EF43FA890ED086AC8
:105BA0009DED0E5A25EE866AA5EE076AB0EE675A9D
:105BB000A6EE265ABDEEC56A16EE108A16EE106ADB
:105BC000F045A8BF76469845B8BF1E4606EE106A57
:105BD000B8EEC66A032A81ED026A3EF41EA890ED73
:105BE0000C6A9DED0F5A25EE866AA5EE076AB0EEA7
:105BF000675AA6EE265ABDEEC56A16EE108A16EE54
:105C0000106AF045A8BF76469845B8BF1E4606EE16
:105C1000106AB8EEC66A042A81ED036A3DF4FDAF4E
:105C200090ED106A9DED105A25EE866AA5EE076A82
:105C3000B0EE675AA6EE265ABDEEC56A16EE108A79
:105C400016EE106AF045A8BF76469845B8BF1E46C6
:105C500006EE106AB8EEC66A052A81ED046A3DF4C4
:105C6000DCAF90ED146A9DED115A25EE866AA5EE23
:105C7000076AB0EE675AA6EE265ABDEEC56A16EE62
:105C8000108A16EE106AF045A8BF76469845B8BF50
:105C90001E4606EE106AB8EEC66A062A81ED056A4F
:105CA0003DF4BBAF90ED186A9DED125A25EE866A61
:105CB000A5EE076AB0EE675AA6EE265ABDEEC56A93
:105CC00016EE108A16EE106AF045A8BF7646984583
:105CD000B8BF1E46FDF77FBF634EDBED017A9BED3B
:105CE000006A3188736977EEA77AF0EE006AB0EE49
:105CF000677AA6EE267A4E1E0BEBC601D6EE267A02
:105D000008391033F6EE003A27EE237A67EEA37ACD
:105D10008BED207ACBED217ADFF85CB15F460BF199
:105D2000800091ED027A91ED036AD7ED036AD7ED19
:105D3000027A53ED014A13ED025A37EE674A76EEC6
:105D4000C65A77EE277AE4EE845A013EA1F10801A3
:105D5000E5EE047A07F1080703F1080336EE267A28
:105D600000F10800E4EE877AE5EE475A67EEA37A81
:105D700025EEA37AC0ED007A80ED017AD1D1BEF193
:105D8000140F7EF496AEF5F79FF8DFF8F080DBF89D
:105D90001421401BA8F80200FEF78BBEDBF81801A7
:105DA000BBF81031DFF8D8C0C3F120095FFA89F9D8
:105DB00003EB401E5FEA99020CEB8E0E01F0FB85AF
:105DC00001321701294E2A490EEB07080EF1100285
:105DD00012ED024A12ED035A12ED016A12ED047A35
:105DE00056ED024A56ED035A56ED016A56ED047A15
:105DF00064EE244A65EE255A66EE266A67EE277A37
:105E00001032904541ED024A41ED035A41ED016ADD
:105E100041ED047A06F1100601F11001D8D11549BF
:105E2000A7F11006B64401EB06085E4419F0030220
:105E300009D0BEEC017AF8EC017A67EE277A013AD4
:105E4000E6EC017AF5D1002B41F02081029B1B7812
:105E5000142B01F0C783DBF81421FEF72ABE00BF24
:105E600018890020A03B0020D43B00207C3D00206E
:105E7000302E00206C3D0020202E0020D0890020F4
:105E8000EC3B0020C84F39785FEA910C01F06E8737
:105E9000C64E0CF101094FEA491906EB090806F153
:105EA0002003A6F1700013ED076A53ED056A13EDA8
:105EB000037A53ED017A53ED025A13ED084A53ED7C
:105EC000064A13ED045A26EE066A66EEA66A27EE27
:105ED000077A67EEA77AA4EE046A20339845E4EEC9
:105EE000A46A00F11000A5EE057AE5EEA57AF1EEC0
:105EF000C65AB1EEE66AF1EEC76AB1EEE77A40ED56
:105F0000085A00ED076A40ED066A00ED057ACAD12D
:105F1000A9F1200333440BEB0C1611F0030010D051
:105F2000083353ED017A13ED027A67EEA77A013850
:105F3000E7EE077A03F10803B1EEE77AA6EC017AFF
:105F4000EFD1BEF1140F01F093850132CBF814218B
:105F5000FEF71ABDDBF81821954B9649964E184668
:105F6000D30019441A448B88016800EE103A10EEF1
:105F7000103A643BC82BA8BFC823782BB8BF78233E
:105F800007EE903AB8EEC07AF8EEE77A06EB8206B2
:105F900077EE670A77EE876A67EE877A20EEA67A51
:105FA000B8EE400AC7EE870A3046D6F81890D6F801
:105FB0001C80376A96ED058A22F080FB029B86EDF5
:105FC000058A1B78C6F81890142BC6F81C80376217
:105FD00001F03985DBF818317848DBF814210133FA
:105FE00080FB0310A0EBE37000EB4000181A0132B5
:105FF000CBF81801CBF81421D2E6714E7148B26883
:10600000B1892CF0BBF9029B93F800E0BEF1140FAC
:1060100001F02285DBF814210132CBF814215CE673
:10602000674E3288D6F804904FEA52084FEA88014A
:106030005FEAD20C0BEB01030BEB820700F0A180AF
:1060400001F110020CF1010C5F4803EB0C1C3A4407
:10605000103309F1100E07F1100151ED032A51ED33
:10606000043A10ED043A10ED032A51ED026A11EDE5
:10607000016A10ED021A50ED010A12ED044A12ED08
:10608000035A53ED044A53ED035A13ED027A53EDCC
:10609000017A52ED021A12ED010A73EE238A32EEF2
:1060A000228A40ED048A00ED038A71EE268A30EEE2
:1060B000868A40ED028A00ED018A74EE848A35EE0C
:1060C000858A43ED048A03ED038A77EE218A37EE51
:1060D000808A43ED028A03ED018A73EE633A75EE1E
:1060E000655A1EED035A32EE623A74EE644A25EEAA
:1060F000638A1EED044A23EE052A64EE652AA3EEA8
:10610000048A10339C4524EE843AA3EE842A00F1DD
:1061100010000EF1100EA5EE853A01F1100102F10A
:106120001002E4EE852A01ED078A01ED082A02ED4E
:10613000073A42ED082A5EED055A1EED065A71EE49
:10614000666A30EEC66A31EEC77A70EE677A26EE7E
:10615000253A65EEE63A25EE674A67EE054AE6EE31
:10616000053AA6EE853AA7EE254AE7EEA54A01EDE7
:10617000063A41ED053A02ED064A42ED054A7FF442
:106180006CAF1FFA88F84A4641460E4821F03AFCA7
:1061900041467268384621F035FC029B1B78142B6F
:1061A0007FF459AEEFE500BFCE3B0020A02E0020CB
:1061B0004C620020C43E0020E06100205655555539
:1061C000D43B0020202E0020302E0020306E99BCC1
:1061D0002716983DA40DC93F843459BEDB0F4940B2
:1061E000D06D393A00000000F0EEE76AB7EE005AD1
:1061F00035EE665A1FED0B4A5FED0B5A1FED0A6A2A
:106200001FED0C7A9BED770A0893F1EEC54AE6EE96
:10621000845AF5EEC07AA6EEA56AF1EE10FAA6EE63
:10622000867A48BF5FED137A27EE247A48BF37EEAF
:10623000C77A27EE000A2DF06BFAB0F5617F089B54
:1062400000F3018707EE900AB8EEE70A5FED1C7ACB
:1062500020EE270A07EE907AB8EEE78AFDEEC07AC4
:1062600017EE902A2032402A40F2F3861FED230ACF
:1062700008932DF04DFA00B207EE900A089BB8EE95
:10628000E77AFFF7D6BA9BF8A021002A7FF418AB73
:10629000C34BC44993ED007AD1ED007A9BF9943158
:1062A000CBED637A77EE676A012BCBED617ACBEDAC
:1062B000606A8BED647A01F06D83049BCBF89831B2
:1062C000B94B9FEDBA7A93ED005A8BED677A0123B3
:1062D0008BF89431FEF7D9B9B5481FF056F8FEF7A0
:1062E0008ABCB4481FF051F8FEF77FBCB2481FF0DB
:1062F0004CF8FEF774BCB14EB14F96ED004A96EDE6
:10630000057AD6ED014A96ED066AD6ED046A96ED59
:10631000035AD6ED025A67EE897A07EB8503A4EE9D
:10632000277AA4EEA76A66EEC76AA5EE476AE5EE8D
:10633000A76A20EE070A86ED056AC6ED066A29EE11
:10634000088A69EE288A83ED007A2DF0E1F9D6ED0E
:106350000E5AD6ED176A96ED091AD6ED121A96ED79
:106360000F5A96ED187A96ED0A2AD6ED132A96ED75
:106370000D6AD6ED167A96ED0C3AD6ED0B3A96EDFF
:10638000154AD6ED144AE1EE085A002207EB8501C2
:10639000E8EEA16A00B2CBF80021A2EE085ACBF8D1
:1063A0000421CBF80821A8EEA27A26EE656A67EEF2
:1063B000E67AA3EE655AA3EE886AA6EEC47AE8EE02
:1063C000A47A86ED0E5AC1ED205A86ED0F6AC1ED12
:1063D000406A86ED177AC6ED187AFEF77ABADBF8CE
:1063E0009821049B9A1AFEF740B9B4F9383022621A
:1063F00007EE903A0122F8EEE77A2366E26700237F
:10640000012FC4ED1C7AC4ED1B7A636701F08C8206
:10641000B7427CF439ADB4F93A30636607EE903A8E
:1064200000220123F8EEE77A6262C4F8903000237C
:10643000012FC4ED217AC4ED207AC4F8883001F030
:106440009782B7427CF451ADB4F93C30A36607EEB5
:10645000903A00220123F8EEE77AA262C4F8A43051
:106460000023012FC4ED267AC4ED257AC4F89C30B0
:106470007CF46CAD9FED4D8A032D2AD0B9F1000F4D
:1064800009D007EE909AF8EEE77AF4EEC87AF1EECA
:1064900010FA01F170844B4BDFF83CB11A68A36E1F
:1064A0009BF82011A8F8060003EB560393FBF6F6C1
:1064B0000023A66293621363D36229B1424B1B6827
:1064C00033F480637CF446AD012026F04FFBFCF7EB
:1064D00041BDB0EE480A2DF01BF900B2CEE72369AA
:1064E0000622652BA27032D92278032A14BF6FF0DE
:1064F000FF026FF07F02A3F1650303EA020303F1D9
:10650000010314BF4FF4807280229A4223611ED28D
:106510003268E66802329F19974281F086842B4ADE
:106520006660D16FA760490203FB01F30521166085
:1065300042F81C3C42F8183CA170A2682449012092
:1065400011F0C0FD012841F066840623A3700021EC
:10655000204811F07FFD012841F05D84A3780133CC
:10656000DBB2A370FFF78DB903236370FDF793BF10
:1065700000230CAD29461846092211F02BFC0128F6
:106580007DF489AF0C9B93F8FE21552A01F0188207
:1065900041F2B41202210123A1546370FDF77BBFC5
:1065A000809D002098890020B48900200000000010
:1065B00040B00020FCAF002010B10020583E002069
:1065C000EC3B0020389800204C960020ECB00020D6
:1065D0005C9F0020C8B00020202E00202278237D60
:1065E000D24EDFF8A883032A14BF4FF480778027A8
:1065F000002B41D0012BFBD1CD4B6268196830686C
:1066000000234FEA412E4FF0FF31B1FBFEF112EBB8
:10661000010A43F1000B0021594500F1020008BFB7
:10662000504538BF82465246C249022011F07CFED6
:10663000032801F2BD8101A353F820F0974401081B
:106640004D660108974401084D6601086268A36819
:106650002569991AA94284BFE260216103283FF4A9
:106660003EAF0133B3FBF7F207FB12320AB13B44F2
:106670009B1A002263602275326841460232002074
:1066800011F052FE032801F2938101A353F820F088
:10669000974401080967010897440108DF6401086D
:1066A000A54B00930320A07030230522A349A448E2
:1066B0001EF018FFFDF7EFBE41F27013E35C002BF4
:1066C0003DF4E9AE9E481EF060FEFDF7E4BE0CAD61
:1066D00041F2FC162946A0590023092211F07AFB49
:1066E00001287DF4D8AE00230C9A2370B2F80B3049
:1066F000B3F5007F01F0A28341F2B412032101231C
:10670000A1546370FDF7C7BE636884F81490013329
:10671000A36071E7DFED8B7A8B4B9BED677AC3ED5E
:10672000007AC3ED017AC3ED027A884BB0EE676A56
:10673000F0EE673A1E68FCF7D8BE854B854AD3ED6C
:10674000006A854B92ED006A1B78CBED636A8BED96
:10675000646A002B00F0CC8276EE665A9BF9943185
:10676000CBED605A0133CBED616A00F0FF85049BED
:10677000CBF89831002237EE677AFCEEE77A77495A
:106780008BED677A17EE903AABF88831FF2391EDE5
:10679000005A8BF89431FDF778BF714BDB78002BF2
:1067A0007EF48EACDFED6F7A6F4938EE678AC6F5FE
:1067B000FA63FDEEC87A1BB2CDED057ABDF914205F
:1067C000120381FB0201D217C2EBA11203FB02F3F9
:1067D00043F30F33334407EE903AB8EEE78A85ED82
:1067E000038AFEF76DBC614B614AB3F90430DFEDFB
:1067F000617A82FB0312DB17C3EBA2031BB208EE24
:10680000103AB8EEC88A28EE278AB0EE480A03F09C
:1068100061FDF0EE408AB0EE480A03F0E1FC564B11
:10682000DC78002C00F0CC83544ABBF93E12B2F95C
:10683000023044F250605B1A834240F3DE86A3F5D7
:106840000C43A03B65429D4200F3ED86A342A8BFE6
:106850002346B2F90020BBF93C020B44121A44F261
:1068600050611BB28A42ABF83E3240F3D486A2F5A7
:106870000C42A03A954203DC9442A8BF1446254638
:10688000421912B207EE902A07EE103AF8EEE77AB4
:10689000B8EEC77A67EEE86A9FED396AABF83C223A
:1068A000E0EE076A60EE277AE8EE877A26EE867ACF
:1068B00067EE867ABDEEC77AFDEEE77A17EE102A0C
:1068C00017EE903AABF84821ABF84A31FDF7DEBD40
:1068D00099F80300BBF9C011002800F08B83A7EBE7
:1068E000010C99F802008CEAEC7EAEEBEC7E86455A
:1068F00040F39C868F42C8BF404207EE900AF8EEF4
:10690000E77A4FF0010E37EE888ACBF8C4218BF876
:10691000C8E185ED038AFDF770BB1A4B18781A4B56
:10692000059300F0010CFDF778B900BF60B10020BD
:1069300068B10020609F0020254203080C7C0408F9
:10694000C8B00020000000004C3B002054960020FE
:106950007C9D00209C89002080640020B08900205C
:106960003041002000007A44D34D62100096002090
:106970006766666635FA8E3CFC430020584400206A
:10698000CDCCCC3D1C770020084700205C9F002028
:10699000E64BDFEDE77A1B68CBED4A7A13F08059BE
:1069A00040F07E83DAF8003013F4800900F0B38100
:1069B0004FF00009B6EE007A67EE877AF4EEE75AF8
:1069C000F1EE10FA48BFF0EE675A40F16983CBED63
:1069D000675AFCF7CBBFF4F777FA029B93F800E015
:1069E000BEF1140F05BFDFF85883DBF81421DBF884
:1069F0001421A8F800200546FCF7E5B973EEC67A25
:106A0000B7EE007AF4EEC77AF1EE10FACBED4A7ADF
:106A100040F3C68784EEA77A8DED0C7AFCF79CBF15
:106A2000002E00F0678625EE866AC249A5EE076A49
:106A3000B0EE675AA6EE265ABDEEC56A16EE10CA2B
:106A400016EE106AF445A8BF76466345C8BF1E46D9
:106A500006EE106AB8EEC66A012A81ED006A3DF4BE
:106A6000E0A890ED046A9DED0D5A25EE866AA5EE2C
:106A7000076AB0EE675AA6EE265ABDEEC56A16EE54
:106A800010CA16EE106AF445A8BF76466345C8BF23
:106A90001E4606EE106AB8EEC66A022A81ED016A49
:106AA0003DF4BFA890ED086A9DED0E5A25EE866A6A
:106AB000A5EE076AB0EE675AA6EE265ABDEEC56A85
:106AC00016EE10CA16EE106AF445A8BF7646634566
:106AD000C8BF1E4606EE106AB8EEC66A032A81EDEC
:106AE000026A3DF49EA890ED0C6A9DED0F5A25EECA
:106AF000866AA5EE076AB0EE675AA6EE265ABDEE84
:106B0000C56A16EE10CA16EE106AF445A8BF76469E
:106B10006345C8BF1E4606EE106AB8EEC66A042A70
:106B200081ED036A3DF47DA890ED106A9DED105A49
:106B300025EE866AA5EE076AB0EE675AA6EE265ADB
:106B4000BDEEC56A16EE10CA16EE106AF445A8BF6F
:106B500076466345C8BF1E4606EE106AB8EEC66AA2
:106B6000052A81ED046A3DF45CA890ED146A9DED60
:106B7000115A25EE866AA5EE076AB0EE675AA6EEB0
:106B8000265ABDEEC56A16EE10CA16EE106AF44516
:106B9000A8BF76466345C8BF1E4606EE106AB8EE2B
:106BA000C66A062A81ED056A3DF43BA890ED186A95
:106BB0009DED125A25EE866AA5EE076AB0EE675A79
:106BC000A6EE265ABDEEC56A16EE10CA16EE106A7B
:106BD000F445A8BF76466345C8BF1E4606EE106A58
:106BE000B8EEC66A072A81ED066A3DF41AA890ED50
:106BF0001C6A9DED135A65EE865AE5EE075AE5EEDE
:106C0000A67AFDEEE77A17EE902A9645A8BF96463B
:106C10009A42A8BF734607EE903AF8EEE77AC1EDC4
:106C2000077AFCF7FEBF012940F37E8607EE10EAE3
:106C3000B8EEC77AC7EE876AB1EEE68A032D14D0A4
:106C4000B9F1000F09D007EE909AF8EEE77AF4EE6A
:106C5000C87AF1EE10FA01F18E80236E03EB560331
:106C600093FBF6F32362FFF7D3BBB0EE480A2CF098
:106C70004FFD00B2E4E7012940F37A8607EE10EAFF
:106C8000B8EEC77AC7EE876AB1EEE68A032D14D054
:106C9000B9F1000F09D007EE909AF8EEE77AF4EE1A
:106CA000C87AF1EE10FA01F16680636E03EB5603C9
:106CB00093FBF6F36362FFF7C4BBB0EE480A2CF017
:106CC00027FD00B2E4E701297FF7D4AB07EE10EA15
:106CD000B8EEC77AC7EE876AB1EEE68AFFF7CCBB9B
:106CE000F7EE006AFDF70FBBF7EE006AFDF79DBBFC
:106CF00076EEC65AF0EE466A30E58223FDF7C5BE51
:106D0000DFED0D7AFDF78DBE0C4AD2F800C0BCF95C
:106D100032E0FEF78EB9B6EE007AF4EEC75AF1EE25
:106D200010FA3FF747AEFCF721BE00BF343B00200E
:106D300000000080A03B0020000002435496002089
:106D4000D089002090ED006A9DED0C4ADA4925EECD
:106D5000866AFDEEE43AA4EE076AB0EE674AA6EE54
:106D6000264A13EE903AB4EEC45AF1EE10FAB0EEA1
:106D7000446A88BFB0EE646ABDEEC66A16EE108A39
:106D800016EE106AF045A8BF76464345C8BF1E46BA
:106D900006EE106AB8EEC66A012A81ED006A3CF47C
:106DA0003CAF90ED046A9DED0D4A25EE866AA4EE97
:106DB000076AB0EE674AA6EE264AB4EEC45AF1EE70
:106DC00010FAB0EE446A88BFB0EE646ABDEEC66ADF
:106DD00016EE108A16EE106AF045A8BF7646984562
:106DE000B8BF1E4606EE106AB8EEC66A022A81EDEA
:106DF000016A3CF412AF90ED086A9DED0E4A25EE53
:106E0000866AA4EE076AB0EE674AA6EE264AB4EE9A
:106E1000C45AF1EE10FAB0EE446A88BFB0EE646A6C
:106E2000BDEEC66A16EE108A16EE106AF045A8BFCF
:106E300076469845B8BF1E4606EE106AB8EEC66A9A
:106E4000032A81ED026A3CF4E8AE90ED0C6A9DEDF8
:106E50000F4A25EE866AA4EE076AB0EE674AA6EEF0
:106E6000264AB4EEC45AF1EE10FAB0EE446A88BF76
:106E7000B0EE646ABDEEC66A16EE108A16EE106AAF
:106E8000F045A8BF76469845B8BF1E4606EE106A84
:106E9000B8EEC66A042A81ED036A3CF4BEAE90EDFA
:106EA000106A9DED104A25EE866AA4EE076AB0EEE0
:106EB000674AA6EE264AB4EEC45AF1EE10FAB0EED6
:106EC000446A88BFB0EE646ABDEEC66A16EE108AE8
:106ED00016EE106AF045A8BF76469845B8BF1E4624
:106EE00006EE106AB8EEC66A052A81ED046A3CF423
:106EF00094AE90ED146A9DED114A25EE866AA4EEDB
:106F0000076AB0EE674AA6EE264AB4EEC45AF1EE1E
:106F100010FAB0EE446A88BFB0EE646ABDEEC66A8D
:106F200016EE108A16EE106AF045A8BF7646984510
:106F3000B8BF1E4606EE106AB8EEC66A062A81ED94
:106F4000056A3CF46AAE90ED186A9DED124A25EE92
:106F5000866AA4EE076AB0EE674AA6EE264AB4EE49
:106F6000C45AF1EE10FAB0EE446A88BFB0EE646A1B
:106F7000BDEEC66A16EE108A16EE106AF045A8BF7E
:106F800076469845B8BF1E4606EE106AB8EEC66A49
:106F9000072A81ED066A3CF440AE90ED1C6A9DED37
:106FA000134A65EE865AE7EE045AE6EEA57AB4EE89
:106FB000E75AF1EE10FAC8BFF0EE647AFCF71DBE96
:106FC0003E4B9FED3F6AB3F90020B3F9023007EE64
:106FD000902A06EE903AF8EEE77AF8EEE66A27EEA7
:106FE000E87A60EE277AA0EE267AE8EEA67A27EE17
:106FF000067A5DE47A1A99F802E082EAE27CACEB68
:10700000E27CF44540F31E8302EBD2720120521061
:10701000CBF8D0218BF8D4018BF8C801DBF8BC2168
:107020000A44B2F5FA6FA8BF4FF4FA62B2F57A7F5C
